:020000040800F2
:10000000A84C0020450100087F5F00081D5800082B
:100010007B5F00083D110008D16900080000000066
:100020000000000000000000000000006166000801
:100030004B11000800000000875F0008636600089D
:10004000E16900085F0100085F0100085F01000826
:100050005F0100085F0100084D1100087B110008D6
:10006000851100088F110008991100085F01000830
:100070005F0100085F0100085F0100085F010008E0
:100080005F0100085F0100085F0100085F010008D0
:100090005F0100085F0100085F010008A31100086C
:1000A0005F0100085F0100085F0100085F010008B0
:1000B0005F0100087D6600085F0100085F0100081D
:1000C0005F0100085F0100085F0100087962000815
:1000D00089620008A1690008B1690008C1690008C7
:1000E00057110008B15F00085F0100085F010008B8
:1000F0005F0100085F0100085F0100085F01000860
:100100005F0100085F0100085F01000899620008B4
:100110008D6600089D6600085F0100085F01000809
:100120005F0100085F0100085F0100085F0100082F
:10013000DFF80CD000F038FD004800470B2701081D
:10014000A84C00200648804706480047FEE7FEE727
:10015000FEE7FEE7FEE7FEE7FEE7FEE7FEE7FEE777
:100160006D660008310100082DE9F05F05460020AA
:1001700092469B4688460646814640241BE0284618
:1001800041464746224600F02FF853465A46C01AC9
:10019000914110D311461846224600F016F82D1A48
:1001A00067EB01084F4622460120002100F00DF8C0
:1001B00017EB00094E41201EA4F10104DFDC484684
:1001C00031462A464346BDE8F09F202A04DB203A08
:1001D00000FA02F1002070479140C2F1200320FA9A
:1001E00003F3194390407047202A04DB203A21FA98
:1001F00002F00021704721FA02F3D040C2F1200240
:10020000914008431946704700487047483D01082F
:1002100010B50446FFF7F8FF0068005D00F001002C
:1002200010BD40EA01039B0703D009E008C9121F73
:1002300008C0042AFAD203E011F8013B00F8013BA0
:10024000521EF9D27047D2B201E000F8012B491ECC
:10025000FBD270470022F6E710B513460A46044663
:100260001946FFF7F0FF204610BD30B505462A4677
:100270000B4612F8010B13F8014B08B1A042F8D05D
:100280001CB1002802D06D1CF1E7284630BDCAB26F
:10029000401E10F8011F8A4202D00029F9D1002027
:1002A0007047421C10F8011B0029FBD1801A7047CF
:1002B00030B505460020034600E05B1C934205D2A2
:1002C000EC5CC85C201A01D1002CF6D130BD70B5B1
:1002D00006460EF081FA046805460A2200213046DF
:1002E00000F0F4FA2C6070BDF0B480EA0102D40F83
:1002F0004200B2EB410F02D20246084611464A00C4
:1003000042D0C30DDDB2C1F3C752AD1A202D35DA8C
:10031000C1F3160141F4000204B15242C5F12006B6
:1003200002FA06F12A411044B3EBD05F23D0C4B1E6
:10033000012DA0EBC35009DCF0BC4FF0004202EAF3
:10034000C352DBB200F5000000F001BB400000F139
:10035000807000EBC350A0F1807040EAD17049007A
:1003600009E0490841EAC071A0EBC35000F5000064
:10037000400800EBC350F0BC00F0E0BA614201223B
:1003800002EB4101001BF6E7F0BC704781F0004131
:10039000AAE780F00040A7E780EA010210B502F06A
:1003A0000043400022D04A001FD0010E01EB126131
:1003B000C0F35600C2F3560240F4000042F40002BB
:1003C000A0FB022000047F39140400D0401C50EA36
:1003D000124001D44000491EC2B20C0604EBD010FA
:1003E000401C4008802A02D003E0002010BD20F00D
:1003F0000100002900DA0020184310BD30B480EA63
:10040000010202F0004530F0004221F0004013D01C
:1004100090B1C30DD40DC2F31601C0F31600E41A57
:1004200041F4000140F400027D34914201D3641C88
:1004300000E04900002C02DA30BC002070474FF485
:1004400000000023914201D3891A034340084FEA78
:100450004101F7D151B1914202D14FF0004105E085
:1004600002D24FF0010101E06FF0010103EBC45033
:10047000284430BC00F062BA2DE9FE4F804681EA84
:100480000300C00F0C46009021F0004123F000450E
:10049000B8EB0200A94105D24046214690461C46D1
:1004A0000B46024623F00040104347D0270DC7F308
:1004B0000A00C3F30A510290401A019040286BDAF7
:1004C000C3F3130040F4801B0098924620B1002330
:1004D000D2EB030A63EB0B0B01985946C0F14002C3
:1004E0005046FFF772FE06460D4650465946019AA1
:1004F00000F08CF910EB08006141002487EA1152EA
:1005000084EAE7731A4340D0009A62B3019A012A41
:100510004FEA075215DC001B61EB02014FF000426D
:1005200002EA0752CDE90042001C41F58011324633
:100530002B4600F049FA03B0BDE8F08F4046214653
:10054000F9E7001B61EB0201001C41F58013001864
:100550005B412018A2F5001747EB030140EAD57074
:10056000B6196D4111E06D084FEA360645EAC075CF
:100570004FEA0752001B61EB0201001C41F580119C
:1005800049084FEA30000019514132462B4603B06A
:10059000BDE8F04F00F009BA0098012240000023A6
:1005A000D0EB020263EBE073009821464FEAE0745F
:1005B000B8EB000061EB0401E9E783F000435BE77F
:1005C00081F0004158E72DE9F04D81EA030404F081
:1005D000004B21F0004514464FF0000A23F0004183
:1005E00050EA050220D054EA01021DD0C5F30A5793
:1005F0000246C5F31303C1F31300C1F30A5640F4D6
:10060000801543F48013A7EB0608101BD64608F2AA
:10061000FD3873EB050002D308F1010801E09218E0
:100620005B41B8F1000F03DA00200146BDE8F08D10
:1006300000204FF48011064684460EE0171B73EB32
:10064000050705D3121B63EB050306434CEA010CB7
:1006500049084FEA300092185B4150EA0107EDD19A
:1006600052EA030012D082EA040083EA050108433B
:1006700005D0101BAB4106D20122002306E0002268
:100680004FF0004302E06FF0010253101AEB060036
:100690004CEB085110EB0A0041EB0B01BDE8F04DAB
:1006A00000F083B9C10F80EAE0700844CA079623BE
:1006B000002100F04CB996230022114600F047B902
:1006C00030B4044696230800214604D0B62330BC3B
:1006D000002200F03CB920460021F8E70EB5C10F1A
:1006E00080EAE0700844CA07002140F233438DE8F5
:1006F0000E000A460B4600F067F903B000BD00F09B
:10070000004220F00040C10DC0F3160040F400008C
:100710007F2901DA00207047962903DCC1F1960198
:10072000C84001E096398840002AF4D04042704722
:1007300020F00040C10DC0F3160040F400007F29F6
:1007400001DA00207047962903DCC1F19601C84008
:10075000704796398840704700F0004230F0004002
:100760000AD0C10D01F56071C0F3160042EA0151D3
:10077000C20840071143704700200146704701F04E
:10078000004330B421F0004150EA010206D00A0DC6
:10079000A2F56072C1F31301002A02DC30BC002014
:1007A0007047440F44EAC104C100E01830BC00EBBC
:1007B000C25000F0C3B80000002801DBC0F10040C7
:1007C000002901DBC1F1004181427047002801DBB3
:1007D000C0F10040002901DBC1F1004188427047AF
:1007E00030B50B46014600202022012409E021FA01
:1007F00002F59D4205D303FA02F5491B04FA02F5FE
:100800002844151EA2F10102F1DC30BD202A06DBCE
:10081000CB17203A41FA02F043EAE07306E041FACE
:1008200002F3D040C2F120029140084319467047BC
:100830000FB4002300B589B00CA900910B996FF09B
:100840000042CB601E4B06931E4B07930423CDE959
:1008500001321D4A089202466B46002000F036FA2B
:1008600009B05DF814FB70B586B006464FF0FF3056
:100870000091CDE90101002015460C460490324656
:10088000694604A8FFF7D4FF03460498211825B150
:1008900008B10A4600E022462A6000280DD0002B4D
:1008A00002DD0098884208D0081B0094CDE90104BD
:1008B0003246694604A8FFF7BBFF06B070BD0000D2
:1008C000050F0008230F0008110200082DE9F0476A
:1008D00091460F4680460446002614F8015B2DB170
:1008E000FFF792FC0068405DC007F6D12B2D02D0C7
:1008F0002D2D18D0641E4A463946204600F022FBB2
:1009000027B13968A14201D1C7F8008071054FF0C5
:1009100002040BD54042002803DD0DF05DFF0460AA
:10092000A007BDE8F08746F48066E4E70028F8DA1F
:100930000DF052FF04606FF00040F2E70029A8BFFD
:100940007047401C490008BF20F00100704710B4F8
:10095000B0FA80FC00FA0CF050EA010404BF10BCAD
:10096000704749B1CCF1200421FA04F411FA0CF1DA
:1009700018BF012121430843A3EB0C01CB1D4FEA13
:1009800000614FEA102042BF002010BC704700EB0E
:10099000C35010440029A4BF10BC7047401C49003C
:1009A00008BF20F0010010BC704710B5141E73F191
:1009B000000408DA401C41F1000192185B411A431F
:1009C00001D120F0010010BD2DE9F04D92469B466B
:1009D00011B1B1FA81F202E0B0FA80F22032904611
:1009E000FFF7F3FB04460F4640EA0A0041EA0B0119
:1009F00053465A46084313D0114653EA010019D012
:100A0000C8F140025046FFF7EFFB05460E46504640
:100A100059464246FFF7D9FB084305D0012004E0C0
:100A200020463946BDE8F08D0020054346EAE076D1
:100A30002C4337430A986305E40AA0EB0800002220
:100A4000FD0A44EA47540A3002D500200146E9E78E
:100A5000010510196941DDE9084500196941BDE842
:100A6000F04DA2E72DE9FE4F81EA030404F00044B3
:100A700021F0004100944FF0000B23F0004350EAB6
:100A800001045ED052EA03045BD0C3F30A54C1F3FD
:100A90000A552C44A4F2F3340194A0FB0254C1F390
:100AA000130141F48011C3F3130343F4801301FBDA
:100AB000024400FB034E840A970A44EA815447EA41
:100AC0008357A4FB076802958D0A05FB07854FEA4B
:100AD000932C04FB0C542705029D4FEA065847EA65
:100AE0001637B5EB08056EEB070C870E920E47EA3A
:100AF000811742EA8312A7FB0201B6EB0B0164EBFC
:100B000000042B0D43EA0C335E1844EB1C50DA460C
:100B10005146E7FB0201C5F313044FEA0B3343EAE6
:100B200014534FEA0432019C43EA0603A4F10C0477
:100B30000294009CCDE900B4FFF746FF03B0BDE886
:100B4000F08F00200146F9E7C1F30A52C1F3130107
:100B500040F2FF3341F480119A4202DA002001464C
:100B6000704740F233439A42A2F2334202DC5242CF
:100B7000FFF73ABBFFF729BB30B5041E71F1000443
:100B800004DB4FF00044404264EB0101141E73F19A
:100B9000000405DB1C464FF00043524263EB0403A4
:100BA000994208BF904230BD064C074D06E0E06810
:100BB00040F0010394E8070098471034AC42F6D3A4
:100BC000FFF7BAFA043E0108243E01082DE9FF4F61
:100BD000087881B09946FF2805D0491C2D2804D0FB
:100BE0000024002308E000230BE00124F9E703EBD5
:100BF000830300EB4303491C0878FF28F7D104B1B5
:100C00005B4200200090147801462D2C01D02B2C43
:100C100004D1521C2D2C12D00024009400251678EB
:100C2000FF2E0ED00A24A0FB04C801FB048100277C
:100C300000FB0711521C16EB0C006941EFE7012481
:100C4000EBE7994450EA01020ED00024AA4D264653
:100C5000DFF8A88200F0D3F982468B46B9F1000094
:100C600009DAC9F100071BE001980021C0E9001171
:100C700005B0BDE8F08F074612E0F80707D022461E
:100C80002B4630464146FFF7EDFE06468846224693
:100C90002B4610461946FFF7E5FE04460D467F1029
:100CA000002FEAD1B9F1000F32464346504659466B
:100CB00002DAFFF788FC01E0FFF7D4FE009A0AB1E0
:100CC00081F00041019AC2E90001D1E72DE9FF4F0F
:100CD0001F468DB0D7E901464FF0FF382E2045461C
:100CE0004FF000090B90B9696D1C0E988847396A5E
:100CF000824688470028F6D1BAF1FF3F0AD024F493
:100D0000D064002E11DDBAF12B0F08D0BAF12D0FEF
:100D10000BD102E0404611B0ABE744F48064B969FE
:100D20006D1C0E9888478246761E6946600501D57F
:100D30002D2000E02B208DF8000001F1010B0DF1BA
:100D4000200809E0B9696D1C0E98884782460F9803
:100D500044F40074761E0560002E02DDBAF1300FF7
:100D6000F0D00B998A453ED144F0800406E00F99FB
:100D7000681CA9F1010944F400740860B9696D1C8C
:100D8000761E0E98884782463028F0D02BE00B99CB
:100D90008A4505D1200603D444F08004761E18E06D
:100DA00050460DF0EFFD08B30DF11301761E44F42B
:100DB00000748B4508D2AAF130000BF8010B200615
:100DC00007D5A9F1010003E0200602D409F10100D2
:100DD0008146A00502D50F99681C0860B9696D1C91
:100DE0000E9888478246002ED1DC53E0002E51DD5C
:100DF000BAF1650F02D0BAF1450F4BD1A00549D524
:100E0000B9696D1C24F44074761E0E98884782469A
:100E1000002E0CDD2B2804D0BAF12D0F07D144F49D
:100E20008074B9696D1C0E9888478246761EE0056D
:100E300001D52D2100E02B2108F8011BCDF82C80D5
:100E400021E00DF12901761E44F4007488450CD28E
:100E5000AAF1300010F0FF0088F8000002D10B99D1
:100E6000884509D908F1010806E0E00501D52448C4
:100E700001E042F20F708146B9696D1C0E988847F7
:100E800082460F980560002E04DD50460DF07AFD75
:100E90000028D6D1F9690E988847FF208BF800000A
:100EA00088F800000020069007904B466A4608A983
:100EB00006A8FFF78BFEA00502D46FF001002AE719
:100EC00014F0240F0AD0E00714D1DDE906123868C7
:100ED000031D3B600068C0E900120BE0DDE906017C
:100EE000FFF74DFC0146E00704D13868021D3A6067
:100EF0000068016028460EE7000024400000F03F33
:100F0000F1D8FFFF426842B1016811F8013B23B1FB
:100F1000521EC0E90012184670470121C160881EA8
:100F2000704742685AB1C368016843B983688B420D
:100F300005D0491E521CC0E90012002070474FF036
:100F4000FF3070472DE9F05F824600780027154694
:100F50008B460AF10104B946302801D09DB113E057
:100F600014F8010B0127782803D0582801D045B187
:100F70000AE00DB1102D07D10027102514F8010B40
:100F800002E0082500E00A250026B0460EE005FB39
:100F9000080005FB06F1012701EB10461FFA80F857
:100FA000B6F5803F00D3B94614F8010B294600F08E
:100FB00018F80028EBDABBF1000F05D00FB1641E62
:100FC00000E05446CBF80040B9F1000F06D00DF018
:100FD00003FC02210160C81EBDE8F09F48EA0640FC
:100FE000FAE73A2800D2303820F02002412A01D313
:100FF000A2F13700884201D34FF0FF3070470EB5A1
:1010000040F2334202920022CDE900221346FFF75C
:10101000DBFC03B000BD30B58C1810F8012B12F0CA
:101020000F0301D110F8013B120906D110F8012B72
:1010300003E010F8015B01F8015B5B1EF9D101E0F0
:1010400001F8013B521EFBD1A142E6D3002030BD86
:1010500070B5044600252068806800F0010018B3D0
:101060002068806820F001002168886001F0B2F8F3
:10107000054613E001F0AEF8401B02280ED92068A7
:10108000806800F0010048B1A06A40F01000A06242
:10109000E06A40F00100E062012070BD20688068D5
:1010A00000F001000028E5D10020F6E738B504463D
:1010B0000025002000902068806800F0010078BBC7
:1010C0002068806840F00100216888601948006845
:1010D0001949B0FBF1F0009002E00098401E00902A
:1010E00000980028F9D101F075F8054619E001F0E3
:1010F00071F8401B022814D92068806800F00100B4
:1011000078B9A06A40F01000A062E06A40F00100E7
:10111000E06200BF002084F8240000BF012038BD39
:1011200005E02068806800F001000028DFD0002082
:10113000F5E700000000002040420F0004E001201D
:101140000DF063FB0DF028FBF9E7704710B50120A7
:1011500000F084FE10BD10B54FF4806000F07EFEFC
:101160004FF4006000F07AFE4FF4805000F076FEFD
:101170004FF4005000F072FE10BD10B5022000F0D8
:101180006DFE10BD10B5042000F068FE10BD10B556
:10119000082000F063FE10BD10B5102000F05EFEC8
:1011A00010BD7047F8B5044600260020009000BF2F
:1011B00094F82400012801D10220F8BD012084F810
:1011C000240000BF2046FFF743FF0646002E6CD1E7
:1011D000A06A20F4885040F00200A062022002F0D1
:1011E0002FF935490968B1FBF0F04000009002E0AA
:1011F0000098401E009000980028F9D12046FFF783
:1012000055FF2068806840F008002168886000F081
:10121000E1FF054616E000F0DDFF401B0A2811D96A
:101220002068806800F0080060B1A06A20F0020029
:1012300040F01000A06200BF002084F8240000BF2E
:101240000120BAE72068806800F008000028E2D199
:101250002068806840F004002168886000F0BAFFD0
:10126000054616E000F0B6FF401B0A2811D9206899
:10127000806800F0040060B1A06A20F0020040F035
:101280001000A06200BF002084F8240000BF0120ED
:1012900093E72068806800F004000028E2D1A06A8B
:1012A00020F0020040F00100A06200BF002084F89E
:1012B000240000BF304680E70000002038B5024619
:1012C00000230020009000BF92F82400012801D1E3
:1012D000022038BD012082F8240000BF486807289A
:1012E00012D21068406B0C79641E04EB84051F2435
:1012F000AC40A0430D796D1E05EB85050C68AC4034
:1013000020431468606327E048680D2812D21068F3
:10131000006B0C79E41F04EB84051F24AC40A04350
:101320000D79ED1F05EB85050C68AC402043146872
:10133000206311E01068C06A0C790D3C04EB840551
:101340001F24AC40A0430D790D3D05EB85050C68CD
:10135000AC4020431468E06208680A2812D3106881
:10136000C0680C780A3C04EB44050724AC40A04359
:101370000D780A3D05EB45058C68AC4020431468A8
:10138000E0600FE0106800690C7804EB4405072466
:10139000AC40A0430D7805EB45058C68AC4020437C
:1013A000146820610868102802D00868112827D125
:1013B000174C1068A0421ED11068806800F400002D
:1013C000F0B91068806840F400001468A0600868F4
:1013D000102815D10F4800680F4CB0FBF4F000EB5B
:1013E00080004000009002E00098401E00900098AD
:1013F0000028F9D104E0906A40F0200090620123B7
:1014000000BF002082F8240000BF184661E70000FA
:10141000002401400000002040420F000146886A7D
:10142000704701460868C06C704700002DE9F04124
:101430000446002700250026A84614B90120BDE86F
:10144000F081A06810B1207D00B100BFA06A30B962
:101450000020E06284F82400204600F097F820463F
:10146000FFF7F6FD0746A06A00F01000002873D1D0
:10147000002F7ED1A06A20F4885040F00200A062C4
:101480003F4AD4E90001904208D1E069B0F5402F0D
:1014900002D14FF4002002E0E06900E0E06901437E
:1014A000207B41EA40000643A068B0F5807F02D06F
:1014B000A068012802D14FF4807000E000200543AD
:1014C000207D012811D1207B38B9A069401E4FF43E
:1014D000006141EA4030054307E0A06A40F0200087
:1014E000A062E06A40F00100E0622068406820F4F9
:1014F0006940284321684860206880682149084085
:10150000304321688860A068B0F5807F02D0A06871
:10151000012802D14FF4807000E00020B0F5807FF8
:1015200003D1208A401E4FEA00582068C06A20F488
:10153000700040EA08002168C8622068806812498B
:101540000840B04209D10020E062A06A20F0020009
:1015500040F00100A06211E00BE0A06A20F0020060
:1015600040F01000A062E06A40F00100E062012754
:1015700004E0A06A40F01000A062012738465EE750
:10158000003C0140FDF7E1FFFE0E1FFF10B58CB0DF
:101590000446022002908003049002A801F0EAFFB2
:1015A0007C49206888427DD100BF7B48806940F437
:1015B0000070794988610846806900F400700190E4
:1015C00000BF00BF00BF0846806940F0040088618A
:1015D0000846806900F00400019000BF00BF0220AF
:1015E00008900320099000200A9008A96B4800F099
:1015F00043FC00BF6848806940F004006649886188
:101600000846806900F00400019000BF00BF102070
:1016100008900320099000200A9008A95F4800F074
:101620002BFC00BF5C48806940F004005A49886187
:101630000846806900F00400019000BF00BF202030
:1016400008900320099000200A9008A9534800F050
:1016500013FC00BF5048806940F004004E49886187
:101660000846806900F00400019000BF00BF4020E0
:1016700008900320099000200A9008A9474800F02C
:10168000FBFB00BF4448806940F004004249886188
:101690000846806900F00400019000BF00BF802070
:1016A000089000E050E00320099000200A9008A96B
:1016B0003A4800F0E1FB00BF3748806940F008007D
:1016C000354988610846806900F00800019000BF34
:1016D00000BF012008900320099000200A9008A96B
:1016E0002F4800F0C9FB00BF2B48806940F008007C
:1016F000294988610846806900F00800019000BF10
:1017000000BF022008900320099000200A9008A939
:10171000234800F0B1FB00BF1F48806940F0100073
:101720001D4988610846806900F01000019000BFE3
:1017300000BF012008900320099000200A9008A90A
:10174000184800F099FB23E01749206888420DD122
:1017500000BF1148806940F480600F4988610846E5
:10176000806900F48060019000BF11E00F4920689B
:1017700088420DD100BF0848806940F40040064906
:1017800088610846806900F40040019000BF00BFF6
:101790000CB010BD002401400010024000080140C0
:1017A000000C01400010014000280140003C0140B5
:1017B000F8B504460D46002600200090002700F0F2
:1017C00009FD06462068806800F4807050B1A06A68
:1017D00040F02000A06200BF002084F8240000BF79
:1017E0000120F8BD2068406800F4807020BB2068AC
:1017F000C06A00F47000F8B917E0681CA8B125B100
:1018000000F0E8FC801BA8420FD92068006800F0B7
:10181000020050B9A06A40F00400A06200BF00209E
:1018200084F8240000BF0320DBE72068006800F094
:1018300002000028E1D053E0022001F001FE384907
:101840000968B1FBF0F021680969364A114091B985
:101850002168C9689211114069B921680969324A41
:10186000114031B92168C9689211114009B9142198
:1018700017E0292115E0216809692B4A114021B997
:101880002168C9689211114041B121680969274A4C
:10189000114029B92168C968114009B9542100E0F3
:1018A000FC2100FB01F718E0681C98B125B100F09D
:1018B00091FC801BA8420DD90098B8420AD2A06AB8
:1018C00040F00400A06200BF002084F8240000BFA4
:1018D000032086E70098401C00900098B842E3D3AC
:1018E0006FF0120021680860A06A40F40070A062E6
:1018F0002068806800F46020B0F5602F0DD1207B57
:1019000058B9A06A20F48070A062A06A00F48050E8
:1019100018B9A06A40F00100A062002061E7000051
:101920000000002024499224922449124992240064
:1019300070B50446002500BF94F82400012801D1A9
:10194000022070BD012084F8240000BF2046FFF76C
:10195000ADFB0546002D77D1A06A40F201218843F6
:1019600040F48070A0623C492068884208D13B481E
:10197000006800F4702008B9012002E0002000E0B7
:10198000012078B1A06A20F48010A062206840682D
:1019900000F4806000B3A06A20F4005040F480504E
:1019A000A06219E0A06A40F48010A0622B49091FD0
:1019B0002068884203D028492068884204D12748FB
:1019C000006800F4806000E0002028B1A06A20F4E4
:1019D000005040F48050A062A06A00F4805020B112
:1019E000E06A20F00600E06201E00020E06200BF53
:1019F000002084F8240000BFC01E21680860206811
:101A0000806800F46020B0F5602F16D1124920687C
:101A1000884208D11148006800F4702008B90120FC
:101A200002E0002000E0012038B12068806840F426
:101A3000A000216888600CE006E02068806840F41F
:101A400080102168886004E000BF002084F8240032
:101A500000BF284675E7000000280140042401402B
:101A600070B50446002500BF94F82400012801D178
:101A7000022070BD012084F8240000BF2046FFF73B
:101A8000E7FA05462DB9A06A20F4885040F001001D
:101A9000A06200BF002084F8240000BF2846E8E7C9
:101AA0000146002291F82100022808D00420886312
:101AB00000BF002081F8200000BF012070470868A7
:101AC000006820F00E000B6818600868006820F0BD
:101AD00001000B68186091F8403001209840CB6BF2
:101AE0005860012081F8210000BF002081F820000B
:101AF00000BF1046E2E7000070B50446002594F8E8
:101B00002100022803D00420A0630125C1E0206841
:101B1000006820F00E00216808602068006820F04E
:101B20000100216808605C492068884252D95A49FE
:101B300078392068884201D1012047E0564964394C
:101B40002068884201D1102040E053495039206874
:101B5000884201D1801539E04F493C3920688842DC
:101B600001D1801432E04C4928392068884202D1E2
:101B70004FF480302AE0484914392068884202D165
:101B80004FF4801022E044492068884201D140048B
:101B90001CE042492068884201D1012016E03F49FB
:101BA00014312068884201D110200FE03B492831D0
:101BB0002068884201D1801508E038493C3120680E
:101BC000884201D1801401E04FF480303349091F6D
:101BD000086051E0304978392068884201D10120FD
:101BE00047E02D4964392068884201D1102040E047
:101BF000294950392068884201D1801539E02649A9
:101C00003C392068884201D1801432E022492839C9
:101C10002068884202D14FF480302AE01E491439EE
:101C20002068884202D14FF4801022E01A492068CF
:101C3000884201D140041CE018492068884201D143
:101C4000012016E0154914312068884201D1102086
:101C50000FE0124928312068884201D1801508E040
:101C60000E493C312068884201D1801401E04FF4D4
:101C70008030094980394860012084F8210000BF84
:101C8000002084F8200000BF606B10B12046616B1B
:101C90008847284670BD00008000024008040240CA
:101CA00070B5044600F096FA06462546681C10B149
:101CB00004480078054400BF00F08CFA801BA8425D
:101CC000FAD370BD0C0000202DE9F04102460B460E
:101CD00000208BE00127874007EA030100297DD01F
:101CE000464F4FEA900C57F82C4087074FEA177C75
:101CF0000F2707FA0CF73C40414FBA4201D10027A9
:101D000019E0404FBA4201D1012714E03E4FBA42D8
:101D100001D102270FE03D4FBA4201D103270AE06B
:101D20003B4FBA4201D1042705E03A4FBA4201D1F4
:101D3000052700E006274FEA807C4FEA1C7C07FA63
:101D40000CF7A74230D187074FEA177C0F2707FA15
:101D50000CF42A4F4FEA900C57F82C70A743DFF889
:101D60009CC04FEA90084CF828702B4F3F688F4377
:101D7000DFF8A4C0CCF800700CF104073F688F4373
:101D80000CF1040CCCF800700CF104073F688F4391
:101D90000CF1040CCCF800700CF104073F688F4381
:101DA0000CF1040CCCF80070FF2901D8174600E0B4
:101DB000171D3D46FF2901D8870002E0A0F1080762
:101DC000BF003E462F684FF00F0C0CFA06FC27EAC6
:101DD0000C074FF0040C0CFA06FC00E005E047EAA3
:101DE0000C072F60D7688F43D760401C23FA00F799
:101DF000002F7FF46FAFBDE8F081000008000140C4
:101E000000080140000C0140001001400014014096
:101E100000180140001C01400004014010B50446B8
:101E2000B4F5806F0ED0B4F5006F0BD0B4F5805FC1
:101E300008D0B4F5005F05D0B4F5804F02D0B4F5FA
:101E4000004F07D1044890F83000012802D1024920
:101E5000486B804710BD00008C02002010B504467E
:101E600004480068204020B1024804602046FFF783
:101E7000D5FF10BD140401402DE9F84702460023A8
:101E80009C467BE14FF0010808FA03F4D1F800808A
:101E900008EA0400A0427DD1DFF8F4A2D1F8048062
:101EA000A8EB0A09D0453AD014DCB8F1030F50D0A2
:101EB00009DCB8F1000F31D0B8F1010F1CD0B8F136
:101EC000020F49D120E0B8F1110F18D0B8F1120F6C
:101ED00042D11EE0B9F5881F25D006DCB9F5803F58
:101EE00020D0B9F5801F37D11AE0B9F5001F18D0FE
:101EF000B9F5041F30D117E0D1F80CC02DE0D1F8AE
:101F00000C8008F1040C28E0D1F80C8008F1080CD2
:101F100023E0D1F80C8008F10C0C1EE000BF00BFDC
:101F200000BF00BF00BF00BFD1F80880B8F1000FAC
:101F300002D14FF0040C0BE0D1F80880B8F1010F8A
:101F400003D14FF0080C146102E04FF0080C54610B
:101F500003E04FF0000C00E000BF00BFFF2801D8F5
:101F6000904601E002F104084646FF2802D84FEAF5
:101F7000830803E0A3F108084FEA88084746D6F82B
:101F800000804FF00F0909FA07F928EA09080CFA4E
:101F900007F900E07AE048EA0908C6F80080D1F8BD
:101FA000048008F08058B8F1805F6FD100BFDFF87F
:101FB000E481D8F8188048F00108DFF8D891C9F812
:101FC0001880C846D8F8188008F00108CDF80080BD
:101FD00000BF00BF4FEAB9384FEA930958F82950BB
:101FE0004FEA83784FEA18794FF00F0808FA09F89A
:101FF00025EA0805DFF8A081424502D14FF000082C
:1020000024E0DFF89881424502D14FF001081DE03D
:10201000DFF88C81424502D14FF0020816E0DFF86C
:102020008481424502D14FF003080FE0DFF8788148
:10203000424502D14FF0040808E0DFF870814245C4
:1020400002D14FF0050801E04FF006084FEA83790E
:102050004FEA197908FA09F848EA0505DFF85081CE
:102060004FEA930948F82950D1F8048008F48038E1
:10207000B8F5803F0BD1DFF83C81D8F8008048EA02
:102080000008DFF83091C9F800800AE075E0DFF859
:102090002481D8F8008028EA0008DFF81891C9F8F0
:1020A0000080D1F8048008F40038B8F5003F0ED164
:1020B000DFF8008108F10408D8F8008048EA000839
:1020C000DFF8F09009F10409C9F800800DE0DFF8AD
:1020D000E48008F10408D8F8008028EA0008DFF856
:1020E000D49009F10409C9F80080D1F8048008F4FB
:1020F0008018B8F5801F0ED1DFF8B88008F1080805
:10210000D8F8008048EA0008DFF8A89009F108092B
:10211000C9F800800DE0DFF89C8008F10808D8F8C5
:10212000008028EA0008DFF88C9009F10809C9F856
:102130000080D1F8048008F40018B8F5001F0ED113
:10214000DFF8708008F10C08D8F8008048EA000831
:10215000DFF8609009F10C09C9F800800DE0DFF8A4
:10216000548008F10C08D8F8008028EA0008DFF84D
:10217000449009F10C09C9F800805B1CD1F800807B
:1021800028FA03F8B8F1000F7FF47CAEBDE8F887B9
:10219000000011100010024000080140000C014036
:1021A000001001400014014000180140001C0140D3
:1021B0000800014000040140024693680B400BB147
:1021C000012000E0002070470AB1016101E00B042A
:1021D0000361704701480068704700000400002058
:1021E00010B504460CB9012010BD242084F83D0030
:1021F0002068006820F0010021680860204600F097
:10220000BDFD0020206484F83D00206384F83E007A
:1022100000BF84F83C0000BF00BFE5E770B504468E
:102220000CB9012070BD94F83D0028B9002084F855
:102230003C00204600F0F2FD242084F83D00206898
:10224000006820F00100216808602068006840F400
:102250000040216808602068006820F40040216880
:10226000086001F0EBFA05465C496068884206D8D0
:102270005B48854201D2012007E0002005E0594873
:10228000854201D2012000E00020012800D1C9E7E9
:102290005548B5FBF0F62068406820F03F00304319
:1022A000216848604D496068884201D8701C07E089
:1022B0004FF4967070434FF47A71B0FBF1F0401C0C
:1022C0002168096A21F03F010843216808624349F7
:1022D0006068884214D8681E61684900B0FBF1F05C
:1022E000401CC0F30B00042801D204203DE0681E0E
:1022F00061684900B0FBF1F0401CC0F30B0034E012
:10230000A06838B9681E616801EB4101B0FBF1F0CB
:10231000401C0AE0681E616801EBC10202EB01117A
:10232000B0FBF1F0401C40F48040C0F30B0008B952
:1023300001201AE0A06848B9681E616801EB4101FC
:10234000B0FBF1F0401CC0F30B000CE0681E6168AC
:1023500001EBC10202EB0111B0FBF1F0401CC0F334
:102360000B0040F4804040F400402168C9694CF6FD
:10237000FF72914308432168C861D4E9070108430B
:102380002168096821F0C001084321680860D4E988
:10239000031008432168896848F2FF3291430843DB
:1023A00021688860D4E9050108432168C96821F0E3
:1023B000FF0108432168C8602068006840F0010000
:1023C0002168086000202064202084F83D0000205F
:1023D000206384F83E0000BF24E70000A0860100CF
:1023E00080841E0000093D0040420F002DE9FC479B
:1023F00004468946174698460A9E00200190FFF73A
:10240000E9FE054694F83D0020286FD119230122EA
:10241000C8492046009503F071FC10B10220BDE8C8
:10242000FC8700BF94F83C00012801D10220F6E7A8
:10243000012084F83C0000BF2068006800F0010023
:1024400028B92068006840F0010021680860206811
:10245000006820F4006021680860222084F83D00B4
:10246000102084F83E00002020646762A4F82A80CF
:10247000608D2085B048E0622B46324649462046B2
:1024800003F0F2F908B10120C9E7208D88B900BF37
:1024900000200090206840690090206880690090CA
:1024A00000BF00BF2068006840F400702168086029
:1024B0004BE0208D01281AD12068006820F480604C
:1024C0002168086072B600BF002000902068406953
:1024D000009020688069009000BF00BF20680068FD
:1024E00040F400702168086062B62EE020E1208D83
:1024F000022819D12068006840F400602168086053
:1025000072B600BF002000902068406900902068EB
:102510008069009000BF00BF2068006820F48060E0
:102520002168086062B610E02068006840F48060AE
:102530002168086000BF002000902068406900907A
:1025400020688069009000BF00BFE2E0208D032872
:102550007ED8208D012815D12A463146204603F029
:1025600072FC08B101205AE720680069616A0870AE
:10257000606A401C6062208D401E2085608D401E78
:102580006085C6E0208D02282CD1334600226B499D
:102590002046009503F0B2FB08B101203FE772B678
:1025A0002068006840F400702168086020680069B5
:1025B000616A0870606A401C6062208D401E208540
:1025C000608D401E608562B620680069616A08708F
:1025D000606A401C6062208D401E2085608D401E18
:1025E000608596E03346002254492046009503F06A
:1025F00085FB08B1012012E72068006820F48060A4
:102600002168086072B620680069616A0870606AB3
:10261000401C6062208D401E2085608D401E6085BC
:10262000474800681921B0FBF1F04FF47A71B0FB14
:10263000F1F0C0EBC00000EB8000019000BF0198FA
:10264000401E01900198A8B900202063202000E0DE
:1026500038E084F83D00002084F83E00206C40F013
:102660002000206462B600BF002084F83C0000BF58
:102670000120D4E620684069C0F380000028DED045
:102680002068006840F400702168086020680069D4
:10269000616A0870606A401C6062208D401E20855F
:1026A000608D401E608562B620680069616A0870AE
:1026B000606A401C6062208D401E2085608D401E37
:1026C000608526E02A463146204603F0BCFB08B16F
:1026D0000120A4E620680069616A0870606A401CF5
:1026E0006062208D401E2085608D401E60852068C0
:1026F0004069C0F3800060B120680069616A0870B9
:10270000606A401C6062208D401E2085608D401EE6
:102710006085208D00287FF419AF202084F83D00CB
:10272000002084F83E0000BF84F83C0000BF76E63D
:10273000022074E6020010000000FFFF0400010008
:10274000000000202DE9F8430446894616461F463E
:10275000DDF82080FFF73EFD054694F83D00202877
:102760007ED11923012251492046009503F0C6FA73
:1027700010B10220BDE8F88300BF94F83C000128A6
:1027800001D10220F6E7012084F83C0000BF206858
:10279000006800F0010028B92068006840F00100DE
:1027A000216808602068006820F4006021680860E3
:1027B000212084F83D00102084F83E000020206491
:1027C00066626785608D20853948E0622B46424607
:1027D0004946204603F0E4F808B10120CAE700BFEB
:1027E0000020009020684069009020688069009077
:1027F00000BF00BF44E02A464146204603F08FFB5D
:1028000050B1206C042805D12068006840F40070A5
:10281000216808600120ADE7606A007821680861DE
:10282000606A401C6062608D401E6085208D401E85
:10283000208520684069C0F3800070B1208D60B1B0
:10284000606A007821680861606A401C6062608D7F
:10285000401E6085208D401E20852A46414600E0AE
:1028600022E0204603F01CFA50B1206C042805D168
:102870002068006840F4007021680860012079E752
:10288000208D0028B7D12068006840F400702168CE
:102890000860202084F83D00002084F83E0000BF3E
:1028A00084F83C0000BF65E7022063E702001000E7
:1028B0000000FFFF2DE9FE4F04460F469046994663
:1028C000DDE90CAB0E9E00200290FFF783FC05466D
:1028D00094F83D00202872D119230122CA492046CC
:1028E000009503F00BFA10B10220BDE8FE8F00BF87
:1028F00094F83C00012801D10220F6E7012084F879
:102900003C0000BF2068006800F0010028B9206882
:10291000006840F00100216808602068006820F429
:10292000006021680860222084F83D00402084F87F
:102930003E0000202064C4F824A0A4F82AB0608DD2
:102940002085B248E0624B46424639462046CDE9F2
:10295000006503F085F808B10120C6E7208D88B92D
:1029600000BF0020019020684069019020688069C4
:10297000019000BF00BF2068006840F4007021682B
:1029800008604BE0208D01281AD12068006820F4EF
:1029900080602168086072B600BF00200190206846
:1029A0004069019020688069019000BF00BF2068E5
:1029B000006840F400702168086062B62EE020E1F3
:1029C000208D022819D12068006840F40060216839
:1029D000086072B600BF0020019020684069019035
:1029E00020688069019000BF00BF2068006820F463
:1029F00080602168086062B610E02068006840F4DA
:102A000080602168086000BF002001902068406954
:102A1000019020688069019000BF00BFE2E0208D36
:102A200003287DD8208D012815D12A46314620461D
:102A300003F009FA08B1012057E720680069616ACC
:102A40000870606A401C6062208D401E2085608D89
:102A5000401E6085C6E0208D02282CD1334600221E
:102A60006B492046009503F049F908B101203CE785
:102A700072B62068006840F4007021680860206821
:102A80000069616A0870606A401C6062208D401EA7
:102A90002085608D401E608562B620680069616A8D
:102AA0000870606A401C6062208D401E2085608D29
:102AB000401E608596E03346002255492046009529
:102AC00003F01CF908B101200FE72068006820F42A
:102AD00080602168086072B620680069616A0870C9
:102AE000606A401C6062208D401E2085608D401E03
:102AF0006085484800681921B0FBF1F04FF47A7105
:102B0000B0FBF1F0C0EBC00000EB8000029000BF12
:102B10000298401E02900298A8B90020206300E0AD
:102B200039E0202084F83D00002084F83E00206C2D
:102B300040F02000206462B600BF002084F83C0012
:102B400000BF0120D1E620684069C0F38000002862
:102B5000DED02068006840F40070216808602068BA
:102B60000069616A0870606A401C6062208D401EC6
:102B70002085608D401E608562B620680069616AAC
:102B80000870606A401C6062208D401E2085608D48
:102B9000401E608526E02A463146204603F053F960
:102BA00008B10120A1E620680069616A0870606AC6
:102BB000401C6062208D401E2085608D401E608517
:102BC00020684069C0F3800060B120680069616AD4
:102BD0000870606A401C6062208D401E2085608DF8
:102BE000401E6085208D00287FF419AF202084F8D6
:102BF0003D00002084F83E0000BF84F83C0000BF88
:102C000073E6022071E60000020010000000FFFFE2
:102C100004000100000000202DE9FC5F04460F467F
:102C200090469946DDE90CAB0E9EFFF7D3FA0546B8
:102C300094F83D0020287DD1192301224D492046DA
:102C4000009503F05BF810B10220BDE8FC9F00BFC7
:102C500094F83C00012801D10220F6E7012084F815
:102C60003C0000BF2068006800F0010028B920681F
:102C7000006840F00100216808602068006820F4C6
:102C8000006021680860212084F83D00402084F81D
:102C90003E0000202064C4F824A0A4F82AB0608D6F
:102CA00020853548E0624B46424639462046CDE90C
:102CB000006502F085FF08B10120C6E731E02A4631
:102CC0003146204603F02BF950B1206C042805D181
:102CD0002068006840F40070216808600120B4E7B3
:102CE000606A007821680861606A401C6062208D1B
:102CF000401E2085608D401E608520684069C0F3BD
:102D0000800070B1208D60B1606A00782168086130
:102D1000606A401C6062208D401E2085608D401ED0
:102D20006085208D0028CAD12A463146204602F00F
:102D3000B7FF00E01CE050B1206C042805D12068EA
:102D4000006840F400702168086001207DE7206879
:102D5000006840F4007021680860202084F83D007D
:102D6000002084F83E0000BF84F83C0000BF6CE700
:102D700002206AE7020010000000FFFF10B50446C1
:102D80002049206888421BD11F48006940F4001088
:102D90001D4908610846006920F4001008610846D2
:102DA000C06920F40010C861002018490870402153
:102DB0001748FEF789FF80211548FEF785FF20E0C0
:102DC0001449206888421CD10F48006940F48000F3
:102DD0000D4908610846006920F480000861084632
:102DE000C06920F48000C86100200B4908704FF4CE
:102DF00080610748FEF768FF4FF400610448FEF762
:102E000063FF10BD00540040001002401600002077
:102E1000000C0140005800401700002010B586B09B
:102E200004464049206888423AD100BF3E48806944
:102E300040F008003C4988610846806900F00800BD
:102E4000019000BF00BF00BF0846806940F0080045
:102E500088610846806900F00800019000BF00BF4B
:102E600000BF0846C06940F40010C8610846C06948
:102E700000F40010019000BF00BF4020029012201B
:102E80000390012004900320059002A92748FEF733
:102E9000F3FF8020029002A92448FEF7EDFF3EE0F8
:102EA0002349206888423AD100BF1F48806940F01A
:102EB00008001D4988610846806900F008000190FB
:102EC00000BF00BF00BF0846806940F0080088616D
:102ED0000846806900F00800019000BF00BF00BFF5
:102EE0000846C06940F48000C8610846C06900F423
:102EF0008000019000BF00BF0815029012200390CF
:102F0000012004900320059002A90848FEF7B4FFB1
:102F10004FF40060029002A90448FEF7ADFF06B02E
:102F200010BD00000054004000100240000C0140A1
:102F3000005800402DE9F84304460D4616461F464A
:102F4000FFF748F9804694F83D0020287ED105B16E
:102F500016B90120BDE8F88300BF94F83C000128B1
:102F600001D10220F6E7012084F83C0000BF206870
:102F7000006800F0010028B92068006840F00100F6
:102F8000216808602068006820F4006021680860FB
:102F9000222084F83D00202084F83E000020206498
:102FA00065626685608D20854048E0622068006823
:102FB00040F48060216808603B4600223C4920467E
:102FC000CDF8008002F09AFE08B10120C2E700BFF0
:102FD000002000902068406900902068806900907F
:102FE00000BF00BF2EE042463946204602F02BFFCC
:102FF00038B12068006820F48060216808600120F2
:10300000A8E720680069616A0870606A401C606215
:10301000208D401E2085608D401E6085206840699F
:10302000C0F3800070B1208D60B120680069616AD2
:103030000870606A401C6062208D401E2085608D93
:10304000401E6085208D0028CDD100E02CE0424656
:103050003946204602F037FF38B12068006820F476
:10306000806021680860012074E700BF00200090A4
:103070002068406900902068006840F001002168E5
:10308000086000BF00BF2068006820F480602168ED
:103090000860202084F83D00002084F83E0000BF36
:1030A00084F83C0000BF55E7022053E70000FFFF13
:1030B000020001002DE9F84304460E4617469846E3
:1030C000FFF788F8054694F83D00202871D106B135
:1030D00017B90120BDE8F88300BF94F83C0001282F
:1030E00001D10220F6E7012084F83C0000BF2068EF
:1030F000006800F0010028B92068006840F0010075
:10310000216808602068006820F400602168086079
:10311000212084F83D00202084F83E000020206417
:1031200066626785608D20854548E062206800689A
:1031300040F48060216808604346002241492046EF
:10314000009502F0DBFD08B10120C3E700BF0020BD
:10315000009020684069009020688069009000BF5E
:1031600000BF2069B0F5404F14D1434600223549D5
:103170002046009502F0C2FD08B10120AAE700BF79
:1031800000200090206840690090206880690090CD
:1031900000BF00BF2FE02A464146204602F0BFFE96
:1031A00040B12068006820F4806021680860012038
:1031B00090E743E0606A007821680861606A401C1B
:1031C0006062608D401E6085208D401E20852068D5
:1031D0004069C0F3800070B1208D60B1606A0078F2
:1031E00021680861606A401C6062608D401E6085D5
:1031F000208D401E2085208D0028CCD14346002202
:103200004FF482312046009502F078FD08B101208C
:1032100060E76FF48060216848612068006820F4EE
:10322000806021680860202084F83D00002084F838
:103230003E0000BF84F83C0000BF4BE7022049E796
:103240000000FFFF020001000348006803490978FD
:103250000844014908607047040000200C00002069
:1032600010B50848006840F01000064908600320C7
:1032700000F0A2F80F2000F007F800F02BF8002073
:1032800010BD00000020024070B504460E480078D2
:103290004FF47A71B1FBF0F00C490968B1FBF0F51D
:1032A000284601F016FC08B1012070BD102C07D291
:1032B00000222146501E00F041F80548046001E05C
:1032C0000120F2E70020F0E70C00002000000020C1
:1032D000080000207047000010B50146084600288D
:1032E00017DB00F01F0301229A400B4B440943F8FF
:1032F000242000BF00BF00BFBFF34F8F00BF00BF3F
:1033000000BF00BF00BF00BFBFF36F8F00BF00BF93
:1033100000BF00BF10BD000080E100E0014608468C
:10332000002809DB00F01F0301229A4043099B009B
:1033300003F1E023C3F8002100BF70472DE9F05FDF
:1033400080460D46164600270BF00AFA0746394616
:103350002A46334601F00700C0F1070ABAF1040F0C
:1033600002D94FF0040A01E0C0F1070AD14600F18A
:10337000040ABAF1070F02D24FF0000A01E0A0F1EF
:10338000030AD4464FF0010A0AFA09FAAAF1010A1F
:103390000AEA020A0AFA0CFA4FF0010B0BFA0CFBCC
:1033A000ABF1010B0BEA030B4AEA0B042146404642
:1033B0000BF0DEF9BDE8F09F00BF00F00702064BFE
:1033C00019684FF6FF031940044B0B4343EA0221EF
:1033D000014B196000BF70470CED00E00000FA05DA
:1033E000012001490862704700000E4270B5044692
:1033F0000D461148006820F002000F490860084699
:10340000006820F00100204308600C48006840F08C
:1034100004000A490860012D01D130BF04E040BF1B
:1034200002F0AEFD02F0ACFD0448006820F004009C
:103430000249086070BD00000070004010ED00E01F
:103440002DE9F04385B0064642A30FCB01AC0FC473
:1034500044A0006800904FF00008002500270024D9
:10346000A146042E36D004DC012E3BD0022E6BD1B7
:103470005FE0082E32D0102E66D13B4844680068C9
:1034800000F0807000B301A8C4F38341475C04F4EA
:10349000803070B134484068C0F340401DF800806F
:1034A00004F4803040B13148B0FBF8F000FB07F580
:1034B00002E02F4807FB00F52B48406800F480002D
:1034C000B0F5800F01D1A94603E068000321B0FBED
:1034D000F1F93AE000F0D2F9814636E000F0CEF999
:1034E000814632E02048046A04F44070B0F5807FE1
:1034F00005D104F0020010B14FF4004918E004F4C3
:103500004070B0F5007F07D11748406A00F0020014
:1035100010B149F640490BE004F44070B0F5407F2B
:1035200006D11148006800F4003008B14FF2244978
:103530000BE000F093F90C494968C1F38131491C53
:103540004900B0FBF1F900E000BF00BF484605B0FC
:10355000BDE8F08302030405060708090A0B0C0DF9
:103560000E0F1010010200000010024000127A003D
:1035700000093D00F8B5044600260025207800F03B
:10358000010000286BD000274348C06900F080503C
:1035900070B900BF4048C06940F080503E49C861E2
:1035A0000846C06900F08050009000BF00BF0127AE
:1035B0003A48006800F48070B0B93848006840F4B8
:1035C000807036490860FEF705FE064606E0FEF705
:1035D00001FE801B642801D90320F8BD2F48006834
:1035E00000F480700028F2D02B48006A00F4407587
:1035F0002DB3A08800F44070A84220D02648006A6D
:1036000020F4407501202649086000200860224807
:10361000056205F0010090B1FEF7DCFD064608E00A
:10362000FEF7D8FD801B41F28831884201D9032082
:10363000D3E71948006A00F002000028F0D01648CD
:10364000006A20F440706168084313490862012F42
:1036500004D10846C06920F08050C86100BF2078BE
:1036600000F00200022807D10B48406820F44040D7
:10367000A168084308494860207800F0100010282D
:1036800007D10548406820F4800061690843024979
:1036900048600020A1E700000010024000700040D8
:1036A0004004424270B504460D460CB9012070BD7D
:1036B0005A48006800F00700A8420ED25748006838
:1036C00020F007002843554908600846006800F0CC
:1036D0000700A84201D00120E9E7207800F00200AD
:1036E00002281DD1207800F00400042805D14C48A0
:1036F000406840F4E0604A494860207800F00800E3
:10370000082805D14648406840F460504449486064
:103710004348406820F0F000A168084340494860F1
:10372000207800F0010078B36068012806D13C4899
:10373000006800F4003090B90120B8E76068022802
:1037400006D13748006800F0007040B90120AEE7AC
:103750003348006800F0020008B90120A7E73048AC
:10376000406820F00300616808432D494860FEF777
:1037700031FD064609E0FEF72DFD801B41F2883140
:10378000884202D9032092E707E02548406800F00C
:103790000C006168B0EB810FEDD12048006800F0AB
:1037A0000700A8420ED91D48006820F007002843F2
:1037B0001A4908600846006800F00700A84201D0D6
:1037C000012074E7207800F00400042807D1144891
:1037D000406820F4E060E1680843114948602078BF
:1037E00000F00800082808D10D48406820F4605017
:1037F000216940EAC1000A49486000F03FF80849E1
:103800004968C1F30311074A515CC8400649086082
:1038100006480068FFF738FD002048E70020024016
:1038200000100240B6370108000000200800002008
:1038300001480068704700000000002000B5FFF755
:10384000F7FF04494968C1F30221034A515CC840AB
:1038500000BD000000100240C637010800B5FFF7A8
:10386000E7FF04494968C1F3C221034A515CC840DB
:1038700000BD000000100240C6370108F0B585B059
:103880000FF26C0C9CE8E01001A8A0E8E0101CA569
:103890002D68009500210022002300240020194DEE
:1038A000696801F00C05F5B1042D02D0082D19D17D
:1038B00001E0154819E001ADC1F38346AC5D01F4A8
:1038C000803555B10F4D6D68C5F340451DF8052095
:1038D0000D4D6543B5FBF2F302E00C4D04FB05F31F
:1038E000184602E000BF084800BF00BF05B0F0BDA9
:1038F00002030405060708090A0B0C0D0E0F101031
:10390000010200000010024000127A0000093D0090
:10391000F8B504460CB90120F8BD207800F001008C
:10392000002878D0F848406800F00C0004280CD03B
:10393000F548406800F00C00082811D1F2484068B2
:1039400000F48030B0F5803F0AD1EF48006800F401
:10395000003000285FD0606800285CD10120DBE7E0
:1039600000BF6068B0F5803F06D1E748006840F4CA
:103970008030E549086028E0606858B9E24800688E
:1039800020F48030E04908600846006820F4802078
:1039900008601AE06068B0F5A02F0BD1DA48006823
:1039A00040F48020D84908600846006840F4803020
:1039B00008600AE0D448006820F48030D2490860EA
:1039C0000846006820F48020086000BF606888B165
:1039D000FEF700FC054606E0FEF7FCFB401B6428F2
:1039E00001D9032098E7C848006800F40030002897
:1039F000F2D010E0FEF7EEFB054606E0FEF7EAFB2C
:103A0000401B642801D9032086E7BF48006800F402
:103A100000300028F2D1207800F00200022857D1AF
:103A2000B948406800F00C0050B1B748406800F059
:103A30000C00082818D1B448406800F4803098B9C8
:103A4000B148006800F0020020B12069012801D0CF
:103A5000012061E7AC48006820F0F800616940EAA5
:103A6000C100A949086033E02069E8B10120A749F5
:103A70000860FEF7AFFB054606E0FEF7ABFB401B18
:103A8000022801D9032047E79F48006800F00200A0
:103A90000028F2D09C48006820F0F800616940EAF4
:103AA000C1009949086013E0002098490860FEF7BA
:103AB00091FB054606E0FEF78DFB401B022801D96D
:103AC000032029E79048006800F002000028F2D1A6
:103AD000207800F0080008282DD1A069B8B1012095
:103AE0008B490860FEF776FB054606E0FEF772FBA1
:103AF000401B022801D903200EE78348406A00F0EA
:103B000002000028F2D0012002F03EFA13E000206B
:103B10007F490860FEF75EFB054606E0FEF75AFBAC
:103B2000401B022801D90320F6E67748406A00F0DE
:103B300002000028F2D1207800F00400042873D19C
:103B400000277148C06900F0805070B900BF6E480E
:103B5000C06940F080506C49C8610846C06900F0F7
:103B60008050009000BF00BF01276A48006800F441
:103B70008070B0B96748006840F48070654908609B
:103B8000FEF728FB054606E0FEF724FB401B6428F1
:103B900001D90320C0E65F48006800F48070002867
:103BA000F2D000BFE068012806D15748006A40F013
:103BB00001005549086227E0E06858B95248006A98
:103BC00020F00100504908620846006A20F0040015
:103BD000086219E0E06805280BD14B48006A40F004
:103BE0000400494908620846006A40F00100086282
:103BF0000AE04548006A20F001004349086208468F
:103C0000006A20F00400086200BFE068A0B1FEF77F
:103C1000E1FA054609E0FEF7DDFA401B41F2883182
:103C2000884202D9032077E622E03748006A00F094
:103C300002000028EFD012E0FEF7CCFA054608E0BB
:103C4000FEF7C8FA401B41F28831884201D90320AF
:103C500062E62D48006A00F002000028F0D1012F32
:103C600005D12948C06920F080502749C86100BFAC
:103C7000E069C8B32448406800F00C00082860D010
:103C8000E069022848D1002020490866FEF7A2FA20
:103C9000054606E0FEF79EFA401B022801D90320E4
:103CA0003AE61948006800F000700028F2D1206A56
:103CB000B0F5803F07D11448406820F40030A16877
:103CC000084311494860D4E9080108430E4949688E
:103CD00021F4741108430C49486001200B4908661F
:103CE000FEF778FA054607E03DE0FEF773FA401B61
:103CF000022801D903200FE60348006800F0007095
:103D00000028F2D02FE000000010024000004242E4
:103D10008004424200700040002014490866FEF70B
:103D200059FA054606E0FEF755FA401B022801D96C
:103D30000320F1E50E48006800F000700028F2D181
:103D400011E0E069012800D1E6E50948466806F47B
:103D50008031206A814204D106F47011606A814288
:103D600001D00120D8E50020D6E500000000424245
:103D70000010024070B505460948007801280DD1B1
:103D8000002409E0074810F8340020B1054901EB90
:103D9000C40148688047641C142CF3DB70BD00002C
:103DA0001A0000206C03002010B50446206800684B
:103DB000C0F3400068B120684068C0F3400040B1E3
:103DC0002046FFF7D7FF2068406820F002002168F6
:103DD00048604FF40030024908600120607410BD53
:103DE00014040140F8B505460C4616460020009024
:103DF00005B10CB90120F8BD00226946284600F043
:103E00001AF808B10120F6E7287B2070E87BE07003
:103E1000687B6070A87BA0705EB1E07802F0DBF890
:103E2000E070607802F0D7F86070A07802F0D3F804
:103E3000A0700020DFE72DE9F04780460C46914650
:103E400000250026AA460027B8F1000F00D014B9BB
:103E50000120BDE8F087D8F800004068C0F380007A
:103E600008B10120F5E7404602F07CF905464FF421
:103E70006160B5FBF0F7B5FBF0F100FB11503C21A0
:103E8000B0FBF1F060704FF46160B5FBF0F100FB46
:103E900011503C21B0FBF1F201FB1200A070182F71
:103EA00039D31820B7FBF0FAB7FBF0F100FB117023
:103EB0002070404602F04AF90646701C18B1AE4226
:103EC00001D9761B01E04FF0FF360AEB4A00C00033
:103ED000C0EB4011C1EB0020A5EB00152946404680
:103EE00002F0B3F908B10120B3E7701C38B12E44D9
:103EF0003146404602F092F940B10120A9E731462F
:103F0000404602F08BF908B10120A2E75146404635
:103F100002F06EF800E02770B9F1000F0BD02078A6
:103F200002F059F82070607802F055F86070A078BF
:103F300002F051F8A07000208BE7000070B5044635
:103F400000250CB9012070BD607C20B900202074D0
:103F5000204600F05BF802206074204600F000FA72
:103F600018B1042060740120EDE7204602F09BF8B0
:103F700018B1042060740120E5E72068406820F053
:103F8000070021684860A06828B11F48006820F039
:103F900001001D4908601C48001F006820F4607083
:103FA000A16808431849091F08606068401C08B1EF
:103FB000656809E00120FFF743FA05461DB90420B2
:103FC00060740120BFE76D1E2068806820F00F003C
:103FD00040EA1540216888602068C06865F30F00DA
:103FE0002168C860204602F07BF818B10420607494
:103FF0000120A8E70021E17301216173A173012071
:10400000607400209FE70000306C004010B592B053
:1040100004461849206888422AD100BF1648C06962
:1040200040F080501449C8610846C06900F08050D3
:10403000019000BF00BFFFF7D3F9042008900020D3
:104040000F9001200B900002039008A8FFF760FC7E
:104050000120029002A8FFF78DFA012007490860AD
:1040600000220F212920FFF769F92920FFF756F9CF
:1040700012B010BD00280040001002403C04424233
:104080002DE9F84304460D4617460026002000900F
:1040900004B115B90120BDE8F88300BF207C0128D8
:1040A00001D10220F7E70120207400BF02206074D4
:1040B000002269462046FFF7BEFE08B10120EAE76C
:1040C0009DF800004FF4616148439DF80110C1EB79
:1040D000011100EB81009DF8021000EB01085FB9AF
:1040E00028784FF4616148436978C1EB011100EB16
:1040F0008100A978461812E0287801F061FF4FF49A
:10410000616100FB01F9687801F05AFFC0EB001013
:1041100009EB8009A87801F053FF09EB000646453A
:1041200001D2184806443146204602F077F838B1EB
:104130000420607400BF0020207400BF0120AAE7A3
:104140002068406820F0020021684860206800680C
:1041500040F00200216808600B48006840F400301D
:104160000949086008480830006840F400300649F2
:10417000083108600120607400BF0020207400BF77
:1041800000BF88E780510100000401402DE9F0479D
:1041900004460D46904600260027B14604B115B9E5
:1041A0000120BDE8F08700BF207C012801D102205A
:1041B000F7E70120207400BF02206074B8F1000FFF
:1041C00006D1E978E17369786173A978A1730BE08E
:1041D000E87801F0F5FEE073687801F0F1FE6073B5
:1041E000A87801F0EDFEA073A27B617BE07B01F07B
:1041F000D3FF2073207B2870204601F0B3FF0646D2
:104200004FF46160B6FBF0F9B9F1180F2FD91820FF
:10421000B9FBF0F000EB4000C000C0EB4011C1EB77
:104220000020A6EB00163146204602F00EF838B109
:104230000420607400BF0020207400BF0120B0E79C
:10424000204601F083FF0746781C80B1B7420ED2AA
:104250000B4807443946204601F0E0FF38B10420FE
:10426000607400BF0020207400BF012099E7012086
:10427000607400BF0020207400BF00BF91E7000001
:10428000805101002DE9F04704460D469046002676
:10429000002704B115B90120BDE8F08700BF207CDC
:1042A000012801D10220F7E70120207400BF02207D
:1042B0006074B8F1000F0BD128784FF46161484366
:1042C0006978C1EB011100EB8100A978461812E072
:1042D000287801F075FE4FF4616100FB01F9687800
:1042E00001F06EFEC0EB001009EB8009A87801F028
:1042F00067FE09EB00063146204601F0A6FF38B103
:104300000420607400BF0020207400BF0120C3E7B8
:104310002068406820F0050021684860204601F0D0
:1043200015FF0746781C80B1B7420ED20B480744F0
:104330003946204601F072FF38B10420607400BF96
:104340000020207400BF0120A6E70120607400BF98
:104350000020207400BF00BF9EE7000080510100D4
:1043600070B5044600250CB9012070BD2068406876
:1043700020F0080021684860FDF72CFF054607E0A3
:10438000FDF728FF401BB0F57A7F01D90320ECE749
:104390002068406800F008000028F1D00020E4E721
:1043A0004FF0E020006940F002004FF0E02108618A
:1043B000704710B504460CB9012010BD022084F8E6
:1043C00051002068006820F0400021680860204605
:1043D00000F010F90020606584F8510000BF84F8F7
:1043E000500000BF00BFE8E770470000F8B5044682
:1043F0002068466820688568C5F3801048B905F0D4
:10440000010030B1C6F3801018B12046216C8847F6
:10441000F8BDC5F3400030B1C6F3C01018B1204656
:10442000616C8847F4E7C5F3401018B9C5F38010F4
:10443000002871D0C6F3401000286DD0C5F380105D
:10444000F0B194F8510003280ED0606D40F00400E4
:10445000606500BF002000902068C0680090206860
:104460008068009000BF0BE000BF00200090206833
:10447000C068009020688068009000BF00BFC7E758
:10448000C5F3401088B1606D40F00100606500BF69
:10449000002000902068806800902068006820F06C
:1044A00040002168086000BF00BF606D70B32068E5
:1044B000406820F0E00021684860012084F8510045
:1044C00006F0020010B906F0010000B32068406851
:1044D00020F0030021684860E06C50B10F48E16CA7
:1044E0004863E06CFDF708FB18B1606D40F04000D8
:1044F0006065A06C50B10948A16C4863A06CFDF7E1
:10450000FBFA18B1606D40F04000606502E02046A3
:10451000FFF76AFF7CE7FFE700BF79E74565000822
:1045200010B504460CB9012010BD606A38B9606846
:10453000B0F5827F00D105E00021E16102E00021B9
:1045400021616161A06AB0F5005F00D100BF94F8FD
:10455000510028B9002084F85000204600F0CAF825
:10456000022084F851002068006820F04000216893
:104570000860A08800F48270218901F40441084396
:10458000A18901F400610843217C01F00201084384
:10459000217D01F001010843218B01F400710843E2
:1045A000217F01F0380108432021095D01F08001DD
:1045B0000843218D01F4005108432168086004215B
:1045C000A06901EA104021684860A06AB0F5005F68
:1045D00003D1A08D80B2216808612068C06920F4F1
:1045E00000602168C86100206065012084F85100E6
:1045F000002099E710B504463449206888421DD14F
:104600003348806920F48050314988612021314845
:10461000FDF75AFB20212F48FDF756FB80212D483E
:10462000FDF752FB4FF400612B48FDF74DFB2320B3
:10463000FEF752FE00202949087045E0284920680D
:10464000884220D12248C06920F480402049C861B6
:104650004FF400512348FDF737FB4FF480412148C8
:10466000FDF732FB4FF400411E48FDF72DFB4FF4E0
:1046700080511C48FDF728FB2420FEF72DFE00206A
:104680001949087020E01949206888421CD1104857
:10469000C06920F400400E49C86108211148FDF7A7
:1046A00013FB10210F48FDF70FFB20210D48FDF7EC
:1046B0000BFB4FF400410748FDF706FB3320FEF7E4
:1046C0000BFE00200A49087010BD000000300140B8
:1046D0000010024000080140002001401B000020A3
:1046E00000380040000C01401C000020003C00404D
:1046F0001D00002010B586B00446B14920688842EC
:1047000070D100BFAF48806940F48050AD498861E6
:104710000846806900F48050019000BF00BF00BFD0
:104720000846806940F0040088610846806900F00E
:104730000400019000BF00BF00BF0846806940F040
:10474000040088610846806900F00400019000BF01
:1047500000BF00BF0846806940F004008861084639
:10476000806900F00400019000BF00BF00BF084650
:10477000806940F4807088610846806900F4807028
:10478000019000BF00BF2020029002200390012072
:1047900004900320059002A98B48FDF76DFB2020B3
:1047A00002900120049002A98748FDF765FB802054
:1047B00002900120049002A98348FDF75DFB4FF4AD
:1047C000006002900120049002A98048FDF754FB8C
:1047D000002201212320FEF7B1FD2320FEF79EFDDC
:1047E000ECE0FFE77A492068884273D100BF754842
:1047F000C06940F480407349C8610846C06900F44C
:104800008040019000BF00BF00BF0846806940F0B3
:10481000080088610846806900F00800019000BF28
:1048200000BF00BF0846806940F008008861084664
:10483000806900F00800019000BF00BF00BF08467B
:10484000806940F0080088610846806900F008002F
:10485000019000BF00BF00BF0846806940F008001B
:1048600088610846806900F00800019000BF00BF21
:104870004FF4005002900220039001200490032086
:10488000059002A95348FDF7F7FA4FF480400290D3
:104890000120049002A94F48FDF7EEFA4FF40040C2
:1048A00002900120049002A94A48FDF7E5FA4FF46E
:1048B000805002900120049002A94648FDF7DCFADE
:1048C000002201212420FEF739FD2420FEF726FDD9
:1048D00074E0FFE74049206888426FD100BF394843
:1048E000C06940F400403749C8610846C06900F417
:1048F0000040019000BF00BF00BF0846806940F043
:10490000080088610846806900F00800019000BF37
:1049100000BF00BF0846806940F008008861084673
:10492000806900F00800019000BF00BF00BF08468A
:10493000806940F0080088610846806900F008003E
:10494000019000BF00BF00BF0846806940F004002E
:1049500088610846806900F00400019000BF00BF34
:10496000082002900220039000200490032005906C
:1049700002A91848FDF780FA102002900020049048
:1049800002A91448FDF778FA202002900020049034
:1049900002A91048FDF770FA4FF400400290012080
:1049A0000390049002A90848FDF766FA002201214D
:1049B0003320FEF7C3FC3320FEF7B0FC06B010BD79
:1049C000003001400010024000080140002001407A
:1049D00000380040000C0140003C004070470000DF
:1049E000F0B50446002700BF94F85000012801D11B
:1049F0000220F0BD012084F8500000BF94F851500F
:104A00006668012D08D0B6F5827F03D1A06808B989
:104A1000042D01D002274BE009B102B10BB90127E7
:104A200046E094F85100042802D0052084F8510093
:104A3000002060652163A386E386A263A387E387E2
:104A4000E06820B11E4820641E48606403E01E48F0
:104A500020641E486064A06AB0F5005F11D100BFF9
:104A60002068006820F40050D4F800C0CCF80000A2
:104A70002068006840F40050D4F800C0CCF8000072
:104A800000BF2068406840F0E000D4F800C0CCF8D7
:104A900004002068006800F04000402807D020682B
:104AA000006840F04000D4F800C0CCF8000000BF1F
:104AB00000BF002084F8500000BF384699E700008E
:104AC000A96200088B63000815630008E36300080F
:104AD000704770B504462546681EB0F1807F01D34B
:104AE00001200FE0681E4FF0E02148610F214FF0D8
:104AF000FF3009F03DFE00204FF0E02188610720E3
:104B00000861002070BD4FF0E020006920F0020035
:104B10004FF0E0210861704770477047704710B54B
:104B2000044620680069C0F34000D8B12068C0681E
:104B3000C0F34000B0B16FF00200216808610120AD
:104B400020772068806900F0030018B12046FFF745
:104B5000E5FF05E0204600F0ADF8204600F0ABF898
:104B60000020207720680069C0F38000D8B1206859
:104B7000C068C0F38000B0B16FF004002168086124
:104B8000022020772068806900F4407018B1204628
:104B9000FFF7C4FF05E0204600F08CF8204600F047
:104BA0008AF80020207720680069C0F3C000D8B1DF
:104BB0002068C068C0F3C000B0B16FF00800216881
:104BC0000861042020772068C06900F0030018B154
:104BD0002046FFF7A3FF05E0204600F06BF82046D3
:104BE00000F069F80020207720680069C0F3001009
:104BF000D8B12068C068C0F30010B0B16FF01000E9
:104C000021680861082020772068C06900F440709E
:104C100018B12046FFF782FF05E0204600F04AF871
:104C2000204600F048F8002020772068006900F056
:104C3000010058B12068C06800F0010030B16FF089
:104C4000010021680861204600F036F820680069FC
:104C5000C0F3C01058B12068C068C0F3C01030B1B4
:104C60006FF08000216808612046FFF755FF20683B
:104C70000069C0F3801058B12068C068C0F380108C
:104C800030B16FF0400021680861204600F068F8FC
:104C900020680069C0F3401058B12068C068C0F3B4
:104CA000401030B16FF02000216808612046FFF706
:104CB00034FF10BD7047704770B505462548006841
:104CC000401C2449086024492868884241D10024B6
:104CD0003DE02248005D012838D12048283850F8AE
:104CE00024001C490968884219D31C48283850F808
:104CF000240018490968401AC0F1FF3117480C30E8
:104D000050F824000068814220D314490C3151F836
:104D100024104868804700211048015516E00F48CC
:104D2000283850F824000B490968091A0B480C3040
:104D300050F824000068814208D308490C3151F82A
:104D4000241048688047002104480155641C0A2C3F
:104D5000BFDB70BD2000002000040040980500204B
:104D60007047704710B504460CB9012010BD2420CF
:104D700084F83D002068C06820F400502168C860B5
:104D8000204600F06FF90020206484F83D0084F88C
:104D90003E00206300BF84F83C0000BF00BFE5E791
:104DA000704700002DE9F84F044620680568206828
:104DB000C668206847694FF00009CA4605F00F0928
:104DC000B9F1000F0AD105F0200038B106F020003B
:104DD00020B1204601F09FFCBDE8F88FB9F1000F2B
:104DE00071D007F0010018B906F4907000286AD05D
:104DF00005F0010030B106F4807018B1206C40F06D
:104E00000100206405F0040030B107F0010018B182
:104E1000206C40F00200206405F0020030B107F081
:104E2000010018B1206C40F00400206405F0080077
:104E300048B106F0200010B907F0010018B1206C4D
:104E400040F008002064206C68B305F0200028B111
:104E500006F0200010B1204601F05DFC206840699A
:104E6000C0F3801A206C00F0080010B9BAF1000FEE
:104E700022D0204601F024FC2068406900F0400068
:104E8000B0B12068406920F0400021684861A06B03
:104E900050B15648A16B4863A06BFCF72DFE10B1D2
:104EA000A06B416B88470CE02046FFF779FF08E0D4
:104EB0002046FFF775FF04E02046FFF771FF002052
:104EC000206489E7FFE7206B012878D105F0100006
:104ED000002874D006F01000002870D000BF002019
:104EE000009020680068009020684068009000BF33
:104EF00000BF2068406900F04000C0B3A06B0068AC
:104F000040681FFA80F8B8F1000F2FD0A08D4045FF
:104F10002CDDA4F82E80A06B806920281FD020688B
:104F2000C06820F480702168C8602068406920F063
:104F30000100216848612068406920F04000216834
:104F40004861202084F83E00002020632068C0686B
:104F500020F010002168C860A06BFCF7A1FDA08DB7
:104F6000E28D801A81B22046FFF7FBFE34E7FFE7AF
:104F7000A08DE18D401A1FFA80F8E08DE8B1B8F1FC
:104F8000000F1AD02068C06820F490702168C860B3
:104F90002068406920F0010021684861202084F8E1
:104FA0003E00002020632068C06820F010002168C7
:104FB000C86041462046FFF7D4FE0DE7FFE705F045
:104FC000800030B106F0800018B1204601F0B7FC37
:104FD00002E705F0400030B106F0400018B120466D
:104FE00001F089FBF8E600BFF6E60000AD660008B8
:104FF00010B504460CB9012010BDA06900B100E055
:1050000000BF94F83D0028B9002084F83C002046F9
:1050100000F0D2F8242084F83D002068C06820F415
:1050200000502168C860204601F0E8FB2068006954
:1050300020F49040216808612068406920F02A002F
:10504000216848612068C06840F400502168C86049
:1050500000202064202084F83D0084F83E000020D9
:10506000CAE7000010B5044649492068884217D1B4
:105070004848C06840F480404649C8600846C06857
:1050800020F48040C86009154348FCF71DFE4FF42A
:1050900080614148FCF718FE2520FEF71DF976E0F7
:1050A0003E492068884216D13A48006940F40030F1
:1050B000384908610846006920F40030086104217D
:1050C0003548FCF701FE08213348FCF7FDFD26209A
:1050D000FEF702F95BE032492068884217D12D487B
:1050E000006940F480202B4908610846006920F4DB
:1050F0008020086189152B48FCF7E6FD4FF400710C
:105100002848FCF7E1FD2720FEF7E6F83FE02649B6
:10511000206888421CD11F48006940F400201D49C6
:1051200008610846006920F40020086109151F483D
:10513000FCF7CAFD4FF400611C48FCF7C5FD4FF4B5
:1051400000711A48FCF7C0FD3420FEF7C5F81EE0D8
:105150001749206888421AD10E48006940F480102F
:105160000C4908610846006920F480100861891420
:105170000E48FCF7A9FD04210A48FCF7A5FD4FF4F1
:1051800080710C48FCF7A0FD3520FEF7A5F810BD96
:105190000038014000100240000801400044004077
:1051A0000048004000140140004C00400010014045
:1051B000005000400020014010B586B00446E74989
:1051C0002068884249D100BFE548806940F48040AA
:1051D000E34988610846806900F48040019000BF7F
:1051E00000BF00BF0846806940F00400886108469F
:1051F000806900F00400019000BF00BF00BF0846B6
:10520000806940F0040088610846806900F004006D
:10521000019000BF00BF48150290022003900120BA
:1052200004900320059002A9CE48FCF725FE4FF418
:1052300080600290002003900120049003200590DC
:1052400002A9C848FCF718FE002201212520FEF71C
:1052500075F82520FEF762F87EE1C3492068884290
:1052600048D100BFBE48C06940F40030BC49C861A5
:105270000846C06900F40030019000BF00BF00BFC5
:105280000846806940F0040088610846806900F0A3
:105290000400019000BF00BF00BF0846806940F0D5
:1052A000040088610846806900F00400019000BF96
:1052B00000BF0420029002200390012004900320EC
:1052C000059002A9A748FCF7D7FD0820029000200E
:1052D0000390012004900320059002A9A148FCF747
:1052E000CBFD002205212620FEF728F82620FEF718
:1052F00015F831E19D492068884255D100BF984892
:10530000C06940F480209649C8610846C06900F42D
:105310008020019000BF00BF00BF9549486820F081
:10532000300040F0E06040F03000486000BF00BF57
:105330008B48806940F0200089498861084680696F
:1053400000F02000019000BF00BF00BF0846806948
:1053500040F0200088610846806900F0200001903C
:1053600000BF00BF88150290022003900120049026
:105370000320059002A97F48FCF77EFD4FF40070E2
:10538000029000200390012004900320059002A9C0
:105390007848FCF771FD002205212720FDF7CEFF9C
:1053A0002720FDF7BBFFD7E073492068884268D10A
:1053B00000BF6B48C06940F400206949C8610846D5
:1053C000C06900F40020019000BF00BF00BF084684
:1053D000806940F0100088610846806900F0100084
:1053E000019000BF00BF00BF0846806940F0100078
:1053F00088610846806900F01000019000BF00BF7E
:1054000008150290022003900120049003200590CB
:1054100002A95A48FCF730FD4FF4006002900020CA
:105420000390012004900320059002A95348FCF743
:1054300023FD00BF4A48806940F010004849886158
:105440000846806900F01000019000BF00BF4815B9
:1054500002900120039004900320059002A9474880
:10546000FCF70AFD00224FF400714448FCF7ACFE43
:10547000002201213420FDF761FF3420FDF74EFFAB
:105480006AE03F492068884266D100BF3448C0695D
:1054900040F480103249C8610846C06900F48010A9
:1054A000019000BF00BF00BF0846806940F01000B7
:1054B00088610846806900F01000019000BF00BFBD
:1054C00000BF0846806940F0200088610846806976
:1054D00000F02000019000BF00BF8814029002205D
:1054E0000390012004900320059002A92348FCF7B3
:1054F000C3FC0420029000200390012004900320AC
:10550000059002A91B48FCF7B7FC00BF144880694E
:1055100040F48070124988610846806900F4807008
:10552000019000BF00BF88150290012003900490F5
:105530000320059002A91348FCF79EFC00224FF4BB
:1055400080711048FCF740FE002201213520FDF754
:10555000F5FE3520FDF7E2FE06B010BD0038014033
:105560000010024000080140004400400048004094
:105570000000014000140140004C004000100140B8
:10558000005000400020014070B504460D4616460C
:1055900094F83E00202816D105B10EB9012070BD47
:1055A00000BF94F83C00012801D10220F7E7012058
:1055B00084F83C0000BF0020206332462946204684
:1055C00001F09AF9EBE70220E9E7000010B5044684
:1055D0002C49206888420DD12B48006820B12B4807
:1055E0000078294909688847012228492848FFF797
:1055F000CBFF46E02749206888420DD12648006845
:1056000020B12648007824490968884701222349A7
:105610002348FFF7B9FF34E02249206888420DD1C2
:105620002148006820B1214800781F49096888474F
:1056300001221E491E48FFF7A7FF22E01D492068EE
:1056400088420DD11C48006820B11C4800781A49D6
:1056500009688847012219491948FFF795FF10E0AA
:105660001849206888420CD11748006820B11748B3
:105670000078154909688847012214491448FFF742
:1056800083FF10BD003801403800002028000020B2
:10569000CC050020004400404000002029000020EC
:1056A0001006002000480040480000202A0000208A
:1056B00054060020004C0040500000202B00002029
:1056C0009806002000500040580000202C000020C8
:1056D000DC06002010B5034693F83D00202823D1B6
:1056E00001B10AB9012010BD00BF93F83C000128A8
:1056F00001D10220F7E7012083F83C0000BF1962C6
:105700009A84DA8400201864212083F83D0000BFC9
:10571000002083F83C0000BF1868C06840F080009B
:105720001C68E0600020DEE70220DCE710B50446DC
:105730001B492068884206D11A48006818B31948E6
:10574000006880472AE018492068884206D1174837
:105750000068C0B11548006880471FE01449206800
:10576000884206D11348006868B112480068804733
:1057700014E011492068884206D11048006810B131
:105780000E480068804709E00D492068884205D12D
:105790000C48006810B10B480068804710BD00003D
:1057A0000038014034000020004400403C0000204C
:1057B0000048004044000020004C00404C00002005
:1057C000005000405400002010B5044605480088F1
:1057D000401E044908800846008810B1204600F0A9
:1057E00017F810BD5E00002010B504462068406820
:1057F000C0F3402058B12068806800F0010030B14B
:105800006FF00100216888602046FFF7DDFF10BDC2
:1058100001460A68C86810600020704704E0012053
:1058200008F0F3FF08F0B8FFF9E70146086840699F
:10583000C0F38020B0B16FF480600A68506100202E
:105840000863202081F83D00002081F83E00086CAC
:1058500040F00400086400BF002081F83C0000BF55
:10586000012070470020FCE72DE9F84304460D466F
:1058700090461E46E76A2068006840F48060216810
:105880000860082F04D0012F02D017F5803F06D101
:105890002068006840F480702168086008E0206B90
:1058A000112805D12068006840F4807021680860E4
:1058B000434600224FF001112046009600F01EFAE8
:1058C00060B12068006800F48070B0F5807F02D17C
:1058D0004FF4007020640320BDE8F8832069B0F520
:1058E000804F05D1E8B240F001002168086149E02D
:1058F00005F44070F02141EAE01021680861334668
:1059000042462649204600F03CFA08B10120E3E770
:10591000E8B221680861334642462049891F204683
:1059200000F02FFA08B10120D6E700BF0020009058
:1059300020684069009020688069009000BF00BF27
:105940002068006840F480702168086043460022A7
:105950004FF001112046009600F0D0F958B12068B0
:10596000006800F48070B0F5807F02D14FF40070C1
:1059700020640320B0E705F44070F12141EAE01013
:1059800021680861334642460449891F204600F0D9
:10599000F8F908B101209FE700209DE70800010009
:1059A0002DE9F84304460D4617469846E66A082E48
:1059B00004D0012E02D016F5803F06D12068006881
:1059C00040F480702168086008E0206B122805D13F
:1059D0002068006840F48070216808603B4600221F
:1059E0004FF001112046CDF8008000F087F960B13A
:1059F0002068006800F48070B0F5807F02D14FF419
:105A0000007020640320BDE8F8832069B0F5804F62
:105A100004D105F0FE002168086112E005F4407031
:105A2000F02141EAE0102168086143463A460B49FB
:105A3000204600F0A6F908B10120E4E7E8B22168A9
:105A4000086143463A460549891F204600F099F906
:105A500008B10120D7E70020D5E7000008000100C9
:105A60002DE9F84304460F4615469946DDE90886B8
:105A70002068006840F48060216808602068006841
:105A800040F4807021680860434600224FF0011105
:105A90002046009600F032F960B12068006800F4FA
:105AA0008070B0F5807F02D14FF400702064032035
:105AB000BDE8F88307F0FE002168086133464246DE
:105AC0003E49204600F05DF908B10120F0E700BF33
:105AD0000020009020684069009020688069009054
:105AE00000BF00BF32464146204600F018FA50B1D0
:105AF000206C042805D12068006840F400702168FB
:105B000008600120D4E7B9F1010F03D1E8B22168A0
:105B1000086117E0C5F30720216808613246414655
:105B2000204600F0FCF950B1206C042805D1206813
:105B3000006840F40070216808600120B8E7E8B20E
:105B40002168086132464146204600F0E8F950B12C
:105B5000206C042805D12068006840F4007021689A
:105B600008600120A4E72068006840F48070216884
:105B70000860434600224FF001112046009600F0D5
:105B8000BDF858B12068006800F48070B0F5807FDF
:105B900002D14FF400702064032089E7F8B240F08E
:105BA000010021680861334642460449204600F05E
:105BB000E8F808B101207BE7002079E70200010046
:105BC0002DE9F8430446884615469946DDE90867FD
:105BD0002068006840F48070216808603346002225
:105BE0004FF001112046009700F088F860B120685E
:105BF000006800F48070B0F5807F02D14FF400702F
:105C000020640320BDE8F88308F0FE0021680861E5
:105C10003B4632462149204600F0B3F808B1012046
:105C2000F0E700BF002000902068406900902068E5
:105C30008069009000BF00BF3A463146204600F020
:105C40006EF950B1206C042805D12068006840F43A
:105C50000070216808600120D4E7B9F1010F03D179
:105C6000E8B22168086117E0C5F3072021680861E0
:105C70003A463146204600F052F950B1206C0428D3
:105C800005D12068006840F4007021680860012098
:105C9000B8E7E8B2216808610020B3E7020001001C
:105CA00070B504460D46164620E02046FFF7BDFDC0
:105CB00008B1012070BD681CC0B1FCF78BFA801BD5
:105CC000A84200D895B900202063202084F83D0028
:105CD000002084F83E00206C40F02000206400BFCB
:105CE000002084F83C0000BF0120E3E72068406901
:105CF000C0F380000028D8D00020DBE72DE9F04178
:105D000004460D4617461E46DDF818801CE0701C40
:105D1000D0B1FCF75FFAA0EB0800B04200D89EB902
:105D200000202063202084F83D00002084F83E00FD
:105D3000206C40F02000206400BF002084F83C006C
:105D400000BF0120BDE8F081C5F3074001280AD15A
:105D500020684069A9B20840A9B2884201D1012057
:105D60000BE0002009E020688069A9B20840A9B2D0
:105D7000884201D1012000E00020B842C7D00020B5
:105D8000E0E72DE9F04104460D4616461F463DE08A
:105D900020684069C0F38020E8B12068006840F4C2
:105DA0000070216808606FF48060216848610020FD
:105DB0002063202084F83D00002084F83E00206C01
:105DC00040F00400206400BF002084F83C0000BFC5
:105DD0000120BDE8F081701CC0B1FCF7FBF9C01BCD
:105DE000B04200D896B900202063202084F83D00FE
:105DF000002084F83E00206C40F02000206400BFAA
:105E0000002084F83C0000BF0120E2E7C5F3074012
:105E100001280AD120684069A9B20840A9B2884285
:105E200001D101200BE0002009E020688069A9B2BF
:105E30000840A9B2884201D1012000E000200028DA
:105E4000A6D00020C5E770B504460D46164632E0E0
:105E500020684069C0F30010A0B16FF01000216805
:105E6000486100202063202084F83D00002084F851
:105E70003E00206C206400BF002084F83C0000BF7E
:105E8000012070BDFCF7A6F9801BA84200D895B987
:105E900000202063202084F83D00002084F83E008C
:105EA000206C40F02000206400BF002084F83C00FB
:105EB00000BF0120E5E720684069C0F3801000289A
:105EC000C6D00020DDE770B504460D4616461EE03C
:105ED0002046FFF7AAFC08B1012070BDFCF77AF953
:105EE000801BA84200D895B900202063202084F8A8
:105EF0003D00002084F83E00206C40F0200020642B
:105F000000BF002084F83C0000BF0120E5E72068C6
:105F10004069C0F300100028DAD00020DDE770B53A
:105F200004460D46164620E02046FFF77EFC08B1E9
:105F3000012070BD681CC0B1FCF74CF9801BA84261
:105F400000D895B900202063202084F83D0000206F
:105F500084F83E00206C40F02000206400BF002048
:105F600084F83C0000BF0120E3E720684069C0F3EB
:105F7000C0100028D8D00020DBE700BFFEE7704744
:105F800020BF00BF7047704708B508490968C908B5
:105F90004FF47A72B1FBF2F14143009100BF00BFB0
:105FA00000994A1E00920029F9D108BD0000002086
:105FB00010B50248FDF7F8FE10BD00000C040020EB
:105FC000014600BF080900EB8000420001F00F000D
:105FD0001044C0B270470146002203E0521CA1F1F8
:105FE0000A00C1B20A29F9D2100741EA10607047CD
:105FF0002DE9F04706468846002700240025A146E3
:10600000F77B747BB57B00BF40E0012C0BD0032CE9
:1060100009D0052C07D0072C05D0082C03D00A2C5A
:1060200001D00C2C0CD11F2D01D26D1C2CE00C2C9E
:1060300002D0641C012527E0012401257F1C23E0F8
:10604000042C05D0062C03D0092C01D00B2C06D132
:106050001E2D01D26D1C17E0641C012514E0022CDA
:1060600012D11C2D01D26D1C0EE01C2D08D1B8B22E
:1060700000F053F808B16D1C06E0641C012503E034
:106080001D2D01D1641C012509F10109C145BCD3B5
:10609000F7737473B573EAB2E1B2384600F07CF876
:1060A0003073BDE8F08770B504460025FCF792F820
:1060B000054607E0FCF78EF8401BB0F57A7F01D962
:1060C000032070BD2068406800F020000028F1D057
:1060D0002068406840F01000216848600020F0E728
:1060E00070B5044600252068406820F01000216843
:1060F0004860FCF76FF8054607E0FCF76BF8401BBB
:10610000B0F57A7F01D9032070BD2068406800F0A7
:1061100020000028F1D00020F6E7014601F003003E
:1061200008B1002070476420B1FBF0F200FB1210B0
:1061300008B10120F6E74FF4C870B1FBF0F200FBA4
:10614000121008B90120EDE70020EBE7014600221C
:1061500000230868006A82B20868406A83B243EA92
:106160000240704730B50146002200230024002081
:106170000D68AD69AAB20D68ED69ACB20D68AD6984
:10618000ABB29A4205D00D68ED6963F31F4528460E
:1061900001E044EA024030BDF0B504460B46002160
:1061A000002504F5FA61032B1BD2C3EBC30000EBFF
:1061B00003100926B0FBF6F01044001D4618481ED7
:1061C00006EB90066427B0FBF7F0361A481EBF00B6
:1061D000B0FBF7F030440726B0FBF6F706FB1705D7
:1061E0001AE0C3EBC30000EB03100926B0FBF6F086
:1061F0001044001D084400EB91006426B1FBF6F644
:10620000801B4FF4C876B1FBF6F63044801E07269B
:10621000B0FBF6F706FB1705E8B2F0BD70B5044613
:106220000D4600262046FFF73EFF08B101260AE092
:10623000280C21680862A8B2216848622046FFF74E
:106240004FFF00B10126304670BD70B504460D46C3
:1062500000262046FFF727FF08B101260AE0280C98
:1062600021688861A8B22168C8612046FFF738FF1D
:1062700000B10126304670BD10B50248FEF7B6F8F1
:1062800010BD00002004002010B50248FEF7AEF853
:1062900010BD00007804002010B50248FEF7A6F8F3
:1062A00010BD0000D004002010B504462068C0686E
:1062B000A16B0880A06B801CA063E08F401EE0876C
:1062C000E08F88B9A06AB0F5005F02D1074820646A
:1062D00010BD2068406820F0400021684860E08ED2
:1062E00010B9204600F0AAF800BFF1E7F1620008FB
:1062F00038B50446002000902068C068009000BFB8
:106300002068406820F0400021684860204600F086
:1063100095F838BD10B504462068007BA16B087065
:10632000A06B401CA063E08F401EE087E08F88B91F
:10633000A06AB0F5005F02D10748206410BD206854
:10634000406820F0600021684860E08E10B9204667
:1063500000F074F800BFF1E75D63000838B504464B
:1063600000200090206800F10C05287800909DF82E
:1063700000002068406820F0600021684860E08EDE
:1063800010B9204600F05AF838BD10B50446206B0D
:1063900000882168C860206B801C2063E08E401E4E
:1063A000E086E08ED8B9A06AB0F5005F0CD1206815
:1063B000006840F48050216808602068406820F040
:1063C00080002168486010BD2068406820F080008F
:1063D00021684860E08F10B9204600F02FF800BF18
:1063E000F1E710B50446206B007821680873206B34
:1063F000401C2063E08E401EE086E08ED8B9A06A83
:10640000B0F5005F0CD12068006840F4805021682E
:1064100008602068406820F080002168486010BD56
:106420002068406820F0800021684860E08F10B943
:10643000204600F003F800BFF1E700007CB50446F9
:106440003F4800681821B0FBF1F04FF47A71B0FBBF
:10645000F1F0642148430190FBF7BCFE054620683B
:10646000406820F020002168486000BF019820B9F2
:10647000606D40F02000606508E00198401E0190CA
:106480002068806800F002000028EFD000BF2A4694
:106490006421204600F060F818B1606D40F02000E3
:1064A0006065A06850B900BF002000902068C068F7
:1064B000009020688068009000BF00BF206880685E
:1064C000C0F3001008B3204600F05AF8012817D195
:1064D00084F85100606D40F00200606500BF2068E4
:1064E000006820F40050216808602068006840F4CB
:1064F00000502168086000BF2046FDF775FF1EE0D0
:106500004FF6EF702168886019E0606D88B994F8E3
:106510005100042806D1012084F851002046FEF7DE
:106520005DFA0CE0012084F851002046FEF7D0FA15
:1065300005E0012084F851002046FDF755FF7CBDA1
:106540000000002070B505466C6A0020E087E086F8
:106550002046FDF749FF70BDF8B504460D461646C6
:106560002B46002280212046009600F00DF828B12D
:10657000606D40F0200060650320F8BD0020FCE75E
:1065800001460120704700002DE9F84F04460D46F2
:1065900090461E46DDF82890FBF71CFEA0EB090094
:1065A000371AFBF717FE82462C480068C0F3CB3041
:1065B0007843009045E0701C002842D0FBF70AFEAB
:1065C000A0EB0A00B84200D2A7BB2068406820F0C8
:1065D000E000216848606068B0F5827F0DD1A06856
:1065E000B0F5004F03D0A068B0F5806F05D12068EA
:1065F000006820F0400021680860A06AB0F5005FE4
:106600000DD100BF2068006820F4005021680860A8
:106610002068006840F400502168086000BF012035
:1066200084F8510000BF002084F8500000BF032010
:10663000BDE8F88FFFE7009800B900270098401EDA
:106640000090206880682840A84201D1012000E025
:1066500000204045AFD10020EAE700000000002004
:10666000704710B5FCF7F0FD10BD00004FF0006062
:10667000014908607047000008ED00E010B50248CD
:10668000FEF74DFA10BD00002805002010B50248A5
:10669000FEF788FB10BD00009806002010B50248E8
:1066A000FEF780FB10BD0000DC06002070B505463B
:1066B0006C6A0020E085E0842046FEF771FB70BD27
:1066C0000168C96821F490710268D1600168496964
:1066D00021F0010102685161016B012905D10168B6
:1066E000C96821F010010268D160202180F83E10B5
:1066F00000210163704710B504462068C06820F08F
:1067000040002168C860202084F83D002046FFF743
:106710000DF8002010BDF8B5044694F83E0022287C
:1067200069D1A068B0F5805F0CD1206950B900250F
:10673000A66A20684068C0F308003080A06A801C08
:10674000A06215E0A56A0026A068B0F5805F03D0BE
:10675000A06828B9206918B920684068287004E04A
:106760002068406800F07F002870A06A401CA0628A
:10677000E08D401E80B2E085A8BB2068C06820F094
:1067800020002168C8602068C06820F480702168FB
:10679000C8602068406920F001002168486120201D
:1067A00084F83E00206B01281ED100202063206861
:1067B000C06820F010002168C8602068006800F000
:1067C000100010280AD100BF002000902068006847
:1067D000009020684068009000BF00BFA18D204657
:1067E000FEF7BFFA03E004E02046FEF7EFFE0020CC
:1067F000F8BD0020FCE70220FAE7000070B504466F
:106800002168096921F44051E2681143226811614D
:106810002269A1681143626941EA02052168C968D9
:1068200041F20C62914329432268D1602168496991
:1068300021F44071A2691143226851612D4A2168F7
:10684000914202D1FDF70AF801E0FCF7F7FF00EBF7
:10685000C00101EB001162689200B1FBF2F100EBA4
:10686000C00202EB001263689B00B2FBF3F26423E8
:10687000B2FBF3F202EBC20303EB0212A1EB8201C3
:10688000322202EB01116422B1FBF2F101F0F001BE
:1068900000EBC00202EB001263689B00B2FBF3F254
:1068A0006423B2FBF3F201EB021200EBC00101EB37
:1068B000001163689B00B1FBF3F100EBC00303EB35
:1068C00000136668B600B3FBF6F36426B3FBF6F379
:1068D00003EBC30606EB0313A1EB8301322303EBA7
:1068E00001116423B1FBF3F101F00F01114422689F
:1068F000916070BD0038014010B5034699629A85D9
:10690000DA8500201864222083F83E0000BF0020B2
:1069100083F83C0000BF1868C06840F480701C68B1
:10692000E0601868406940F001001C686061186808
:10693000C06840F020001C68E060002010BD0146E7
:1069400091F83D00212828D18868B0F5805F0BD1EF
:10695000086948B90A6A1088C0F308000B685860D3
:10696000086A801C086205E00B6A581C08621878E7
:106970000B685860C88C401E80B2C88458B908683B
:10698000C06820F080000B68D8600868C06840F0DC
:1069900040000B68D860002070470220FCE7000030
:1069A00010B50248FEF7FEF910BD0000CC0500202E
:1069B00010B50248FEF7F6F910BD000010060020E1
:1069C00010B50248FEF7EEF910BD00005406002095
:1069D00004E0012007F019FF07F0DEFEF9E70000F0
:1069E00010B50248FEF700FF10BD00002007002090
:1069F000F0B587B004460D46002600274FF6FF701D
:106A0000069038A103C9CDE904010020009001904F
:106A100002900390A0788DF8100006AA062104A821
:106A2000236B9847BDF81800C0B28DF81600BDF86A
:106A30001800000A8DF81700082104A8A26A9047E0
:106A40000F216846626A90479DF80000A17888424D
:106A500002D0701E07B0F0BD4FF6FF70069006AA78
:106A60000D216846236B98479DF80D009DF80E1088
:106A700040EA0120BDF81810884202D04FF0FF30E4
:106A8000E8E72878012810D19DF8060000069DF857
:106A9000051040EA01409DF8041040EA01209DF8ED
:106AA000031040EA010637466F606878012810D16C
:106AB0009DF80A0000069DF8091040EA01409DF883
:106AC000081040EA01209DF8071040EA0106374609
:106AD000AF6094F82000012802D19DF80B00A87047
:106AE0000020B7E7010326000005000010B586B0BE
:106AF00004464FF6FF70059020A003C8CDE90301BE
:106B0000002001900290A0788DF80C0005AA0621C3
:106B100003A8236B9847BDF81400C0B28DF812008B
:106B2000BDF81400000A8DF81300082103A8A26A1A
:106B30009047072101A8626A90479DF80400A17858
:106B4000884203D04FF0FF3006B010BD4FF6FF7003
:106B5000059005AA052101A8236B98479DF8090017
:106B60009DF80A1040EA0120BDF81410884202D0B6
:106B70004FF0FF30E8E70020E6E7000001032500C2
:106B80000001000030B585B004460D464FF6FF7099
:106B9000049024A103C9CDE90201002000900190D6
:106BA000A0788DF8080004AA062102A8236B984754
:106BB000BDF81000C0B28DF80E00BDF81000000A3C
:106BC0008DF80F00082102A8A26A904707216846A5
:106BD000626A90479DF80000A178884203D04FF088
:106BE000FF3005B030BD4FF6FF70049004AA0521B8
:106BF0006846236B98479DF805009DF8061040EA0B
:106C00000120BDF81010884202D04FF0FF30E8E7B5
:106C10009DF803009DF8041040EA01202880002020
:106C2000DFE70000010332000001000070B50446F8
:106C30000025204600F072F80546002D02DA4FF0DC
:106C4000FF3070BD204600F0C3F80546002D02DA83
:106C50004FF0FF30F5E794F8200058B1204600F0DF
:106C600025F90546002D02DA4FF0FF30E9E720460E
:106C700000F006F84FF47A60E16A88470020E0E708
:106C800010B586B004464FF6FF70059020A207CAE3
:106C900002AB07C3002000900190A0788DF8080097
:106CA00005AA072102A8236B9847BDF81400C0B2BB
:106CB0008DF80F00BDF81400000A8DF810000921AE
:106CC00002A8A26A904708216846626A90479DF828
:106CD0000000A178884203D04FF0FF3006B010BD0D
:106CE0004FF6FF70059005AA06216846236B98476A
:106CF0009DF806009DF8071040EA0120BDF8141029
:106D0000884202D04FF0FF30E8E70020E6E70000BD
:106D100001103100000000000000000010B586B036
:106D200004464FF6FF70059026A207CA02AB07C3C0
:106D300000200090019020886188884202D10020C4
:106D400006B010BD20788DF80800A0788DF80F00EF
:106D50006088000A8DF8100005AA092102A8236B9B
:106D60009847BDF81400C0B28DF81100BDF81400AA
:106D7000000A8DF812000B2102A8A26A9047082190
:106D80006846626A90479DF800002188884202D0D8
:106D90004FF0FF30D4E74FF6FF70059005AA0621AB
:106DA0006846236B98479DF806009DF8071040EA57
:106DB0000120BDF81410884202D04FF0FF30BFE729
:106DC0000020BDE7101030000001020000000000AC
:106DD00070B588B00446002500264FF6FF70079076
:106DE00014222DA102A8F9F71CFA002000900190AE
:106DF000A569E669A0788DF80800280E8DF81200C4
:106E0000280C8DF81100280A8DF81000E8B28DF8D2
:106E10000F00300E8DF81600300C8DF81500300A7A
:106E20008DF81400F0B28DF8130007AA0F2102A804
:106E3000236B9847BDF81C00C0B28DF81700BDF851
:106E40001C00000A8DF81800112102A8A26A9047C0
:106E500008216846626A90479DF80000A178884240
:106E600003D04FF0FF3008B070BD4FF6FF700790B1
:106E700007AA06216846236B98479DF806009DF8EF
:106E8000071040EA0120BDF81C10884202D04FF0E4
:106E9000FF30E8E70020E6E70110110000040800D9
:106EA00000000000000000000000000010B588B0E5
:106EB00004464FF6FF7007902BA1D1E900028968C4
:106EC000CDE90521049000200290039001A92046FD
:106ED000FFF758FE608CBDF80410884202D10020F4
:106EE00008B010BDA0788DF8100094F822008DF83D
:106EF0001700608C000A8DF8180007AA092104A861
:106F0000236B9847BDF81C00C0B28DF81900BDF87E
:106F10001C00000A8DF81A000B2104A8A26A9047F1
:106F2000082102A8626A90479DF80800A17888426B
:106F300002D04FF0FF30D3E74FF6FF70079007AA5B
:106F4000062102A8236B98479DF80E009DF80F10AC
:106F500040EA0120BDF81C10884202D04FF0FF30FB
:106F6000BEE70020BCE70000011032000001020073
:106F700000000000F0B587B004460D46002600274B
:106F80004FF6FF70069035A103C9CDE9040100203A
:106F90000090019002900390A0788DF8100006AA4E
:106FA000062104A8E36A9847BDF81800C0B28DF81E
:106FB0001600BDF81800000A8DF81700082104A873
:106FC000626A90470F216846226A90479DF8000048
:106FD000A178884202D0701E07B0F0BD4FF6FF7056
:106FE000069006AA0D216846E36A98479DF80D00B1
:106FF0009DF80E1040EA0120BDF81810884202D01A
:107000004FF0FF30E8E72878012810D19DF80600FE
:1070100000069DF8051040EA01409DF8041040EA82
:1070200001209DF8031040EA010637466F6068783A
:10703000012810D19DF80A0000069DF8091040EAC9
:1070400001409DF8081040EA01209DF8071040EA31
:1070500001063746AF600020BEE7000001032600AE
:107060000005000010B586B004464FF6FF7005908D
:1070700020A003C8CDE90301002001900290A07870
:107080008DF80C0005AA062103A8E36A9847BDF80D
:107090001400C0B28DF81200BDF81400000A8DF87B
:1070A0001300082103A8626A9047072101A8226AF9
:1070B00090479DF80400A178884203D04FF0FF303C
:1070C00006B010BD4FF6FF70059005AA052101A876
:1070D000E36A98479DF809009DF80A1040EA0120EC
:1070E000BDF81410884202D04FF0FF30E8E70020CE
:1070F000E6E70000010325000001000070B504462A
:107100000025204600F016F80546002D02DA4FF063
:10711000FF3070BD204600F067F80546002D02DA0A
:107120004FF0FF30F5E741F28830A16A8847002030
:10713000EFE7000010B586B004464FF6FF700590EB
:1071400026A207CA02AB07C3002000900190208846
:107150006188884202D1002006B010BD20788DF8E9
:107160000800A0788DF80F006088000A8DF81000E4
:1071700005AA092102A8E36A9847BDF81400C0B225
:107180008DF81100BDF81400000A8DF812000B21D3
:1071900002A8626A904708216846226A90479DF8D3
:1071A00000002188884202D04FF0FF30D4E74FF62C
:1071B000FF70059005AA06216846E36A98479DF886
:1071C00006009DF8071040EA0120BDF8141088421F
:1071D00002D04FF0FF30BFE70020BDE701103000C4
:1071E000000102000000000070B588B004460025D0
:1071F00000264FF6FF70079014222DA102A8F9F780
:1072000010F8002000900190A569E669A0788DF83B
:107210000800280E8DF81200280C8DF81100280A9D
:107220008DF81000E8B28DF80F00300E8DF81600C2
:10723000300C8DF81500300A8DF81400F0B28DF87E
:10724000130007AA0F2102A8E36A9847BDF81C00A3
:10725000C0B28DF81700BDF81C00000A8DF81800A8
:10726000112102A8626A904708216846226A904765
:107270009DF80000A178884203D04FF0FF3008B09D
:1072800070BD4FF6FF70079007AA06216846E36AB3
:1072900098479DF806009DF8071040EA0120BDF8C8
:1072A0001C10884202D04FF0FF30E8E70020E6E7EC
:1072B00001101100000408000000000000000000A0
:1072C00000000000FEB505460E460A2D71D2DFE82B
:1072D00005F005082023263F58728BA44FF0FF309D
:1072E000FEBD0120009001900520029069465A4899
:1072F000F9F7E4FF10B14FF0FF30F1E7314656489F
:1073000000F0ACF80446002C02DA4FF0FF30E7E75B
:107310009FE04FF0FF30E3E74FF0FF30E0E704205D
:107320000090012001900520029069464A48F9F733
:10733000C5FF10B14FF0FF30D2E73146464800F0AC
:107340008DF80446002C02DA4FF0FF30C8E780E0E9
:1073500005200090012001900520029069463E48DA
:10736000F9F7ACFF10B14FF0FF30B9E731463A48BA
:1073700000F074F80446002C02DA4FF0FF30AFE75B
:1073800067E00620009001200190052002906946E8
:107390003148F9F793FF10B14FF0FF30A0E73146C5
:1073A0002D4800F05BF80446002C03DA4FF0FF3064
:1073B00096E74BE04DE0072000900120019005206A
:1073C000029069462448F9F779FF10B14FF0FF3079
:1073D00086E73146204800F041F80446002C02DAE6
:1073E0004FF0FF307CE734E008200090012001904E
:1073F0000520029069461848F9F760FF10B14FF078
:10740000FF306DE73146144800F028F80446002CA0
:1074100002DA4FF0FF3063E71BE009200090012003
:1074200001900520029069460B48F9F747FF10B11B
:107430004FF0FF3054E73146074800F00FF804469C
:10744000002C02DA4FF0FF304AE702E04FF0FF3045
:1074500046E700BF002043E7FC0100202DE9F34F81
:1074600097B08946502103A8F8F7F4FE002007469C
:1074700080468246039D039E002427E01798FAF772
:1074800057FA32211798FAF793F91798F9F7C6FFC8
:1074900000F4007070B11798F9F7C3FF03A941F821
:1074A000240003A850F82400C71948F10008601C04
:1074B000C4B20BE00AF1010000F0FF0ABAF1640F58
:1074C00004DD4FF0FF3019B0BDE8F08F142CD5DB90
:1074D0001798FAF7C5FA039D039E002417E003A846
:1074E00050F82400A84201D2284602E003A850F830
:1074F0002400054603A850F82400B04201D93046C4
:1075000002E003A850F824000646601CC4B2142C04
:10751000E5DB791B68F100008A1B60F10001104671
:10752000F9F7CEF809490190F8F768FF029008488A
:1075300001680298F8F730FF83464FF08B41F8F767
:107540005DFFC9F800000020BDE700000000904189
:107550001000002010B52E480078012801D100202D
:1075600010BD2C482C4908600020486000212A48A2
:107570008160017301210161002101750121816197
:107580004FF46021C161F9F751FF10B14FF0FF30A6
:10759000E6E7224822490860002048600021204890
:1075A0008160017301210161002101750121816167
:1075B0004FF46021C161F9F739FF10B14FF0FF308E
:1075C000CEE7184818490860002048600021164896
:1075D0008160017301210161002101750121816137
:1075E0004FF46021C161F9F721FF10B14FF0FF3076
:1075F000B6E70948F9F7D6FD0948F9F7D3FD0A4877
:10760000F9F7D0FD0120024908700020A8E700002A
:107610001400002000240140FC010020002801404B
:107620002C020020003C01405C0200200A48007847
:1076300001280FD10948806920F40070074988614A
:107640000846806920F4806088610846806920F4DB
:1076500000408861704700001400002000100240C4
:1076600000B585B07748007801287DD100BF764805
:10767000806940F40070744988610846806900F4AC
:107680000070009000BF00BF00BF0846806940F452
:10769000806088610846806900F48060009000BFC7
:1076A00000BF00BF0846806940F40040886108467A
:1076B000806900F40040009000BF00BF00BF084692
:1076C000806940F0040088610846806900F0040089
:1076D000009000BF00BF0220019003200290002014
:1076E000039001A95948FAF7C7FB00BF56488069C3
:1076F00040F00400544988610846806900F00400A5
:10770000009000BF00BF10200190032002900020D5
:10771000039001A94D48FAF7AFFB00BF4A488069C2
:1077200040F00400484988610846806900F0040080
:10773000009000BF00BF2020019003200290002095
:10774000039001A94148FAF797FB00BF3E488069C2
:1077500040F004003C4988610846806900F004005C
:10776000009000BF00BF00E069E0402001900320CE
:1077700002900020039001A93448FAF77DFB00BF76
:107780003148806940F004002F49886108468069CB
:1077900000F00400009000BF00BF80200190032093
:1077A00002900020039001A92848FAF765FB00BF6A
:1077B0002548806940F008002349886108468069AF
:1077C00000F00800009000BF00BF012001900320DE
:1077D00002900020039001A91D48FAF74DFB00BF5D
:1077E0001948806940F00800174988610846806997
:1077F00000F00800009000BF00BF022001900320AD
:1078000002900020039001A91148FAF735FB00BF50
:107810000D48806940F010000B4988610846806976
:1078200000F01000009000BF00BF01200190032075
:1078300002900020039001A90648FAF71DFB05B04D
:1078400000BD0000140000200010024000080140AC
:10785000000C01400010014070B504460D46294659
:107860002046FAF7A9FC0646012E00D170BD002083
:10787000FCE700002DE9F04186B004460D461646AF
:107880001F46DDF83080434884420DD100BF424896
:10789000806940F00400404988610846806900F032
:1078A0000400019000BF6AE03C4884420DD100BF53
:1078B0003948806940F00800374988610846806986
:1078C00000F00800019000BF59E0354884420DD116
:1078D00000BF3148806940F010002F498861084698
:1078E000806900F01000019000BF48E02D488442FC
:1078F0000DD100BF2848806940F0200026498861EA
:107900000846806900F02000019000BF37E026485B
:1079100084420DD100BF2048806940F040001E49DC
:1079200088610846806900F04000019000BF26E0B1
:107930001E4884420DD100BF1748806940F0800086
:10794000154988610846806900F08000019000BFF9
:1079500015E0174884420DD100BF0F48806940F4FC
:1079600080700D4988610846806900F4807001903C
:1079700000BF04E04FF0FF3006B0BDE8F081029593
:1079800003960597CDF8108002A92046FAF774FAFD
:107990000020F1E70008014000100240000C014007
:1079A000001001400014014000180140001C01407B
:1079B0000020014070B505460E461446012C04D146
:1079C00031462846FAF700FC04E0002231462846FA
:1079D000FAF7FAFB70BD00002F48007800F00100B4
:1079E00028B92E48806920F004002C4988612A4873
:1079F000007800F00200022805D02848806920F0B5
:107A00000800264988612448007800F00400042812
:107A100005D02248806920F01000204988611E4866
:107A2000007800F00800082805D01C48806920F084
:107A300020001A4988611848007800F010001028CA
:107A400005D01648806920F040001449886112482A
:107A5000007800F02000202805D01048806920F030
:107A600080000E4988610C48007800F040004028F2
:107A700005D00A48806920F480700849886106486A
:107A8000007800F07F007F2805D00448806920F04E
:107A90000100024988617047150000200010024073
:107AA00008B55048007800F07F007F280DD000BF57
:107AB0004D48806940F001004B4988610846806963
:107AC00000F00100009000BF00BF4648007800F0C1
:107AD000010068B900BF4448806940F00400424991
:107AE00088610846806900F00400009000BF00BF74
:107AF0003C48007800F0020002280DD000BF3A4850
:107B0000806940F00800384988610846806900F0C3
:107B10000800009000BF00BF3248007800F0040069
:107B200004280DD000BF3048806940F010002E4975
:107B300088610846806900F01000009000BF00BF17
:107B40002848007800F0080008280DD000BF26481B
:107B5000806940F02000244988610846806900F06F
:107B60002000009000BF00BF1E48007800F0100009
:107B700010280DD000BF1C48806940F040001A4911
:107B800088610846806900F04000009000BF00BF97
:107B90001448007800F0200020280DD000BF1248C3
:107BA000806940F08000104988610846806900F0D3
:107BB0008000009000BF00BF0A48007800F040003D
:107BC00040280DD000BF0848806940F48070064905
:107BD00088610846806900F48070009000BF00BF93
:107BE00008BD0000150000200010024010B504463A
:107BF000012C26D128480078012801D1002010BD91
:107C000026482749086027484860002124488160A9
:107C10000F21C1604FF48041016100214161FF21CA
:107C200081610021C1610162FAF7DAFA1C48FAF7B2
:107C3000F5FA10B14FF0FF30E1E701201649087066
:107C400028E0022C26D118480078012801D1002014
:107C5000D5E71648164908601248486000211448C4
:107C6000816040F20F31C1604FF480410161002119
:107C70004161FF2181610021C1610162FAF7B0FA1F
:107C80000B48FAF7CBFA10B14FF0FF30B7E70120FD
:107C9000054908700020B2E716000020005400409B
:107CA000C4020020801A060017000020005800407F
:107CB000180300202DE9FE4F05460C4690469946D4
:107CC000DDE90CA60E9F0DBB012C0DD14FF4967073
:107CD0003B463246414600903048FAF787FB002881
:107CE0005AD0A01EBDE8FE8F022C0CD14FF4967026
:107CF0003B463246414600902948FAF777FB002878
:107D00004AD0E01EEEE74FF0FF30EBE7012D1AD12D
:107D1000012C09D14FF496733A4631461F48FBF7C0
:107D200009F990B3A01EDDE7022C09D14FF4967338
:107D30003A4631461A48FBF7FDF830B3E01ED1E76A
:107D40004FF0FF30CEE7022D23D1012C0DD14FF49F
:107D5000967053464A464146CDE9006702900F4867
:107D6000FAF7A8FD88B1A01EBCE7022C0ED14FF493
:107D7000967053464A464146CDE90067029008484E
:107D8000FAF798FD08B1E01EACE705E04FF0FF30D0
:107D9000A8E74FF0FF30A5E70020A3E7C4020020CA
:107DA000180300202DE9FE4F05460C4690469946E3
:107DB000DDE90CA60E9F0DBB012C0DD14FF4967082
:107DC0003B463246414600903048FAF7BBFC00285B
:107DD0005AD0A01EBDE8FE8F022C0CD14FF4967035
:107DE0003B463246414600902948FAF7ABFC002852
:107DF0004AD0E01EEEE74FF0FF30EBE7012D1AD13D
:107E0000012C09D14FF496733A4631461F48FBF7CF
:107E100051F990B3A01EDDE7022C09D14FF49673FF
:107E20003A4631461A48FBF745F930B3E01ED1E730
:107E30004FF0FF30CEE7022D23D1012C0DD14FF4AE
:107E4000967053464A464146CDE9006702900F4876
:107E5000FAF7E2FE88B1A01EBCE7022C0ED14FF467
:107E6000967053464A464146CDE90067029008485D
:107E7000FAF7D2FE08B1E01EACE705E04FF0FF30A4
:107E8000A8E74FF0FF30A5E70020A3E7C4020020D9
:107E90001803002000B585B000BF3848806940F065
:107EA0000800364988610846806900F008000090A3
:107EB00000BF00BF00BF0846806940F0080088612D
:107EC0000846806900F00800009000BF00BF402015
:107ED000019012200290012003900320049001A938
:107EE0002748F9F7C9FF8020019001A92448F9F734
:107EF000C3FF24480078012805D12048C06920F438
:107F000000101E49C86100BF1C48806940F008008D
:107F10001A4988610846806900F00800009000BF97
:107F200000BF00BF0846806940F00800886108462D
:107F3000806900F00800009000BF00BF08150190A4
:107F400012200290012003900320049001A90C4804
:107F5000F9F792FF4FF40060019001A90848F9F782
:107F60008BFF09480078012805D10448C06920F436
:107F700080000249C86105B000BD00000010024049
:107F8000000C0140160000201700002008B5124820
:107F9000007801280DD100BF1048C06940F40010DE
:107FA0000E49C8610846C06900F40010009000BF87
:107FB00000BF0B48007801280DD100BF0748C069F9
:107FC00040F480000549C8610846C06900F480009B
:107FD000009000BF00BF08BD160000200010024046
:107FE00017000020014800787047000019000020A9
:107FF0001CB504460020019000900CB9401E1CBD29
:10800000002201A91548FBF716FF10B14FF0FF3011
:10801000F5E7002269461148FBF7E4FE10B14FF086
:10802000FF30ECE79DF8040020709DF805006070BB
:108030009DF80600A0709DF80100E0709DF8020018
:1080400020719DF803000649097801EBC10202EB9B
:10805000011100EB8100E0800020D0E70C0400203B
:108060001800002010B50848084908604FF0FF309C
:108070004860002105488160FBF760FF10B14FF0B8
:10808000FF3010BD0020FCE7002800400C04002059
:108090001CB504460020019000900CB9401E1CBD88
:1080A00020788DF8040060788DF80500A0788DF8B0
:1080B0000600E0788DF8010020798DF80200E08854
:1080C000642190FBF1F201FB1200C0B28DF80300B5
:1080D000E08890FBF1F00C490870002269460B48DB
:1080E000FCF754F810B14FF0FF30D8E7002201A997
:1080F0000648FCF7C7F810B14FF0FF30CFE701207A
:10810000034908700020CAE7180000200C04002072
:10811000190000203EB505460C4600200190029053
:10812000009094480470002269469348FBF783FE50
:1081300010B14FF0FF303EBD00200290062D7DD0E3
:1081400006DC052D7BD2DFE805F02A4F617E980022
:10815000082D75D00C2D74D0182D73D0FF2D6ED135
:108160009DF80100801C3C2806DD9DF80000401CA5
:10817000C0B28DF8040003E09DF800008DF8040003
:108180009DF80100801C3C2190FBF1F201FB1200E4
:10819000C0B28DF8050000208DF80600DEE09DF8E5
:1081A00001001E303C2806DD9DF80000401CC0B2D6
:1081B0008DF8040003E09DF800008DF804009DF8A0
:1081C00001001E303C2808DD9DF801001E305A28B1
:1081D00003DA00208DF8050002E01E208DF805006E
:1081E00000208DF80600B9E09DF800000121084448
:1081F000182190FBF1F201FB1200C0B28DF80400CF
:1082000000208DF805008DF80600A7E09DF800001D
:1082100000EBD0714910A0EB4101C1F10201014412
:10822000182291FBF2F302FB1311C9B28DF804106E
:1082300000208DF805008DF806008FE036E08AE01A
:108240004EE066E07FE09DF80000032190FBF1F234
:1082500001FB1200C0F103009DF800100844182132
:1082600090FBF1F201FB1200C0B28DF80400002077
:108270008DF805008DF8060070E09DF80000C1172C
:1082800000EB91718910A0EB8101C1F1040101445F
:10829000182291FBF2F302FB1311C9B28DF80410FE
:1082A00000208DF805008DF8060057E09DF80000CD
:1082B000062190FBF1F201FB1200C0F106009DF8CF
:1082C00000100844182190FBF1F201FB1200C0B22B
:1082D0008DF8040000208DF805008DF806003DE0C3
:1082E0009DF80000C11700EB5171C910A0EBC1014E
:1082F000C1F108010144182291FBF2F302FB1311B2
:10830000C9B28DF8041000208DF805008DF8060024
:1083100024E09DF800000C2190FBF1F201FB12001B
:10832000C0F10C009DF800100844182190FBF1F2F8
:1083300001FB1200C0B28DF8040000208DF805008A
:108340008DF806000AE000208DF804008DF8050085
:108350008DF8060002E04FF0FF30ECE600BF00228F
:1083600001A90548FBF78CFE10B14FF0FF30E2E6A3
:108370000020E0E61A0000200C04002070B504463E
:108380000D46012C00D170BD022C00D1FBE7032C5F
:1083900005D12A464FF400410248F9F715FF00BF06
:1083A000F1E700000008014010B50446012C01D19E
:1083B000801E10BD022C01D1E01EFAE7032C2ED145
:1083C00019480078012801D10020F2E71748184920
:1083D000086030211648C16100218160416101615E
:1083E000C1600162416281620721C1624FF4007184
:1083F00081614FF482700E4948600846FBF7D9FF4F
:1084000010B14FF0FF30D4E70948FCF789F810B1FC
:108410004FF0FF30CDE701200349087002E04FF034
:10842000FF30C6E70020C4E71D000020003C0040EC
:10843000D004002013B582B00446012C02D10020E4
:1084400004B010BD022C01D10020F9E7032C11D19A
:1084500000BF0A4890F851000128FAD1012301AA6F
:1084600003A90648FCF7BCFA00BF044890F8510085
:108470000128FAD19DF80400E2E70000D0040020B2
:108480000246012A01D1801E7047022A01D1D01E66
:10849000FAE7032A3AD181B91F480068006820F042
:1084A00038001D4B1B6818601B480068006840F0CE
:1084B0000800194B1B6818602BE0012910D11648E1
:1084C0000068006820F03800134B1B6818601248E1
:1084D0000068006840F020000F4B1B68186018E02F
:1084E000022910D10C480068006820F038000A4BBF
:1084F0001B68186008480068006840F03000064BB0
:108500001B68186005E04FF0FF30BDE74FF0FF300B
:10851000BAE70020B8E70000D004002000B585B01D
:1085200034480078012808D13348C06920F400405D
:108530003149C8613320FAF7CFFE00BF2E48806969
:1085400040F008002C4988610846806900F0080066
:10855000009000BF00BF00BF0846806940F00800DF
:1085600088610846806900F00800009000BF00BFE5
:1085700000BF0846806940F00800886108468069AD
:1085800000F00800009000BF00BF00BF08468069EF
:1085900040F0040088610846806900F00400009003
:1085A00000BF00BF0820019011200290022003901C
:1085B000049001A91148F9F75FFC102001900220F6
:1085C000039001A90D48F9F757FC202001900220E3
:1085D000039001A90948F9F74FFC01200290C0035C
:1085E00001900120039001A90548F9F745FC05B069
:1085F00000BD00001D00002000100240000C0140E2
:108600000008014000B585B03848007801286BD1DA
:1086100000BF3748806940F0080035498861084646
:10862000806900F00800009000BF00BF00BF08464E
:10863000806940F0080088610846806900F0080001
:10864000009000BF00BF00BF0846806940F00800EE
:1086500088610846806900F00800009000BF00BFF4
:1086600000BF0846806940F00400886108468069C0
:1086700000F00400009000BF00BF0820019002201D
:108680000290002003900320049001A91948F9F7F3
:10869000F3FB102001900020039001A91548F9F781
:1086A000EBFB202001900020039001A91148F9F76D
:1086B000E3FB4FF40040019001200290039001A9D8
:1086C0000D48F9F7D9FB00BF0948C06940F40040E4
:1086D0000749C8610846C06900F40040009000BF27
:1086E00000BF3320FAF71AFE05B000BD1D000020C0
:1086F00000100240000C01400008014000B58FB09E
:1087000014210AA8F7F7A6FD28216846F7F7A2FD6D
:108710000120009000040190002003900490069036
:10872000102005900020029002200790C1030891BC
:108730004FF4E01109916846FBF7EAF808B100BF71
:10874000FEE70F200A9002200B9000200C900E9064
:108750004FF480600D9002210AA8FAF7A3FF08B138
:1087600000BFFEE70FB000BD08B5FAF779FDFFF7CF
:10877000C5FF00BF1648C06940F080501449C86169
:108780000846C06900F08050009000BF00BF00BFE5
:108790000846806940F0010088610846806900F061
:1087A0000100009000BF00BF00BF0A49486820F0E8
:1087B000E06040F00070486000BF00BF486840F0D3
:1087C000E06040F40040486000BF002008BD0000A9
:1087D00000100240000001402DE9F04105460C4622
:1087E00016461F46012D39D195480078012802D13F
:1087F0000020BDE8F08193489349086054B94FF4D4
:10880000E1304860002190488160C16001610C2125
:1088100041610BE08C49206848608B486168816049
:10882000A168C160E1680161216941610021864858
:108830008161FCF797FA10B14FF0FF30D9E7824819
:10884000FCF7D6FB10B14FF0FF30D2E77F4806604F
:108850007F48076001207A490870EEE0022D38D188
:108860007C480078012801D10020C2E77A487B4982
:10887000086054B94FF41650486000217748816071
:10888000C16001610C2141610BE0744920684860BE
:10889000724861688160A168C160E1680161216915
:1088A000416100216D488161FCF75CFA10B14FF025
:1088B000FF309EE76948FCF79BFB10B14FF0FF309B
:1088C00097E76748066067480760012061490870BC
:1088D000B3E0032D38D164480078012801D100208D
:1088E00087E762486249086054B94FF416504860FF
:1088F00000215F488160C16001610C2141610BE092
:108900005B49206848605A4861688160A168C1601D
:10891000E168016121694161002155488161FCF7ED
:1089200021FA10B14FF0FF3063E75148FCF760FBCC
:1089300010B14FF0FF305CE74E4806604E480760CC
:1089400001204949087078E0042D38D14B4800785F
:10895000012801D100204CE749484A49086054B930
:108960004FF416504860002146488160C1600161A3
:108970000C2141610BE0434920684860414861682F
:108980008160A168C160E1680161216941610021E4
:108990003C488161FCF7E6F910B14FF0FF3028E761
:1089A0003848FCF725FB10B14FF0FF3021E736487F
:1089B0000660364807600120304908703DE0052D0B
:1089C00038D133480078012801D1002011E731481F
:1089D0003149086054B94FF41650486000212E48C0
:1089E0008160C16001610C2141610BE02A4920686E
:1089F0004860294861688160A168C160E1680161DF
:108A000021694161002124488161FCF7ABF910B173
:108A10004FF0FF30EDE62048FCF7EAFA10B14FF0D6
:108A2000FF30E6E61D4806601D4807600120184932
:108A3000087002E04FF0FF30DBE60020D9E60000CE
:108A40002D00002000380140CC050020340000201B
:108A5000380000202E0000200044004010060020B6
:108A60003C000020400000202F0000200048004073
:108A70005406002044000020480000203000002060
:108A8000004C0040980600204C00002050000020C0
:108A90003100002000500040DC060020540000207F
:108AA0005800002070B504460D461646012C11D121
:108AB00000BF3D4890F83D002028FAD132462946B3
:108AC0003948FCF707FE00BF374890F83D002028E2
:108AD000FAD166E0022C11D100BF344890F83D0075
:108AE0002028FAD1324629463048FCF7F3FD00BF72
:108AF0002E4890F83D002028FAD152E0032C11D1E5
:108B000000BF2B4890F83D002028FAD13246294674
:108B10002748FCF7DFFD00BF254890F83D002028DE
:108B2000FAD13EE0042C1BD1012251022148F9F771
:108B30004BFB00BF204890F83D002028FAD1324678
:108B400029461D48FCF7C6FD00BF1B4890F83D00B4
:108B50002028FAD1002201011648F9F735FB20E060
:108B6000052C1BD1012211021448F9F72DFB00BF7F
:108B7000134890F83D002028FAD132462946104883
:108B8000FCF7A8FD00BF0E4890F83D002028FAD160
:108B90000022C1000948F9F717FB02E04FF0FF304F
:108BA00070BD0020FCE70000CC050020100600206E
:108BB00054060020001001409806002000200140CB
:108BC000DC06002000B585B0B0480078012805D14A
:108BD000AF48806920F48040AD4988612520FAF7CC
:108BE0007BFB00BFAA48806940F00400A849886167
:108BF0000846806900F00400009000BF00BF00BF7D
:108C00000846806940F0040088610846806900F0E9
:108C10000400009000BF00BF481501901120029091
:108C200002200390049001A99A48F9F725F94FF41E
:108C3000806001901120029002200390049001A90D
:108C40009448F9F719F994480078012805D190481B
:108C5000C06920F400308E49C8612620FAF73CFB39
:108C600000BF8B48806940F004008949886108464C
:108C7000806900F00400009000BF00BF00BF0846FC
:108C8000806940F0040088610846806900F00400B3
:108C9000009000BF00BF0820019011200290022028
:108CA0000390049001A97B48F9F7E6F87B48007827
:108CB000012805D17648C06920F480207449C86134
:108CC0002720FAF709FB00BF7148806940F02000B7
:108CD0006F4988610846806900F02000009000BF5D
:108CE00000BF00BF0846806940F020008861084648
:108CF000806900F02000009000BF00BF881501903F
:108D00001120029002200390049001A96448F9F711
:108D1000B3F84FF4007001901120029002200390EC
:108D2000049001A95E48F9F7A7F85E480078012889
:108D300005D15748C06920F400205549C861342046
:108D4000FAF7CAFA00BF5248806940F01000504953
:108D500088610846806900F01000009000BF00BFE5
:108D600000BF0846806940F01000886108468069AD
:108D700000F01000009000BF00BF08150190112006
:108D8000029002200390049001A94748F9F774F873
:108D90004FF4006001901120029002200390049093
:108DA00001A94148F9F768F800BF3948806940F0E7
:108DB0001000374988610846806900F01000009073
:108DC00000BF00BF481501901120029002200390BF
:108DD000049001A93448F9F74FF834480078012885
:108DE00005D12B48C06920F480102949C86135207D
:108DF000FAF772FA00BF2648806940F01000244953
:108E000088610846806900F01000009000BF00BF34
:108E100000BF0846806940F02000886108468069EC
:108E200000F02000009000BF00BF881401901120C6
:108E3000029002200390049001A91B48F9F71CF846
:108E4000042001901120029002200390049001A9B7
:108E50001348F9F711F800BF0D48806940F480709D
:108E60000B4988610846806900F48070009000BF5B
:108E700000BF8815019011200290022003900490F9
:108E800001A90B48F8F7F8FF05B000BD2D00002040
:108E900000100240000801402E0000202F0000209A
:108EA000001401403000002000100140310000207B
:108EB0000020014010B50446012C05D101221249C1
:108EC0001248FCF761FB1EE0022C05D1012210497B
:108ED0001048FCF759FB16E0032C05D101220E497E
:108EE0000E48FCF751FB0EE0042C05D101220C4981
:108EF0000C48FCF749FB06E0052C04D101220A4985
:108F00000A48FCF741FB10BD28000020CC050020DA
:108F100029000020100600202A000020540600200E
:108F20002B000020980600202C000020DC060020EA
:108F300000B585B0CC480078012843D100BFCB48AC
:108F4000806940F48040C94988610846806900F41E
:108F50008040009000BF00BF00BF0846806940F01D
:108F6000040088610846806900F00400009000BF9A
:108F700000BF00BF0846806940F0040088610846D1
:108F8000806900F00400009000BF00BF4815019008
:108F900002200290012003900320049001A9B4480C
:108FA000F8F76AFF4FF480600190002002900120E2
:108FB00003900320049001A9AD48F8F75DFF252038
:108FC000FAF7ACF9AB480078012836D100BFA748C2
:108FD000C06940F40030A549C8610846C06900F482
:108FE0000030009000BF00BF00BF0846806940F01D
:108FF000040088610846806900F00400009000BF0A
:1090000000BF00BF0846806940F004008861084640
:10901000806900F00400009000BF00BF08200190AC
:1090200000200290012003900320049001A99048A1
:10903000F8F722FF2620FAF771F98F480078012807
:1090400043D100BF8948C06940F480208749C86186
:109050000846C06900F48020009000BF00BF00BF38
:109060000846806940F0200088610846806900F069
:109070002000009000BF00BF00BF0846806940F09C
:10908000200088610846806900F02000009000BF41
:1090900000BF881501900220029001200390032058
:1090A000049001A97548F8F7E7FE4FF400700190AD
:1090B00000200290012003900320049001A96F4832
:1090C000F8F7DAFE2720FAF729F96D480078012829
:1090D00062D100BF6548C06940F400206349C8619F
:1090E0000846C06900F40020009000BF00BF00BF28
:1090F0000846806940F0100088610846806900F0E9
:109100001000009000BF00BF00BF0846806940F01B
:10911000100088610846806900F01000009000BFD0
:1091200000BF081501900220029001200390032047
:10913000049001A95348F8F79FFE4FF40060019096
:1091400000200290012003900320049001A94D48C3
:10915000F8F792FE00BF4548806940F0100043498F
:1091600088610846806900F01000009000BF00BFD1
:10917000481501900120029003900320049001A95A
:109180004048F8F779FE00224FF400713D48F9F7A6
:109190001BF83420FAF7C2F83B480078012861D167
:1091A00000BF3248C06940F480103049C8610846A9
:1091B000C06900F48010009000BF00BF00BF0846E7
:1091C000806940F0100088610846806900F0100056
:1091D000009000BF00BF00BF0846806940F020003B
:1091E00088610846806900F02000009000BF00BF41
:1091F0008814019002200290012003900320049023
:1092000001A92048F8F738FE0420019000200290C0
:10921000012003900320049001A91848F8F72CFEC0
:1092200000BF1248806940F4807010498861084688
:10923000806900F48070009000BF00BF8815019025
:109240000120029003900320049001A90F48F8F731
:1092500013FE00224FF480710C48F8F7B5FF35205B
:10926000FAF75CF805B000BD2D00002000100240A8
:10927000000801402E0000202F00002000140140B3
:10928000300000200010014031000020002001408B
:1092900010B500224FF480710148FEF78BFB10BD22
:1092A0000018014010B5002280210248FEF782FB21
:1092B00010BD00000014014010B5012280210248B9
:1092C000FEF778FB10BD00000014014008B5012036
:1092D00003230022410200903548FEF7CBFA01201B
:1092E00003230022810200903148FEF7C3FA0120D7
:1092F00003230022C10200902D48FEF7BBFA012093
:1093000003230022010300902948FEF7B3FA01204D
:1093100003230022410300902548FEF7ABFA012009
:1093200003230022810300902148FEF7A3FA0120C5
:1093300003230022C10300901D48FEF79BFA012081
:1093400003230022010200901A48FEF793FA00203E
:1093500003230122022100901748FEF78BFA012017
:1093600003230022014600901348FEF783FA0020F1
:1093700003230122202100901048FEF77BFA0020F1
:1093800003230122082100900C48FEF773FA002005
:1093900003230122510200900648FEF76BFA0020D9
:1093A00003230122802100900448FEF763FA08BDE0
:1093B00000200140000C0140001801400014014051
:1093C00008B5022003461122010200903748FEF73B
:1093D00051FA022003461122410200903348FEF761
:1093E00049FA022003461122810200902F48FEF71D
:1093F00041FA022003461122C10200902B48FEF7D9
:1094000039FA022003461122010300902748FEF793
:1094100031FA022003461122410300902348FEF74F
:1094200029FA022003461122810300901F48FEF70B
:1094300021FA022003461122C10100901C48FEF7C8
:1094400019FA022003461122014600901948FEF73E
:1094500011FA022003461122012100901548FEF75F
:1094600009FA022003461122202100901248FEF73B
:1094700001FA022003461122082100900E48FEF74F
:10948000F9F9022003461122010200900848FEF774
:10949000F1F9022003461122802100900648FEF7D0
:1094A000E9F901F063FA01F075FA08BD0020014006
:1094B000000C0140001801400014014010B50022CA
:1094C0004FF400710148FEF775FA10BD000C014021
:1094D00010B5012251020248FEF76CFA10BD0000DF
:1094E000000C014010B500F0AFFDFFF7E7FFFFF7FC
:1094F000EFFFFFF7E3FF00F0B1FD10BD10B504462C
:10950000002C7DD104223A21422001F0CEFA102213
:109510004021422001F0C9FA14221221422001F018
:10952000C4FA80223221422001F0BFFA162217210C
:10953000422001F0BAFA04221821422001F0B5FAC3
:1095400002221921422001F0B0FA7A221A21422087
:1095500001F0ABFA0A220321422001F0A6FA0C2204
:109560001146422001F0A1FA00221521422001F00B
:109570009CFA00223E21422001F097FA002270213D
:10958000422001F092FA01227121422001F08DFA6D
:1095900011227221422001F088FA0922732142200F
:1095A00001F083FA0222A221422001F07EFA002279
:1095B0001121422001F079FA20227A21422001F083
:1095C00074FA1C227B21422001F06FFA28227C21B0
:1095D000422001F06AFA3C227D21422001F065FA26
:1095E00055227E21422001F060FA68227F2142202C
:1095F00001F05BFA76228021422001F056FA00E069
:10960000C2E180228121422001F04FFA882282218A
:10961000422001F04AFA8F228321422001F045FACC
:1096200096228421422001F040FAA3228521422083
:1096300001F03BFAAF228621422001F036FAC42223
:109640008721422001F031FAD7228821422001F0FF
:109650002CFAE8228921422001F027FAE022132186
:10966000422001F022FA00221146422001F01DFAA8
:1096700000221021422001F018FA00220D21422080
:1096800001F013FA20221421422001F00EFA0522E3
:10969000A521422001F009FA0722AB21422001F066
:1096A00004FA75222421422001F0FFF963222521CA
:1096B000422001F0FAF9A5222621422001F0F5F915
:1096C00078229F21422001F0F0F96822A021422057
:1096D00001F0EBF90322A121422001F0E6F9DF229B
:1096E000A621422001F0E1F9DF22A721422001F06A
:1096F000DCF9F022A821422001F0D7F99022A9211B
:10970000422001F0D2F99422AA21422001F0CDF9A1
:10971000E5221321422001F0C8F961220E214220E6
:1097200001F0C3F94B220F21422001F0BEF90222C1
:109730001621422001F0B9F917221E21422001F022
:10974000B4F902222121422001F0AFF99122222115
:10975000422001F0AAF907222921422001F0A5F9AF
:109760000B223321422001F0A0F90B2235214220A7
:1097700001F09BF91D223721422001F096F9712258
:109780003821422001F091F92A223921422001F0AA
:109790008CF978223C21422001F087F940224D21AA
:1097A000422001F082F920224E21422001F07DF971
:1097B0005D226921422001F078F940226B2142208C
:1097C00001F073F919227421422001F06EF94F2241
:1097D0008D21422001F069F900228E21422001F002
:1097E00064F900228F21422001F05FF900229021CC
:1097F000422001F05AF900229121422001F055F94E
:1098000000229221422001F050F9002296214220AC
:1098100001F04BF980229A21422001F046F984227E
:10982000B021422001F041F90C22B121422001F087
:109830003CF90E22B221422001F037F98222B321F5
:10984000422001F032F90A22B821422001F02DF91C
:1098500014224321422001F028F9F0224421422021
:1098600001F023F934224521422001F01EF958224B
:109870004621422001F019F928224721422001F017
:1098800014F93A224821422001F00FF98822592187
:10989000422001F00AF988225A21422001F005F9FC
:1098A00044225B21422001F000F967225C21422022
:1098B00001F0FBF849225D21422001F0F6F80E226A
:1098C0005E21422001F0F1F804226421422001F0DF
:1098D000ECF820226521422001F0E7F805226621FC
:1098E000422001F0E2F804229421422001F0DDF848
:1098F00008229521422001F0D8F80A226C2142204A
:1099000001F0D3F855226D21422001F0CEF88022DB
:109910004F21422001F0C9F880225021422001F05D
:10992000C4F800225121422001F0BFF82222522126
:10993000422001F0BAF85E225321422001F0B5F82E
:1099400080225421422001F0B0F803220921422054
:1099500001F0ABF811226E21422001F0A6F89F22FF
:109960006F21422001F0A1F800225521422001F090
:109970009CF840225621422001F097F8802257217E
:10998000422001F092F85DE3012CFCD1022211216A
:10999000422001F08AF88A226B21422001F085F8EA
:1099A00004223A21422001F080F8042212214220B0
:1099B00001F07BF813221721422001F076F80122F2
:1099C0001821422001F071F8B6223221422001F024
:1099D0006CF802221921422001F067F87A221A213C
:1099E000422001F062F80F220321422001F05DF8CD
:1099F00000220C21422001F058F800223E21422092
:109A000001F053F83A227021422001F04EF835223D
:109A10007121422001F049F811227221422001F007
:109A200044F8F0227321422001F03FF83B22A221AA
:109A3000422001F03AF80F221E21422001F035F8B1
:109A400020227A21422001F030F803227B2142209B
:109A500001F02BF80A227C21422001F026F81A227C
:109A60007D21422001F021F83F227E21422001F099
:109A70001CF84E227F21422001F017F85B22802142
:109A8000422001F012F868228121422001F00DF8F5
:109A900075228221422001F008F87F228321422092
:109AA00001F003F889228421422000F0FEFF9A226F
:109AB0008521422000F0F9FFA6228621422000F0F5
:109AC000F4FFBD228721422000F0EFFFD32288213E
:109AD000422000F0EAFFE8228921422000F0E5FF61
:109AE000E0221321422000F0E0FF00221146422034
:109AF00000F0DBFF00221021422000F0D6FF5022B0
:109B00000D21422000F0D1FF40224221084600F002
:109B1000CCFF28221421422000F0C7FF0322A521F8
:109B2000422000F0C2FF0322AB21422000F0BDFF23
:109B300050222421422000F0B8FF43222521422058
:109B400000F0B3FFA3222621422000F0AEFF7822CE
:109B50009F21422000F0A9FF6822A021422000F0AE
:109B6000A4FF0322A121422000F09FFFD222A621C0
:109B7000422000F09AFFD222A721422000F095FF58
:109B8000F022A821422000F090FF8022A92142204B
:109B900000F08BFF1422AA21422000F086FFE5226C
:109BA0001321422000F081FF61220E21422000F0AB
:109BB0007CFF4B220F21422000F077FF022216216A
:109BC000422000F072FF02222121422000F06DFFAE
:109BD00091222221422000F068FF07222921422001
:109BE00000F063FF0B223321422000F05EFF0B22C6
:109BF0003521422000F059FF1D223721422000F07C
:109C000054FF71223821422000F04FFF2A223921CF
:109C1000422000F04AFF78223C21422000F045FF1C
:109C200040224D21422000F040FF20224E214220C0
:109C300000F03BFF00226921422000F036FF102295
:109C40007421422000F031FF4F228D21422000F08C
:109C50002CFF00228E21422000F027FF00228F21BE
:109C6000422000F022FF00229021422000F01DFF40
:109C700000229121422000F018FF0022962142206C
:109C800000F013FF80229A21422000F00EFF842270
:109C9000B021422000F009FF0C22B121422000F047
:109CA00004FF0E22B221422000F0FFFE8222B321E7
:109CB000422000F0FAFE0A22B821422000F0F5FE10
:109CC00002224321422000F0F0FEF22244214220F1
:109CD00000F0EBFE46224521422000F0E6FE632222
:109CE0004621422000F0E1FE32224721422000F0CE
:109CF000DCFE3B224821422000F0D7FE922259216F
:109D0000422000F0D2FE9B225A21422000F0CDFEDC
:109D1000A5225B21422000F0C8FE7A225C2142206D
:109D200000F0C3FE4A225D21422000F0BEFE0A225E
:109D30005E21422000F0B9FE0A226C21422000F090
:109D4000B4FE55226D21422000F0AFFE11226E219B
:109D5000422000F0AAFE9E226F21422000F0A5FEC4
:109D600040226A21422000F0A0FE40220121422030
:109D700000F09BFE40220221422000F096FEF722D6
:109D80001321422000F091FE9C224F21422000F03E
:109D90008CFE99225021422000F087FE02225121A0
:109DA000422000F082FE29225221422000F07DFE56
:109DB0008B225321422000F078FEB522542142200C
:109DC00000F073FE1E225821422000F06EFE082291
:109DD0006221422000F069FE10226321422000F03F
:109DE00064FE04226421422000F05FFE002265210F
:109DF000422000F05AFE05226621422000F055FE66
:109E000004229421422000F050FE06229521422097
:109E100000F04BFE08224121422000F046FE0022C5
:109E20003F21422000F041FE44227521422000F0F3
:109E30003CFEE1227621422000F037FE00224C2138
:109E4000422000F032FE01227721422000F02DFE58
:109E5000C0223D21422000F028FE09224B21422051
:109E600000F023FE6022C921422000F01EFE3822AD
:109E70004121422000F019FE40225621422000F0EC
:109E800014FE11223421422000F00FFE02223B2159
:109E9000422000F00AFE8822A421422000F005FEA4
:109EA00000229221422000F000FE00229621422052
:109EB00000F0FBFD30229721422000F0F6FD202229
:109EC0009821422000F0F1FD20229921422000F04B
:109ED000ECFD84229A21422000F0E7FD29229B21FB
:109EE000422000F0E2FD03229C21422000F0DDFD33
:109EF00099229D21422000F0D8FD7F229E21422000
:109F000000F0D3FD00227821422000F0CEFD012296
:109F10007921422000F0C9FDF022C821422000F042
:109F2000C4FD0F227921422000F0BFFD0022C8218C
:109F3000422000F0BAFD10227921422000F0B5FD48
:109F40007E22C821422000F0B0FD0A227921422061
:109F500000F0ABFD8022C821422000F0A6FD0B22BC
:109F60007921422000F0A1FD0122C821422000F009
:109F70009CFD0C227921422000F097FD0F22C82180
:109F8000422000F092FD0D227921422000F08DFD4B
:109F90002022C821422000F088FD09227921422098
:109FA00000F083FD8022C821422000F07EFD0222C5
:109FB0007921422000F079FDC022C821422000F022
:109FC00074FD03227921422000F06FFD4022C82158
:109FD000422000F06AFD05227921422000F065FD53
:109FE0003022C821422000F060FD26227921422043
:109FF00000F05BFD02223B21422000F056FD0222D0
:10A000004321422000F051FDF2224421422000F081
:10A010004CFD4F223021422000F047FD0022092153
:10A02000422000F042FD00221521422000F03DFDBB
:10A03000D0224021422000F038FD00228C21422015
:10A0400000F033FD10BD000010B5002220210248B1
:10A05000FDF7B0FC10BD00000014014010B5012256
:10A0600020210248FDF7A6FC10BD000000140140AD
:10A0700010B5002202210248FDF79CFC10BD000033
:10A080000018014010B5012202210248FDF792FCA0
:10A0900010BD00000018014010B500F00DF800F0F0
:10A0A00015F8FFF7EFFF10BD10B5FFF7E1FF00F067
:10A0B00003F800F00BF810BD10B50022082102488B
:10A0C000FDF778FC10BD00000014014010B501221E
:10A0D00008210248FDF76EFC10BD0000001401408D
:10A0E0002DE9F05F04460D4616461F46DDE90CAB30
:10A0F000DDE90A8900F034F8104800682060104853
:10A10000006828600F48006830600F4800683860B9
:10A110000E480068C8F800000D480068C9F8000043
:10A120000C480068CAF800000B480068CBF8000033
:10A130000A4801680E980160BDE8F09F7800002091
:10A140007C00002080000020840000208800002087
:10A150008C00002090000020940000209800002037
:10A160002DE9F04F97B00024002500260027A046D7
:10A17000A146A246A34600200D900C900B900A9099
:10A1800009900890079006900590049003903C2158
:10A19000C348F6F75FF80020C2490870C24908704A
:10A1A0003AE000F0BDF9552836D100F0B9F9512850
:10A1B00032D10024553404F15100C4B200F0B0F99A
:10A1C00005466019C4B200F0ABF90646A019C4B246
:10A1D00000F0A6F90746E019C4B200F0A1F98046E4
:10A1E00004EB0800C4B200F09BF9814604EB0900BF
:10A1F000C4B200F095F9824604EB0A00C4B200F044
:10A200008FF92044C4B200F08BF92044C4B200F0AE
:10A2100087F9A04200D100E0C3E700BF3DE000F0B5
:10A220007FF9552839D100F07BF9522835D1002427
:10A23000553404F15200C4B200F072F9834604EBC5
:10A240000B00C4B200F06CF90D900D982044C4B21C
:10A2500000F066F90C900C982044C4B200F060F94C
:10A260000B900B982044C4B200F05AF90A900A9857
:10A270002044C4B200F054F9099009982044C4B2B3
:10A2800000F04EF92044C4B200F04AF92044C4B2B0
:10A2900000F046F9A04200D100E0C0E700BF3DE079
:10A2A00000F03EF9552839D100F03AF9532835D15C
:10A2B0000024553404F15300C4B200F031F9089081
:10A2C00008982044C4B200F02BF907900798204466
:10A2D000C4B200F025F9069006982044C4B200F0FC
:10A2E0001FF9059005982044C4B200F019F90490B4
:10A2F00004982044C4B200F013F90390039820445A
:10A30000C4B200F00DF92044C4B200F009F92044B1
:10A31000C4B200F005F9A04200D100E0C0E700BFE0
:10A3200045EA062000B2169047EA082000B21590D0
:10A3300049EA0A2000B214900D984BEA002000B2BE
:10A340001390DDE90B1040EA012000B21290DDE924
:10A35000091040EA012000B21190DDE9071040EA3F
:10A36000012000B21090DDE9051040EA012000B2A2
:10A370000F90DDE9031040EA012000B20E9016981C
:10A38000F6F790F94FF08E410090F6F737F84FF05E
:10A3900083410190F6F700F844490290F5F7FCFF7D
:10A3A000434908601598F6F77DF94FF08E4100900B
:10A3B000F6F724F84FF083410190F5F7EDFF3B49A4
:10A3C0000290F5F7E9FF3B4908601498F6F76AF93F
:10A3D0004FF08E410090F6F711F84FF08341019055
:10A3E000F5F7DAFF31490290F5F7D6FF32490860F8
:10A3F0001398F6F757F94FF08E410190F5F7FEFFED
:10A400002E490290F5F7C8FF2D4908601298F6F71B
:10A4100049F94FF08E410190F5F7F0FF274902907E
:10A42000F5F7BAFF274908601198F6F73BF94FF0A6
:10A430008E410190F5F7E2FF20490290F5F7ACFF5D
:10A44000214908601098F6F72DF94FF08E410190E0
:10A45000F5F7D4FF1D490290F5F79EFF1C490860EF
:10A460000F98F6F71FF94FF08E410190F5F7C6FFF0
:10A4700016490290F5F790FF164908600E98F6F716
:10A4800011F94FF08E410190F5F7B8FF0F49029096
:10A49000F5F782FF1049086017B0BDE8F08F0000A3
:10A4A000340700206500002064000020CDCC1C4152
:10A4B000780000207C000020800000200000FA448A
:10A4C00084000020880000208C000020000034431D
:10A4D00090000020940000209800002000B585B076
:10A4E00014216846F5F7B6FE4FF416500090002090
:10A4F0000190029003900C200490084B00226946C2
:10A500000220FEF769F9002803DA4FF0FF3005B0AA
:10A5100000BD0220FEF7CEFC0020F8E761A5000890
:10A5200000BF0C4800780C4909788842F9D00948E6
:10A530000078401C07490870084600783C2190FBD1
:10A54000F1F201FB12000349087004480978405CED
:10A5500070470000640000206500002034070020E0
:10A5600009490A4A1278885408490978491C074A57
:10A570001170114609783C2291FBF2F302FB131192
:10A58000024A117070470000340700206500002067
:10A5900010B50446012C08D101220D490220FEF716
:10A5A00081FA002810DAA01E10BD0A48007808B908
:10A5B0000020F9E7032208490220FEF773FA002879
:10A5C00002DA4FF0FF30EFE7024804700020EBE7BB
:10A5D0006F000020760000206C00002070B504465B
:10A5E000002534B1012C06D0032C06D0042C08D150
:10A5F00005E0B02505E0982503E0182501E03025A9
:10A6000000BF00BF2A465521422000F04EFA70BD1F
:10A610002DE9F0410446802522265E2734B1012C25
:10A6200008D0032C0AD0042C10D10BE040251126B1
:10A630002F270BE066251B264B2707E099252826A8
:10A64000712703E0C02533268D2700BF00BF2A46AF
:10A650004F21422000F029FA2A465021422000F0E2
:10A6600024FA00225121422000F01FFA32465221E2
:10A67000422000F01AFA3A465321422000F015FA1F
:10A680002A465421422000F010FA9E2258214220EE
:10A6900000F00BFABDE8F08170B50446402534B1F6
:10A6A000012C06D0032C06D0042C08D105E030255F
:10A6B00005E0382503E0502501E0602500BF00BF1C
:10A6C0002A465621422000F0F0F970BD10B504462C
:10A6D0002046FEF713FF1420F7F7E2FA10BD10B57D
:10A6E000FEF7EAFD10BD10B5FEF7F0FDFFF7ACFC7C
:10A6F000FFF7DAFCFEF7E0FD00F0C0F8802212213F
:10A70000422000F0D2F93220F7F7CAFA0B2142209A
:10A7100000F003F90446732C02D06FF0010010BD65
:10A720000A21422000F0F9F80446762C02D06FF09E
:10A730000200F4E70020F2E738B50446002000905C
:10A740002080FEF7BBFE684600F046F8FEF7C0FE2C
:10A7500020889DF8001040EA01202080FEF7AEFE20
:10A76000684600F039F820889DF8001008432080E2
:10A77000FEF7AEFE38BD2DE9F0410446E725002680
:10A780000027012C06D0022C08D0032C0AD0042C60
:10A7900010D10BE0E5255A265C270BE0E52558266D
:10A7A000602707E0E52584264C2703E0E52596266B
:10A7B000402700BF00BF2A461321422000F075F950
:10A7C00032460121422000F070F93A46022142202F
:10A7D00000F06BF9BDE8F08170B504464FF480716C
:10A7E0001A48FDF739F8C5014FF400411848FDF744
:10A7F00033F845EA80154FF480411548FDF72CF8F1
:10A8000045EA40154FF400511148FDF725F845EA97
:10A8100000154FF480510E48FDF71EF845EAC005BB
:10A820004FF400610A48FDF717F845EA80054FF438
:10A8300080610748FDF710F845EA40054FF40071C4
:10A840000348FDF709F80543257070BD000C014071
:10A850000020014010B501210148FCF7FDFF10BDAB
:10A8600000180140232105E000E0491E0029FCD129
:10A87000401E23210028F7D17047000008B50020B2
:10A8800003230122102100900748FCF7F3FF012069
:10A8900003230022402100900348FCF7EBFF002037
:10A8A00000F08CF808BD00000014014010B54FF412
:10A8B0007A70FFF7D7FF00F06DF800F057F83220FC
:10A8C000FFF7D0FF00F05CF83220FFF7CBFF00F07D
:10A8D0006BF83220FFF7C6FF10BD70B5012000F005
:10A8E0006DF8082512E03220FFF7BCFF00F03EF8BB
:10A8F0006006040E00F07AF808B1601CC4B2322081
:10A90000FFF7B0FF00F03CF8681EC5B2002DEADC8E
:10A91000002000F053F8204670BD70B504460D4687
:10A92000002600F06DF8204600F08BF86420FFF759
:10A9300099FF284600F085F86420FFF793FF00F0A8
:10A940006FF86420FFF78EFF00F05AF844F0010022
:10A9500000F077F86420FFF785FFFFF7BEFF06469B
:10A96000FFF7A4FF00F05CF8304670BD10B501227F
:10A9700010210248FDF71EF810BD00000014014030
:10A9800010B5002210210248FDF714F810BD000098
:10A990000014014010B5012240210248FDF70AF8D9
:10A9A00010BD00000014014010B5002240210248F3
:10A9B000FDF700F810BD00000014014038B5044652
:10A9C00044B9002003230122402100900648FCF7EF
:10A9D00051FF07E00120032300224021009002489C
:10A9E000FCF748FF38BD00000014014010B54021BD
:10A9F0000248FCF731FFC0B210BD00000014014056
:10AA000010B5FFF7C7FFFFF7B1FF3220FFF72AFFAE
:10AA1000FFF7CAFF3220FFF725FFFFF7B1FF10BD98
:10AA200010B5FFF7C1FF3220FFF71CFFFFF79EFFB5
:10AA30003220FFF717FFFFF7ADFF3220FFF712FFBD
:10AA400010BD70B50446002615E004F0800010B17A
:10AA5000FFF7A0FF01E0FFF7A7FF6006040E32201A
:10AA6000FFF700FFFFF782FF3220FFF7FBFEFFF743
:10AA700087FF701CC6B2082EE7DB0120FFF79EFFA0
:10AA80003220FFF7EFFEFFF771FF3220FFF7EAFEFB
:10AA9000FFF7ACFF08B1012500E00025FFF770FFCC
:10AAA0000020FFF78BFF284670BD2DE9F0410646D8
:10AAB0000C4615460027FFF7A3FF3046FFF7C1FFFE
:10AAC00000B101276420FFF7CDFE2046FFF7B9FF54
:10AAD00000B101276420FFF7C5FE2846FFF7B1FF4C
:10AAE00000B10127FFF79CFF3846BDE8F0812DE952
:10AAF000F04104460425C0268027072C1DD2DFE83C
:10AB000004F01C04080C101418002425802680274B
:10AB100013E02425802680270FE024258026802727
:10AB20000BE024258026802707E024258026802727
:10AB300003E024258026802700BF00BF2A463A2153
:10AB40004220FFF7B2FF324667214220FFF7ADFFF8
:10AB50003A4668214220FFF7A8FFBDE8F08110B512
:10AB6000FEF7A0FB00BFFFF775FE0128FBD000BF7A
:10AB7000FFF770FE0028FBD0FFF78EFA00BFFFF74B
:10AB800069FE0128FBD000BFFFF764FE0028FBD060
:10AB9000FFF78AFAFEF7A6FCFEF79AFC10BD2DE936
:10ABA000F04705460E461746984605EB47004FF41A
:10ABB000447190FBF1F201FB12001FFA80F906EBE1
:10ABC00048001FFA80FA03214220FFF7A6FE044640
:10ABD00004F0F0040AF00301304661F39F000443DF
:10ABE000224603214220FFF760FFC6F387021921A6
:10ABF0004220FFF75AFFCAF387021A214220FFF7CB
:10AC000054FF32214220FFF788FE044604F0C004BE
:10AC100009F00701284661F3DF0004432246322190
:10AC20004220FFF742FFC5F3C70217214220FFF77A
:10AC30003CFFC9F3C70218214220FFF736FFBDE8E9
:10AC4000F08710B5012000F012FAFF2000F016FA8C
:10AC500010BD10B5402000F011FA002000F00EFAEF
:10AC6000002000F00BFA002000F008FA002000F0AD
:10AC700005FA952000F002FA10BD70B505460122D4
:10AC80000021092000F0B7F9044624B91021284614
:10AC900000F05CF90446FFF7D4FF0CB1012070BD51
:10ACA0000020FCE770B505464FF6FF7401E0601E1A
:10ACB00084B2FF2000F0E2F9A84201D0002CF6D1C6
:10ACC0000CB9FF2070BD0020FCE77FB56846FFF798
:10ACD000D4FF10B1002004B070BD9DF8000000F05A
:10ACE000C000402809D19DF809009DF8081000EB2C
:10ACF0000120401C84B2A50220E09DF8050000F070
:10AD00000F009DF80A1000EBD1109DF8091001F01A
:10AD1000030100EB4100861C9DF8080080119DF89E
:10AD2000071000EB81009DF8061001F0030100EB15
:10AD30008120441CA6F1090004FA00F52846CAE760
:10AD4000F8B50320FDF730FB012000F090F9022058
:10AD500000F09BF9002504E0FF2000F08FF9681C4B
:10AD600085B2642DF8DB1426FFF773FF00BF952230
:10AD70000021084600F03FF90446012C04D0301EA3
:10AD8000A6F101018EB2F2D1002052490870012CC7
:10AD90004AD187224FF4D571082000F02CF9012800
:10ADA00047D1002506E0FF2000F068F90DF8050006
:10ADB000681C85B2042DF6DB9DF80200012879D1CC
:10ADC0009DF80300AA2875D14FF6FE7600BF012238
:10ADD0000021372000F00FF901229107292000F00F
:10ADE0000AF9044624B1301EA6F101018EB2EED15B
:10ADF000002E5FD0012200213A2000F0FCF800284C
:10AE000058D1002506E0FF2000F038F90DF80500C4
:10AE1000681C85B2042DF6DB9DF8000000F04000B0
:10AE200018B106202B49087044E004202949087015
:10AE300040E001220021372000F0DDF8012200214E
:10AE4000292000F0D8F80446012C17DC0220214903
:10AE500008704FF6FE7600BF01220021372000F077
:10AE6000CAF801220021292000F0C5F80446BCB12F
:10AE7000301EA6F101018EB2EED111E0012015497C
:10AE800008704FF6FE7600BF01220021104600F048
:10AE9000B2F8044624B1301EA6F101018EB2F3D1FE
:10AEA0002EB101225102102000F0A5F810B10020AF
:10AEB00008490870FFF7C5FE002000F0E6F80548D5
:10AEC000007808B10020F8BD0CB12046FBE7AA20AD
:10AED000F9E70000600000202DE9F04106460F462A
:10AEE000154619480078062800D07F02012D0CD1A4
:10AEF00001223946112000F07EF80446FCB96902AF
:10AF0000304600F023F8044619E0012239461220A9
:10AF100000F071F8044600BF4FF40071304600F0B5
:10AF200015F8044606F50076681EC0B2051E01D06D
:10AF3000002CF1D0012200210C2000F05CF8FFF77A
:10AF400080FE2046BDE8F0816000002070B5044618
:10AF50000D46FE20FFF7A6FE08B1012070BD04E0FB
:10AF6000FF2000F08BF82070641C281EA5F1010161
:10AF70008DB2F5D1FF2000F081F8FF2000F07EF8BF
:10AF80000020EBE710B5002000F071F800F084F825
:10AF900008B9002010BDFFF754FE0120FAE72DE9A3
:10AFA000F04106460D4600F077F8074617B101203C
:10AFB000BDE8F081284600F061F8FD2D19D000248D
:10AFC00004E0305D00F05AF8601C84B2B4F5007FF4
:10AFD000F7DBFF2000F052F8FF2000F04FF8FF20D1
:10AFE00000F04CF8074607F01F00052801D00220AA
:10AFF000DEE70020DCE72DE9F04105460C46174668
:10B000004FF00008FFF71DFEFFF7BCFF10B1FF2057
:10B01000BDE8F08145F0400000F030F8200E00F06F
:10B020002DF8C4F3074000F029F8C4F3072000F01E
:10B0300025F8E0B200F022F8384600F01FF80C2D99
:10B0400002D1FF2000F01AF84FF01F0800BFFF20C8
:10B0500000F014F8064606F0800030B1B8F10000A8
:10B06000A8F1010101F0FF08F1D13046D0E710B599
:10B07000044621460320FDF781F910BD10B50446B2
:10B0800021460320FDF7D6F910BD10B50446214630
:10B090000320FDF7F5F910BD70B5002400BFFF20B7
:10B0A000FFF7ECFF0546FF2D01D1002070BD641CA9
:10B0B0006FF07F40B4FBF0F100FB114028B9032092
:10B0C000FDF772F90120FFF7D2FF6FF07040844264
:10B0D000E5D30120EAE700002DE9F04106460F46DE
:10B0E000154620480078062800D07F02012D0CD19B
:10B0F000012239461820FFF77EFF04466CBBFE2173
:10B100003046FFF74CFF044627E016480078012838
:10B1100009D0012200213720FFF76DFF01222946C7
:10B120001720FFF768FF012239461920FFF763FF58
:10B13000044694B900BFFC213046FFF730FF0446B7
:10B1400006F50076681EC0B2051E01D0002CF2D0B4
:10B15000FD210020FFF723FF0446FFF772FD204684
:10B16000BDE8F081600000202DE9F04104460D4665
:10B1700016461F464FF000080020134908700DE0E6
:10B180000A20F6F78DFDB8F57A7F03DB4FF0FF302C
:10B19000BDE8F08108F101001FFA80F80A48007844
:10B1A0000028EDD0094903C9F5F7E9FA20600848FD
:10B1B00000782870074903C9F5F7E1FA30600648BE
:10B1C000007838700020E3E7B2000020A8000020DB
:10B1D000B1000020A0000020B000002000B587B022
:10B1E000142102A8F5F736F84FF41650029000200B
:10B1F0000390049005900C2006900F4B002202A9AA
:10B200000320FDF7E9FA002803DA4FF0FF3007B01A
:10B2100000BD0320FDF74EFE0120032302468021DE
:10B2200000900648FCF726FB012000F00BF80020F8
:10B230000349088000BFEAE7C5B3000800200140C9
:10B24000B800002010B50446012C05D10122802150
:10B250000548FCF7AFFB04E0002280210248FCF720
:10B26000A9FB002010BD00000020014070B590B087
:10B270000446342103A8F4F7EDFF002002900025D6
:10B28000C4F3C000C4F3800104F00102C4F340031E
:10B29000CDE9001018A103A803F04EFA03A8F5F7B2
:10B2A00000F8C5B202AA2946501D02F0CAFB03A944
:10B2B00048199DF8082016A103F03EFA0025002049
:10B2C0001549087003A8F4F7ECFF0646314603A8B9
:10B2D00000F09AF90AE00A20F6F7E2FC642D03DB9D
:10B2E0004FF0FF3010B070BD681CC5B20A4800783E
:10B2F0000028F0D00020F5E72450474B433131358A
:10B300002C25642C25642C25642C25640000000069
:10B310002A253032780D0A00B600002070B58EB0B4
:10B320000446342101A8F4F795FF00200090002581
:10B33000012C06D0022C04D0032C02D0401E0EB0EB
:10B3400070BD224618A101A803F0F6F901A8F4F790
:10B35000A8FFC5B26A462946501D02F072FB01A93A
:10B3600048199DF8002014A103F0E6F900250020FB
:10B370001349087001A8F4F794FF0646314601A866
:10B3800000F042F909E00A20F6F78AFC642D02DB9E
:10B390004FF0FF30D3E7681CC5B209480078002899
:10B3A000F1D00020CBE700002450474B433033302E
:10B3B0002C25642C310000002A253032780D0A003B
:10B3C000B300002010B504460F48104909884454C2
:10B3D0000E480088401C0D4908800A2C09D1002025
:10B3E00009490A4A1288885400F012F800200749D7
:10B3F000088006480088642190FBF1F201FB1200EE
:10B400000249088010BD000070070020B80000202D
:10B4100070B50025002469A16A48F4F726FF0028CA
:10B420007FD02C216748F4F732FF054605B970BD7F
:10B430006D1C2C212846F4F72AFF044604B9F6E7D0
:10B44000641C2C212046F4F722FF054605B9EEE7DF
:10B45000002028702046F4F724FF10B120784128FE
:10B4600000D0E4E76D1C2C212846F4F710FF0446B9
:10B4700004B9DCE7002020702846F4F712FF00B979
:10B48000D5E7284603F022FE4F4A03C2641C2C2154
:10B490002046F4F7FCFE054605B9C8E700202870F1
:10B4A0002046F4F7FEFE00B9C1E720784E2803D10C
:10B4B00000204649087002E00120444908706D1CD4
:10B4C0002C212846F4F7E3FE044604B9AFE7002038
:10B4D00020702846F4F7E5FE00B9A8E7284603F0F7
:10B4E000F5FD3B4A03C2641C2C212046F4F7CFFE35
:10B4F000054605B99BE7002028702046F4F7D1FEE9
:10B5000008B994E70DE02078452803D1002031499F
:10B51000087002E001202F49087001202E490870B0
:10B5200049E02EA12748F4F7A0FE002843D02C21A3
:10B530002448F4F7ACFE054605B978E76D1C2C21CC
:10B540002846F4F7A4FE044604B970E700202070F2
:10B5500025A12846F4F789FE38B1641C20783328E9
:10B5600029D101202149087025E021A12846F4F7BE
:10B570007CFE38B1641C207833281CD101201D4981
:10B58000087018E01CA12846F4F76FFE38B1641C5F
:10B59000207833280FD10120184908700BE018A13A
:10B5A0002846F4F762FE30B1641C2078332802D1BB
:10B5B00001201449087000BF39E7000024474E52AB
:10B5C0004D43000070070020A8000020B1000020BB
:10B5D000A0000020B0000020B20000202450474B03
:10B5E000433030310000000030333000B300002021
:10B5F00031303100B400002031303500B50000207A
:10B6000031313500B600002070B504460D46AAB2AF
:10B6100021460320FDF746FA70BD000010B5012257
:10B6200011020248FCF7C6F910BD000000180140E5
:10B630000A4602B10022232105E000E0491E00294C
:10B64000FCD1401E23210028F7D1704710B588B0E7
:10B650000220FCF7CBFA19201B4988731B480864A9
:10B660001B484864012008731A4888641A484860D7
:10B67000084603F010FE04461CBB02208DF81B0098
:10B6800008208DF81C0003208DF818008DF81A0092
:10B690008DF8190000208DF80400ADF80800ADF811
:10B6A0000600094A01A9012003F0AEFE044644B990
:10B6B000054906A803F010FE044614B9204608B058
:10B6C00010BD4FF0FF30FAE77013002059B70008A3
:10B6D0007DB7000831B60008A501002010B5002094
:10B6E000174908701749012003F0E4FE044614B11D
:10B6F0004FF0FF3010BD134B114A1349012003F0E6
:10B70000FAFC044614B14FF0FF30F3E70D49002076
:10B7100003F0D0FE044614B14FF0FF30EAE70A49C7
:10B7200088680A4902F09BF907490869084902F04C
:10B7300096F90549C868074902F091F90020D9E750
:10B74000A40100207013002058130020A80100203D
:10B75000AC010020B0010020FEB504460D4616469F
:10B760001F46B0B20121CDE9001502903A78234678
:10B7700002210846FCF79EFA40B2FEBDFEB5044623
:10B780000D4616461F46B0B20121CDE900150290C4
:10B790003A78234602210846FCF704FB40B2FEBD7E
:10B7A00030B5ADF5117D0020049000F0E1F80028DF
:10B7B00004DA4FF0FF300DF5117D30BD0020FEF7AB
:10B7C00085FF0020FEF7D7FF43480078FEF720FFF3
:10B7D00042480078FEF702FF41480078FEF75CFF20
:10B7E0000020FFF784F9F0234FF4A0720A21AE2065
:10B7F000FFF7D5F93B48FCF7FBFB3A48007900908E
:10B800003848C378C28838A13D4802F095FF3C48CB
:10B8100005F03EFB05463348807832494978314A85
:10B820001278304B1B79CDE90032CDE902102D485A
:10B83000C378C28833A13D4802F07EFF0B223B490A
:10B8400006A805F093FF054615B14FF0FF30B2E7AB
:10B8500006AAF0214FF4A07002F013F9FFF77FF968
:10B8600000242BE005A8FEF767FFBDF8140000F0E8
:10B870001F008DF81000BDF81400C0F345108DF8BE
:10B880001100BDF81400C00A8DF812009DF81200D6
:10B89000C006000E8DF812009DF811008006000E03
:10B8A0008DF811009DF81000C006000E8DF81000F4
:10B8B00006AA032104A802F0D6F8641CB4F5963F4A
:10B8C000D0D3FEF70CFF06A805F051F9FDF778FD7F
:10B8D00000F044F800206EE7DA000020D8000020D5
:10B8E000D9000020F20000202F43616D6572612FA6
:10B8F000253034642D253032642D2530326400002B
:10B90000DF0C00202F43616D6572612F2530346498
:10B910002D253032642D253032642F2530326425B8
:10B92000303264253032642E626D70004C0A002083
:10B93000014608480088884208D106480088401C13
:10B94000044A10800020044A107070474FF0FF3006
:10B95000FBE70000DC000020F000002010B5002212
:10B9600020210248FCF726F810BD0000002001400D
:10B9700038B54FF0FF34022003230122202100902C
:10B980000B48FBF777FF0446002C02DA4FF0FF303C
:10B9900038BD00F001F90220F6F782F9FEF7A3FEA8
:10B9A0000446002C02DA4FF0FF30F1E70020EFE709
:10B9B000002001400348007808B9002070474FF08C
:10B9C000FF30FBE7F000002010B50C4800680C4980
:10B9D000096888420FD90B48006860B10120074907
:10B9E000086000200649086006490860064805F01E
:10B9F000BEF8002010BD4FF0FF30FBE7EC00002048
:10BA0000E8000020E0000020E00D0020F8B5002054
:10BA100000900024002656480068002876D10122B4
:10BA20005449554805F0A2FE05460DB1601EF8BD0B
:10BA30005148C0684E4908605048C08842F21071B1
:10BA400048434E49C97801EBC10202EB011100EBFA
:10BA500081004A4909790844494908604448006816
:10BA6000012101EB50204749086001204649087038
:10BA700043480068000E487041480068000C887018
:10BA80003F480088000AC8703D48007808710024CB
:10BA900007E0384904F11300095C601D3A4A11546B
:10BAA000641C34481330F4F7FCFBA042F1D804E0E6
:10BAB0000021601D344A1154641C1E2CF8DB2C48F4
:10BAC0000068000E304981F8230029480068000C06
:10BAD00081F8240026480088000A81F825002448BF
:10BAE000007881F8260027480068000E81F82700BA
:10BAF00024480068000C81F8280022480088000AC9
:10BB000081F829001F48007881F82A001F48006842
:10BB1000000E1D4981F82B001C480068000C81F8BC
:10BB20002C001A480088000A81F82D001748007878
:10BB300081F82E006B464FF400722F310E4805F04D
:10BB400037FF009B2F33104A1149042002F0D0FC2C
:10BB5000064616B94FF0FF3069E70C480068401CF4
:10BB60000A49086001200B49087000205FE70000C7
:10BB7000E00000204C0A0020E00D0020F200002030
:10BB8000E4000020E8000020B00A0020EC000020C3
:10BB9000DC000020F000002010B501222021024826
:10BBA000FBF708FF10BD00000020014010B5002287
:10BBB00002210248FBF7FEFE10BD000000200140FC
:10BBC00038B54FF0FF344FF4165025490860002077
:10BBD00048608860C8600C200861224B0022052064
:10BBE000FCF7FAFD0446002C02DA4FF0FF3038BDB6
:10BBF0000520FDF75FF90220032301220146009092
:10BC00001948FBF737FE00F0E5F84FF4FA60F6F755
:10BC100047F801201549088048804FF07E50886120
:10BC200000211248C1610020104981F8200010480D
:10BC30004862104888621048C86210480863084685
:10BC4000FAF7F4FF0446002C02DA4FF0FF30CEE79B
:10BC5000FFF7ACFF01200A494870087060B2C6E7E0
:10BC60000C100020ADBD0008002001404C10002049
:10BC700059BD0008E9BD0008A11C00080BDA000846
:10BC8000401000202DE9FC5F4FF0000BDA46002148
:10BC90000C460D460E460F462C48FAF727FF25E0C6
:10BCA0004FF4FA60F5F7FCFF29492848FAF7A0FE9F
:10BCB000002800DA18E026494868F4F74DFD804670
:10BCC00022462B46F4F7D8FB04460D4620498868E7
:10BCD000F4F742FD804632463B46F4F7CDFB06467C
:10BCE0000F460AF1010A00BF0BF1010BBBF10A0F6D
:10BCF000D6DBBAF1000F03D14FF0FF30BDE8FC9F57
:10BD00005046F4F7EBFC804642460B462046294657
:10BD1000F4F759FCCDE90001F4F731FD0C49486016
:10BD20005046F4F7DBFC804642460B463046394627
:10BD3000F4F749FCCDE90001F4F721FD04498860DE
:10BD40008868044901F08BFE0020D7E74C100020E2
:10BD5000401000200001002070B506460D4600246A
:10BD6000202D01D9601E70BD06E00120F5F798FF77
:10BD7000641C642C00DB03E00A480068A842F4D38A
:10BD800000BF642C08DA002403E00748005D30554A
:10BD9000641CAC42F9D302E04FF0FF30E3E700202F
:10BDA000E1E70000FC000020201000200749084ABD
:10BDB0001268885406490968491C054A11601146F1
:10BDC000097801F01F011160704700002010002069
:10BDD000FC00002010B5012202210248FBF7EAFD19
:10BDE00010BD00000020014070B504460D46002043
:10BDF00003490860AAB221460520FCF753FE70BD36
:10BE0000FC00002010B5012005490860002005490C
:10BE1000086005490860054804F0A9FE10BD00004F
:10BE2000EC000020E8000020E0000020E00D0020F1
:10BE30002DE9F04F89B00025002600200790B8E2D8
:10BE4000002405E0FE48005D022800D102E0641CE9
:10BE5000032CF7DB00BF032C00DBABE201254DE038
:10BE600040F20D206043F74901EB8000405D7F28E0
:10BE700003D1E0B202F00CFB46E040F20D2060433B
:10BE8000F04901EB8000405D7E2827D16D1C40F217
:10BE90000D20604301EB8000405D012808D17E2128
:10BEA00040F20D206043E74A02EB8000815523E019
:10BEB00040F20D206043E34901EB8000405D022821
:10BEC00008D17F2140F20D206043DE4A02EB800062
:10BED000815511E0E0B202F0DBFA15E040F20D20EE
:10BEE0006043D84901EB8000415D40F20D20604382
:10BEF000D44A02EB80008155761C6D1CD24830F884
:10BF00001400401EA842ABDC00BFCF4830F814003C
:10BF1000401EA84200DD4CE240F20D206043C949BA
:10BF200001EB80008078010640F20D206043C54A95
:10BF300002EB8000C07841EA004140F20D206043EE
:10BF400002EB8000007941EA002040F20D216143BC
:10BF500002EB810149790843059040F20D206043CE
:10BF6000114601EB80008079010640F20D2060430C
:10BF700002EB8000C07941EA004140F20D206043AD
:10BF800002EB8000007A41EA002040F20D2161437B
:10BF900002EB8101497A0843069040F20D2060438C
:10BFA000114601EB8000417840F20D20604312F809
:10BFB000200041EA002A40F20D206043114601EBC7
:10BFC0008000C17B40F20D20604302EB8000807B4B
:10BFD00041EA0020049040F20D206043114601EB3D
:10BFE0008000C17A40F20D20604302EB8000807A2D
:10BFF00000F0030041EA0029944905980968884245
:10C0000004D1934906980968884203D0E0B202F04F
:10C010003FFACEE10020079040F20D2060438949AD
:10C0200001EB8000807A00F00C000C2819D1711E01
:10C0300040F20D226243834B03EB820007AA01F01A
:10C04000C4FC40F20D2060437E4901EB8001701E6C
:10C05000085C9DF81C10884207D0E0B202F018FA84
:10C06000A7E1E0B202F014FAA3E140F20D20604330
:10C07000744901EB8000807A00F0200020280ED166
:10C08000A6F11300484508D002225146049802F058
:10C090000BFAE0B202F0FCF98BE112250DE0A6F1FB
:10C0A0001100484508D002225146049802F0FCF9DC
:10C0B000E0B202F0EDF97CE11025BAF5004F52D163
:10C0C000B9F1050F03D0E0B202F0E2F971E140F2FC
:10C0D0000D2060435B4901EB8001681C095C40F264
:10C0E0000D206043574A02EB8000405D41EA002B7F
:10C0F00040F20D206043114601EB8001E81C095C11
:10C1000040F20D20604302EB8002A81C105C41EA63
:10C11000002740F20D2060434A4901EB8001281DB1
:10C1200011F8008040F20910874206D1B8F1000FE3
:10C1300015D1584600F0A2FD11E0B7F5847F06D175
:10C14000B8F1000F0BD1584600F098FA07E0042F21
:10C1500005D1B8F1000F02D15846FFF7E9FBE0B274
:10C1600002F096F924E148F20100824538D1002717
:10C17000B9F1020F08D002225146049802F094F956
:10C18000E0B202F085F914E140F20D2060432D4940
:10C1900001EB8001681C095C40F20D206043294AD4
:10C1A00002EB8000405D41EA00283C2098FBF0F063
:10C1B0001FFA80F808F0FF0000F068FF0746002F24
:10C1C00005DA01225146049802F06EF904E00022DB
:10C1D0005146049802F068F9E0B202F059F9E7E03C
:10C1E00048F2020082457DD1B9F1080F07D0022242
:10C1F0005146049802F058F9E0B202F049F940F2D1
:10C200000D2060430F4901EB8000405D01060022D4
:10C2100040F20D2060430B4B03EB8003681C185C5D
:10C22000124341EA004040F20D216143054B03EB0C
:10C230008103A91C595C40EA012140F20D2009E06C
:10C24000E4010020F41B0020E8010020CC010020C4
:10C25000D001002060435A4B03EB8003E81C185CBC
:10C26000014340F20D206043554B03EB8003281D32
:10C27000185C00231B0643EA102342EA00621943BC
:10C2800040F20D2060434E4B03EB8003681D1B5CA6
:10C290000020000440EA134C42EA034041EA0C014A
:10C2A00040F20D226243464B03EB8203AA1D9B5CC6
:10C2B0000022120242EA136C40EA032241EA0C0017
:10C2C00040F20D2161433E4B03EB8103E91D595CB4
:10C2D00042EA010780463B4A022338464146F3F7CB
:10C2E00043FF00E05CE080B2ADF80E00364A002368
:10C2F00038464146F3F738FF64220023CDE90001B8
:10C30000F3F732FFD0B28DF80B00304A00233846E5
:10C310004146F3F729FF64220023CDE90001F3F73A
:10C3200023FFD0B28DF80C0042F210720023384681
:10C330004146F3F719FF64220023CDE90001F3F72A
:10C3400013FFD0B28DF8080064220023384641461E
:10C35000F3F70AFF64220023CDE90001F3F704FF9D
:10C36000D0B28DF809006422002338464146F3F725
:10C37000FBFED0B28DF80A0002A8FBF789FE002868
:10C3800005DA02225146049802F08EF804E00022F9
:10C390005146049802F088F8E0B202F079F807E01C
:10C3A00002225146049802F07FF8E0B202F070F8E1
:10C3B00000BF45E500BF002009B0BDE8F08F0000D8
:10C3C000F41B002000E40B5400E1F50540420F008F
:10C3D00010B588B04FF0FF3400200590069007900C
:10C3E0001D4804901D48039005A802900920019063
:10C3F0004FF4E1301A490860002048608860C86046
:10C400000C200861174B00220120FCF7E5F90446D7
:10C41000022003230122C10100901348FBF72AFAEE
:10C420000120FCF747FD012001AB02AA03A90090FF
:10C4300004A801F0B9FF0446012C01D1019818B9F4
:10C440004FF0FF3008B010BD05A8F3F740FF80B2F1
:10C45000064908602046F5E7D4010020DB010020F2
:10C460009034002071C4000800180140D001002061
:10C4700010B501467F2955D1002031E03F4A125CBA
:10C48000012A2CD13E4A32F81020122A06DA002264
:10C490003A4B1A543A4B23F8102023E040F20D2275
:10C4A0004243384B03EB8202354B33F81030D15402
:10C4B000334A32F81020521C314B23F810201A4610
:10C4C00032F8102040F6340392FBF3F403FB1422FD
:10C4D0002B4B23F810200222284B1A5410BD401C6D
:10C4E0000328CBDB00BF002018E0244A125CA2B96D
:10C4F00040F20D224243234B03EB8202204B33F8E0
:10C500001030D1541E4A32F81020521C1C4B23F814
:10C5100010200122194B1A5402E0401C0328E4DBCE
:10C5200000BF28E0002022E0144A125C012A1DD13D
:10C5300040F20D224243134B03EB8202104B33F8BF
:10C540001030D1540E4A32F81020521C0C4B23F8F4
:10C5500010201A4632F8102040F6340392FBF3F410
:10C5600003FB1422064B23F8102002E0401C032892
:10C57000DADB00BF00BF00BFB0E70000E40100202D
:10C58000E8010020F41B002010B500224FF40071D8
:10C590000148FBF70FFA10BD0018014038B54FF005
:10C5A000FF34022003230122010200900748FBF719
:10C5B00061F9044600224FF400710448FBF7FAF9D0
:10C5C000FAF7C8FF0446204638BD000000180140B5
:10C5D00010B51D490520FAF775FE002802DA4FF064
:10C5E000FF3010BD19490620FAF76CFE002802DA68
:10C5F0004FF0FF30F5E716490720FAF763FE0028F1
:10C6000002DA4FF0FF30ECE712490820FAF75AFE41
:10C61000002802DA4FF0FF30E3E70F490A480068CC
:10C6200001F01DFA0D490948006801F018FA0C499B
:10C630000748006801F013FA0A490648006801F04B
:10C640000EFA0020CDE70000340100203801002060
:10C650003C0100204001002024010020280100208E
:10C660002C0100203001002010B5012251020248A7
:10C67000FBF7A0F910BD0000001801400146084872
:10C680000088884208D106480088401C044A10806F
:10C690000020044A107070474FF0FF30FBE70000A5
:10C6A0008E0100208C01002004480088401C0349B2
:10C6B0000880002002490870704700008E010020A9
:10C6C0008C01002010B5FFF769FF044600F05AFC0A
:10C6D000044601F0A5F8044600F076FF0446FFF793
:10C6E0006FFA0446204610BD0348007810B14FF0A1
:10C6F000FF3070470020FCE78C0100202DE9F04F4F
:10C70000ADF54D7D002040903EA8FBF771FCFFF792
:10C71000ABFF00F02BFF01F0FDF801F05DF8FFF733
:10C7200059FB00F043FC4FF4FA60F5F7B9FA00F05A
:10C73000ABFFFFF7A7FA47F23050F5F7B1FA01F077
:10C74000AFF8FFF745FF00F035FFFFF72FFA01F0D4
:10C750005BF8FFF719FF9DF8FC0000909DF8FB3097
:10C76000BDF8FE2074A1784801F0E6FF764804F099
:10C770008FFBCC909DF8FC0000909DF8FB30BDF83D
:10C78000FE2072A1704801F0D7FF32226E4941A805
:10C7900004F0ECFFCC90469868B974496A4801F0FF
:10C7A000CBFF6948F3F77DFD044640AB224666495E
:10C7B00041A805F02FFB6E480068F3F7CDFF044653
:10C7C0000D466C480068F3F7C7FF06460F466A48F7
:10C7D0000068F3F7C1FF8046894668480068F3F7B0
:10C7E000BBFF82468B4666480068F3F7B5FFCDE98C
:10C7F0003C0164480068F3F7AFFFCDE93A016248B5
:10C800000068F3F7A9FFCDE9380160480068F3F745
:10C81000A3FFCDE936015E480068F3F79DFFCDE93F
:10C8200034015C480068F3F797FFCDE932015A48BC
:10C830000068F3F791FFCDE9300158498868F3F7B4
:10C840008BFFCDE92E0156498868F3F785FFCDE9C6
:10C850002C0154480068F3F77FFFCDE92A015248C4
:10C860000068F3F779FFCDE9280150480068F3F735
:10C8700073FFCDE926014E480068F3F76DFFCDE95F
:10C880001CABCDE91E89CDE92067CDE92245CDE974
:10C890002401DDE93C01CDE91A01DDE93A01CDE9E8
:10C8A0001801DDE93801CDE91601DDE93601CDE9F0
:10C8B0001401DDE93401CDE91201DDE93201CDE9F0
:10C8C0001001DDE93001CDE90E01DDE92E01CDE9F0
:10C8D0000C01DDE92C01CDE90A01DDE92A01CDE9F0
:10C8E0000801DDE92801CDE90601DDE92601CDE9F0
:10C8F0000401DDE92401CDE9020101219DF8FA00DE
:10C90000CDE900019DF8F9309DF8F82029490E483D
:10C9100001F012FF0C48F3F7C4FC044640AB22467A
:10C92000094941A805F076FA41A804F020F9002051
:10C930000DF54D7DBDE8F08F2F4C6F672F25642DD1
:10C9400025642D2564000000351100202F4C6F67F1
:10C950002F25642D25642D25642F4465764D6F6E3B
:10C9600069746F72696E672E63737600B03D01085B
:10C970001C010020140100208801002084010020F7
:10C98000800100207C01002078010020740100203B
:10C99000700100206C010020680100204010002080
:10C9A000A0100020400100203C01002034010020A4
:10C9B000380100204C3D010810B501209B4908704A
:10C9C0009B480068000E487099480068000C887009
:10C9D00097480088000AC870954800780871954803
:10C9E0000068000E487193480068000C88719148F7
:10C9F0000088000AC8718F48007808728E48006865
:10CA0000000E48728C480068000C88728A480088C2
:10CA1000000AC87288480078087388480068000EC9
:10CA2000487386480068000C887384480088000AB0
:10CA3000C87382480078087481480068000E487402
:10CA40007F480068000C88747D480088000AC8741C
:10CA50007B48007808757B480068000E4875794867
:10CA60000068000C887577480088000AC87575480A
:10CA70000078087674480068000E487672480068AE
:10CA8000000C887670480088000AC8766E480078E6
:10CA900008776E480068000E48776C480068000C04
:10CAA00088776A480088000AC8776848007881F863
:10CAB000200067480068000E81F821006448006883
:10CAC000000C81F8220062480088000A81F82300E7
:10CAD0005F48007881F824005E480068000E81F805
:10CAE00025005C480068000C81F826005948008841
:10CAF000000A81F827005748007881F82800564836
:10CB00000068000E81F8290053480068000C81F885
:10CB10002A0051480088000A81F82B004E4800780E
:10CB200081F82C004D480068000E81F82D004B481C
:10CB30000068000C81F82E0048480088000A81F83F
:10CB40002F004648007881F8300045480068000E04
:10CB500081F8310042480068000C81F832004048FA
:10CB60000088000A81F833003D48007881F83400DD
:10CB70003C480068000E81F835003A480068000C17
:10CB800081F8360037480088000A81F837003548B8
:10CB9000007881F8380034480068000E81F83900C8
:10CBA00031480068000C81F83A002F480088000ADC
:10CBB00081F83B002C48007881F83C002B48006845
:10CBC000000E81F83D0029480068000C81F83E0005
:10CBD00026480088000A81F83F002448007881F840
:10CBE000400023480068000E81F84100204800689A
:10CBF000000C81F842001E480088000A81F84300BA
:10CC00001B48007881F8440045230A4619494FF42F
:10CC1000847001F06DFC044614B94FF0FF3010BD74
:10CC20000120154908700020F9E70000F0100020ED
:10CC300028010020240100202C01002030010020C8
:10CC400008010020000100204401002048010020CC
:10CC50004C01002050010020540100205801002008
:10CC60005C01002060010020640100200C01002014
:10CC7000100100208E0100208C0100200146084890
:10CC80000088884208D106480088401C044A108069
:10CC90000020044A107070474FF0FF30FBE700009F
:10CCA000920100209001002004480088401C0349A4
:10CCB000088000200249087070470000920100209F
:10CCC0009001002010B5FEF7C1FCFAF743FC0020EC
:10CCD00010BD00000348007810B14FF0FF307047DE
:10CCE0000020FCE7900100202DE9F04FADF51D7DFF
:10CCF000002010900EA8FBF77BF9FEF7EFFC00F088
:10CD000019FE9DF83C0000909DF83B30BDF83E2098
:10CD100038A13C4801F010FD3A4804F0B9F89C9065
:10CD20009DF83C0000909DF83B30BDF83E2036A1B8
:10CD3000344801F001FD3222324911A804F016FDF9
:10CD40009C90169868B937A12E4801F0F5FC2D4843
:10CD5000F3F7A7FA044610AB22462A4911A805F0BA
:10CD600059F83D480068F3F7F7FC04460D463B4888
:10CD70000068F3F7F1FC06460F463949C868F3F737
:10CD8000EBFC8046894636490869F3F7E5FC8246A4
:10CD90008B4633498868F3F7DFFCCDE904ABCDE976
:10CDA0000689CDE90867CDE90A45CDE90C01DDE941
:10CDB0000C01CDE9020101219DF83A00CDE9000105
:10CDC0009DF839309DF8382026A10E4801F0B4FCBA
:10CDD0000C48F3F766FA044610AB2246094911A83D
:10CDE00005F018F811A803F0C2FE00200DF51D7D16
:10CDF000BDE8F08F2F4C6F672F25642D25642D25FE
:10CE000064000000551200202F4C6F672F25642D01
:10CE100025642D25642F4465765374617475732ED3
:10CE20006373760054696D652C4E756D6265722C66
:10CE300074656D70657261747572652C68756D6965
:10CE4000646974792C70726573737572652C4563AF
:10CE50002C52450D0A0000009C010020A00100207A
:10CE60005813002025643A25643A25642C25642C47
:10CE7000252E32662C252E32662C252E32662C2548
:10CE80002E32662C252E32660D0A000010B54FF0AA
:10CE9000FF3401203349087033480068000E4870A1
:10CEA00031480068000C88702F480088000AC8705C
:10CEB0002D48007808712D480068000E48712B48F5
:10CEC0000068000C887129480088000AC87127484A
:10CED0000078087226480068000E487224480068EE
:10CEE000000C887222480088000AC8722048007826
:10CEF000087320480068000E48731E480068000C44
:10CF000088731C480088000AC8731A48007808749F
:10CF100019480068000E487417480068000C8874AF
:10CF200015480088000AC874134800780875002066
:10CF300048758875C875087648768876C876087703
:10CF40001D230A460D4940F2091001F0D1FA0446AA
:10CF500014B94FF0FF3010BD0120094908700020BE
:10CF6000F9E7000038120020A8010020AC010020E1
:10CF7000B0010020940100209801002092010020BF
:10CF80009001002010B5FDF7A9FA04460120FDF735
:10CF9000FFFA4FF4FA70F4F783FE0020FDF7F8FA79
:10CFA0004FF4FA70F4F77CFE204610BD00B585B052
:10CFB0000120FDF7EDFA0220F4F772FE2148224924
:10CFC000224A234BCDE90132CDE903102148224BFF
:10CFD000224A234900902348FDF782F80020FDF7FC
:10CFE000D7FA21491F48006800F039FD1F491C4845
:10CFF000006800F034FD1E491848006800F02FFD5D
:10D000001C491548006800F02AFD1B4911480068BA
:10D0100000F025FD19490E48006800F020FD184970
:10D020000A48006800F01BFD16490748006800F038
:10D0300016FD15490348006800F011FD002005B0F9
:10D0400000BD000088010020840100208001002034
:10D050007C01002078010020740100207001002074
:10D060006C010020680100204401002048010020DC
:10D070004C010020500100205401002058010020E4
:10D080005C010020600100206401002070B592B0B6
:10D090000446342105A8F3F7DDF8114E1148049039
:10D0A00005A80390224610A101F046FB05A8F3F75E
:10D0B000F8F80290012002A903AB04AACDE9001000
:10D0C0003146022001F0ACF90546002D03DA4FF09D
:10D0D000FF3012B070BD054804700020F9E7000071
:10D0E000B4010020BA01002025640000C401002022
:10D0F00010B588B04FF0FF340020059006900790DF
:10D10000F8480490F848039005A80290092001907F
:10D1100002200346112204210090F448FAF7AAFBEA
:10D1200002200346112208210090F048FAF7A2FBE2
:10D1300002200346112210210090EC48FAF79AFBD6
:10D1400002200346112220210090E848FAF792FBC2
:10D1500002200346112240210090E448FAF78AFB9E
:10D1600002200346112201030090E148FAF782FBF6
:10D1700002200346112201210090DE48FAF77AFBD3
:10D1800002200346112201460090DA48FAF772FBAA
:10D1900002200346112204210090D648FAF76AFBC8
:10D1A00002200346112208210090D248FAF762FBC0
:10D1B00002200346112210210090CE48FAF75AFBB4
:10D1C00002200346112220210090CA48FAF752FBA0
:10D1D00002200346112240210090C648FAF74AFB7C
:10D1E00002200346112280210090C248FAF742FB38
:10D1F000022003461122C1010090BE48FAF73AFB13
:10D2000002200346112201020090BA48FAF732FBCD
:10D2100002200346112241020090B648FAF72AFB89
:10D2200002200346112201460090B148FAF722FB82
:10D2300002200346112204210090AD48FAF71AFBA0
:10D2400002200346112208210090A948FAF712FB98
:10D2500002200346112201210090A748FAF70AFB99
:10D2600002200346112210210090A148FAF702FB88
:10D27000022003461122202100909D48FAF7FAFA75
:10D28000022003461122042100909C48FAF7F2FA8A
:10D29000022003461122810200909648FAF7EAFA2A
:10D2A000022003461122C10200909248FAF7E2FAE6
:10D2B000022003461122010300908E48FAF7DAFAA1
:10D2C000022003461122410300908A48FAF7D2FA5D
:10D2D000022003461122810300908648FAF7CAFA19
:10D2E000022003461122802100908048FAF7C2FAFA
:10D2F000022003461122410200907C48FAF7BAFA54
:10D30000022003461122810200907848FAF7B2FA0F
:10D31000022003461122C10200907448FAF7AAFACB
:10D32000022003461122010300907048FAF7A2FA86
:10D33000022003461122410300906C48FAF79AFA42
:10D34000022003461122810300906848FAF792FAFE
:10D35000022003461122C10200906848FAF78AFAB7
:10D36000022003461122010300906448FAF782FA72
:10D37000022003461122410300906048FAF77AFA2E
:10D38000022003461122810300905C48FAF772FAEA
:10D39000022003461122410200905948FAF76AFA26
:10D3A000022003461122810200905548FAF762FAE2
:10D3B000022003461122C10200905148FAF75AFA9E
:10D3C000022003461122010300904D48FAF752FA59
:10D3D000022003461122410300904948FAF74AFA15
:10D3E000022003461122810300904548FAF742FAD1
:10D3F000022003461122012100904248FAF73AFA2E
:10D40000022003461122042100903E48FAF732FA26
:10D41000022003461122082100903A48FAF72AFA1E
:10D42000022003461122102100903648FAF722FA12
:10D43000022003461122402100903248FAF71AFADE
:10D44000022003461122402100902948FAF712FADF
:10D45000022003461122802100902548FAF70AFA9B
:10D46000022003461122C10100902148FAF702FA76
:10D47000022003461122C10100901F48FAF7FAF971
:10D48000022003461122810200901B48FAF7F2F9AC
:10D49000022003461122C10200901748FAF7EAF968
:10D4A000022003461122012100901548FAF7E2F903
:10D4B000022003461122014600901148FAF7DAF9DA
:10D4C000012001AB02AA03A9009004A800F06CFFA0
:10D4D0000446012C01D10198B0B94FF0FF3008B0DB
:10D4E00010BD0000B4010020BA0100200018014066
:10D4F00000100140001C014000080140000C0140E8
:10D50000001401400020014005A8F2F7E0FE0249A6
:10D5100008700020E3E70000C401002010B5FAF70E
:10D5200085F8FAF7B7FCFAF7F9FFFBF74BFBFAF7C8
:10D5300053FA01210C480078FAF7ECFDF7F7E3FA0B
:10D5400001210846F5F752FFF6F72AFFFBF7D6F858
:10D55000FAF7A6FAFBF7ECFCFBF754F8FAF716FD1E
:10D56000FAF77EF810BD0000C401002010B5FAF7EC
:10D570005DF8FAF78FFCFAF7D1FFFBF723FBFAF718
:10D580002BFA0021FF20FAF7C5FDF7F7BCFA0121BD
:10D590000846F5F72BFFF6F703FFFBF7AFF8FAF7AE
:10D5A0007FFAFBF7C5FCFBF72DF8FAF7EFFCFAF76B
:10D5B00057F810BD10B5002202210248FAF7FAF917
:10D5C00010BD00000020014038B54FF0FF344FF48B
:10D5D000165024490860002048608860C8600C200C
:10D5E0000861214B00220420FBF7F6F80446002CCA
:10D5F00002DA4FF0FF3038BD0420FBF75BFC02205D
:10D6000003230122014600901848FAF733F900F08D
:10D61000E3F84FF4FA60F4F743FB0620144948801E
:10D6200008804FF07E50886100211148C161114887
:10D630000F49086210484862104888621048C86262
:10D640000846F9F75BFD0446002C02DA4FF0FF3084
:10D65000D1E7FFF7AFFF01200A494870087060B2B8
:10D66000C9E70000DC100020B1D70008002001400D
:10D67000AC1000205DD70008EDD70008A11C000801
:10D680000BDA0008A01000202DE9FC5F4FF0000B22
:10D69000DA4600210C460D460E460F462C48F9F797
:10D6A000E1FC25E04FF4FA60F4F7FAFA294928483A
:10D6B000F9F760FC002800DA18E026494868F3F71B
:10D6C0004BF8804622462B46F2F7D6FE04460D461E
:10D6D00020498868F3F740F8804632463B46F2F727
:10D6E000CBFE06460F460AF1010A00BF0BF1010B03
:10D6F000BBF10A0FD6DBBAF1000F03D14FF0FF30B8
:10D70000BDE8FC9F5046F2F7E9FF804642460B46D3
:10D7100020462946F2F757FFCDE90001F3F72FF82D
:10D720000C4948605046F2F7D9FF804642460B4606
:10D7300030463946F2F747FFCDE90001F3F71FF80D
:10D74000044988608868044900F089F90020D7E717
:10D75000AC100020A01000200801002070B5064683
:10D760000D460024202D01D9601E70BD06E0012069
:10D77000F4F796FA641C642C00DB03E00A480068A6
:10D78000A842F4D300BF642C08DA002403E0074861
:10D79000005D3055641CAC42F9D302E04FF0FF301D
:10D7A000E3E70020E1E700000401002080100020F2
:10D7B0000749084A1268885406490968491C054AFD
:10D7C00011601146097801F01F01116070470000D7
:10D7D000801000200401002010B50122022102481F
:10D7E000FAF7E8F810BD00000020014070B50446CB
:10D7F0000D46002003490860AAB221460420FBF729
:10D8000051F970BD0401002010B500222021034809
:10D81000FAF7D0F80020FDF715FD10BD00200140FB
:10D8200038B54FF0FF34022003230122202100905D
:10D830001A48FAF71FF80446002C02DA4FF0FF30BE
:10D8400038BD002220211548FAF7B4F8FDF7C6FCD0
:10D850000446002C02DA4FF0FF30F1E70120FDF71B
:10D86000F1FC012220210D48FAF7A4F80220F4F778
:10D8700017FA0520FDF7FAFC0446002C02DA4FF0F7
:10D88000FF30DDE70320FDF749FD4FF47A70F4F730
:10D8900007FAFFF7B9FF2046D2E700000020014059
:10D8A00010B54FF0FF34154B154A16491648FDF7D1
:10D8B0005BFC044614B14FF0FF3010BD11480078F6
:10D8C000012805D11048006880F000400E4908602A
:10D8D0000A480078012805D10948006880F0004016
:10D8E0000749086009490848006800F0B8F8084985
:10D8F0000348006800F0B3F80020DEE720010020B4
:10D900001C01002018010020140100200C0100203F
:10D910001001002010B50120FDF794FC0220F4F75F
:10D92000BFF9012220210248FAF744F810BD000097
:10D930000020014010B50F490420F9F7C3FC00286E
:10D9400002DA4FF0FF3010BD0B490120F9F7BAFCA5
:10D95000002802DA4FF0FF30F5E708490548006873
:10D9600000F07DF806490448006800F078F80020CF
:10D97000E9E700009C010020A001002094010020A4
:10D980009801002070B50024FAF76CFB05460023CF
:10D990001A460849022000F0ABFD044614B94FF0C6
:10D9A000FF3070BD03480088401C024908800020F9
:10D9B000F7E70000C801002010B5FAF713FB10B913
:10D9C0004FF0FF3010BD0020FCE730B5002317E01A
:10D9D00010F8014B15786C40147000230EE0147899
:10D9E00004F001042CB114788C2585EA64041470C9
:10D9F00002E01478641014705C1CE3B2082BEEDBB8
:10DA00000C1EA1F10101E3D130BDF0B503460C4677
:10DA10004FF6FF70002110E05F5C7840002508E0C1
:10DA200000F00106401016B14AF2010778406F1C61
:10DA3000BDB2082DF4DB4F1CB9B2A142ECD310806B
:10DA4000F0BD30B5034600241470002004E01478C3
:10DA50001D5C6C401470401C8842F8D330BD0246F7
:10DA60000A6000207047F8B504460D4616460020AF
:10DA700000906B462A462146304604F0CBF9002040
:10DA8000F8BD70B590B004460D46164600200190D2
:10DA900044F64250ADF8300004FB05F000EB4000C6
:10DAA0003630CDF832000020CDF836003620CDF8E3
:10DAB0003A0001AB02220CA9304604F0ABF901ABED
:10DAC00004220DF13201304604F0A4F901AB042226
:10DAD0000DF13601304604F09DF901AB04220DF141
:10DAE0003A01304604F096F92820029003940495F8
:10DAF0000120ADF814001820ADF8160000200690A3
:10DB000004FB05F000EB400007900020089009900E
:10DB10000A900B9001AB042202A9304604F07AF976
:10DB200001AB042203A9304604F074F901AB0422CE
:10DB300004A9304604F06EF901AB022205A9304673
:10DB400004F068F901AB02220DF11601304604F031
:10DB500061F901AB042206A9304604F05BF901AB80
:10DB6000042207A9304604F055F901AB042208A9A4
:10DB7000304604F04FF901AB042209A9304604F005
:10DB800049F901AB04220AA9304604F043F901AB7C
:10DB900004220BA9304604F03DF9002010B070BDFE
:10DBA0002DE9FF4FADF54F7D89461646DDF87083B0
:10DBB00000250027002041904FF4807101A8F2F762
:10DBC00049FBCF9860B1CF98F2F76BFB40B1B9F148
:10DBD000000F05D0B8F1000F02D00EB1D29828B9CD
:10DBE0004FF0FF300DF5537DBDE8F08F00240FE0BE
:10DBF00056F8240040B156F82400F2F752FB18B151
:10DC0000D29850F8240010B94FF0FF30EAE7641CB6
:10DC1000DD988442ECDB012243A8CF9903F0A6FDF6
:10DC2000CE90CE9810B16FF00100DBE70024FDE04C
:10DC3000ECE043AA4FF4807101A802F0A9FF4290E2
:10DC4000429888B946994898884201D1012000E05D
:10DC5000002018B1002048F82400E1E043A802F0B9
:10DC600086FF6FF00200BDE7002700250EE0F2F707
:10DC7000CBFA006801A9495D405C00F0010020B9C1
:10DC800001A8405D01A9C8557F1C6D1C01A8F2F7D1
:10DC900008FBA842EBD8002001A9C8559DF8040054
:10DCA000232800D1B2E059F8241001A8F2F7DDFAD8
:10DCB000B0B19DF804005B2812D101A8F2F7F1FA87
:10DCC000401E01A9085C5D280AD101A8F2F7E9FA13
:10DCD000A0F1020A59F82400F2F7E3FA824500D0D5
:10DCE00094E087E043AA4FF4807101A802F050FF4E
:10DCF0004290429888B946994898884201D10120BB
:10DD000000E0002018B1002048F824007CE043A87F
:10DD100002F02DFF6FF0020064E7002700250EE0FF
:10DD2000F2F772FA006801A9495D405C00F0010059
:10DD300020B901A8405D01A9C8557F1C6D1C01A830
:10DD4000F2F7AFFAA842EBD8002001A9C8559DF818
:10DD50000400232800D14DE056F8241001A8F2F762
:10DD600084FAA8B33D2101A8F2F791FA80B33D21CE
:10DD700001A8F2F78CFA824600208AF8000001A878
:10DD8000F2F78FFA834656F82400F2F78AFA8345B1
:10DD900000D02FE00AF1010A5046F2F782FA58F853
:10DDA0002410884205D943A802F0E1FE4FF0FF306D
:10DDB00018E75046F2F775FA8346D29951F82400D5
:10DDC0005A465146F2F72DFA4198401C41901BE00B
:10DDD000FFE79DF804005B280BD101A8F2F761FA78
:10DDE000401E01A9085C5D2803D1002048F82400EA
:10DDF0000AE000BF46994898884201D1012000E01E
:10DE0000002000283FF46EAF00BF09E04699489813
:10DE1000884201D1012000E0002000283FF409AF32
:10DE200000BF002143A802F0DBFE641CDD988442A1
:10DE3000FFF6FEAE43A802F09AFE4198D2E600003B
:10DE40002DE9FF4FADF6640D0F461D46DDF8A0A885
:10DE5000DDF89898DDF89C884FF48071C0A8F2F73F
:10DE6000F9F94FF4807180A8F2F7F4F94FF480715A
:10DE700040A8F2F7EFF9DDF8640870B1DDF8640846
:10DE8000F2F70FFA48B1DDF86C0830B1B8F1000FC5
:10DE900003D015B1B9F1000F05D14FF0FF300DF6E9
:10DEA000740DBDE8F08F00240EE055F8240038B161
:10DEB00055F82400F2F7F5F910B159F8240010B91B
:10DEC0004FF0FF30EBE7641C5445EEDB022F02DD20
:10DED0004FF0FF30E3E701220DF5C760DDF864186D
:10DEE00003F044FCCDF80404DDF8040410B16FF035
:10DEF0000100D4E7DDF86408F2F7D3F983465A4607
:10DF000040A8DDF86418F2F78CF9DDF86408F2F740
:10DF1000C8F940A930220A540B220DF20C4003F03C
:10DF200025FCCDF80404DDF8040430B10DF5C7601C
:10DF300002F01DFE6FF00100B1E70BE20DF5C762C4
:10DF40004FF48071C0A802F023FECDF80804DDF87C
:10DF50000804C0B9DDF84416DDF84C06884201D14A
:10DF6000012000E0002000B100E20DF20C4002F0C0
:10DF7000FEFD0DF5C76002F0FAFD40A803F0DCFEDF
:10DF80006FF002008BE70020CDF80004002614E0BB
:10DF9000F2F73AF90068C0A9895D405C00F0010021
:10DFA00050B9C0A8815D80AADDF800041154DDF8E5
:10DFB0000004401CCDF80004761CC0A8F2F771F9EB
:10DFC000B042E5D8002180AADDF8000411540DF21A
:10DFD0000C41C0A803F0D6FC9DF80002232800D114
:10DFE000B8E180A8DDF86C18F2F73FF900287DD081
:10DFF0009DF800025B2879D180A8F2F752F9401E03
:10E0000080A9085C5D28F6D180A8F2F74AF9A0F152
:10E01000020BDDF86C08F2F744F98345EBD12FE1F0
:10E020000DF5C7624FF48071C0A802F0B1FDCDF8C4
:10E030000804DDF80804C0B9DDF84416DDF84C0624
:10E04000884201D1012000E0002000B124E10DF25E
:10E050000C4002F08CFD0DF5C76002F088FD40A871
:10E0600003F06AFE6FF0020019E70020CDF800040B
:10E07000002614E0F2F7C8F80068C0A9895D405C8A
:10E0800000F0010050B9C0A8815D80AADDF800044D
:10E090001154DDF80004401CCDF80004761CC0A823
:10E0A000F2F7FFF8B042E5D8002180AADDF80004BD
:10E0B00011549DF80002232805D10DF20C41C0A88F
:10E0C00003F060FCDCE09DF800025B282ED180A804
:10E0D000F2F7E7F8401E80A9085C5D2826D1FFB959
:10E0E0004FF480716846F2F7B5F800E0F9E00024DB
:10E0F00013E058F8240078B1002048F8240059F8BB
:10E10000243055F82420A5A1684600F015FB0DF237
:10E110000C41684603F036FC641C5445E9DB00BF43
:10E120000DF20C41C0A803F02DFCB5E0B7BB0024F4
:10E130002BE055F82400F2F7B4F8834655F8241084
:10E140005A4680A8F2F7B4F8F0B93D2180A8F2F75A
:10E150009EF83F9000213F98017080A8F2F7A1F847
:10E16000834655F82400F2F79CF883450BD1002034
:10E1700048F8240059F8243055F8242087A1C0A875
:10E1800000F0DAFA03E000BF641C5445D1DB00BFA5
:10E190000DF20C41C0A803F0F5FB70E0FFE7012F82
:10E1A00035D1002420E055F82400F2F77AF88346B0
:10E1B00055F824105A4680A8F2F77AF898B93D210C
:10E1C000C0A8F2F764F83F9000213F98017080A842
:10E1D000F2F767F8834655F82400F2F762F88345B2
:10E1E00000D103E000BF641C5445DCDB00BF80A805
:10E1F000F2F757F8834655F82400F2F752F88345B2
:10E200003DD00DF20C41C0A803F0BCFB37E0022F5B
:10E2100035D100242BE055F82400F2F742F883466C
:10E2200055F824105A4680A8F2F742F8F0B93D217B
:10E2300080A8F2F72CF83F9000213F98017080A849
:10E24000F2F72FF8834655F82400F2F72AF88345B1
:10E250000BD1002048F8240059F8243055F8242028
:10E260004EA1C0A800F068FA03E000BF641C54454A
:10E27000D1DB00BF0DF20C41C0A803F083FB00BF4F
:10E28000DDF84416DDF84C06884201D1012000E09B
:10E29000002000283FF4C4AE00BFDDF84416DDF8CE
:10E2A0004C06884201D1012000E00020D0B1CFB956
:10E2B000002413E058F8240078B1002048F8240026
:10E2C00059F8243055F8242034A1C0A800F034FABD
:10E2D0000DF20C41C0A803F055FB641C5445E9DB6A
:10E2E00044E037E029E00DF5C7624FF48071C0A823
:10E2F00002F04EFCCDF80804DDF80804C0B9DDF8E2
:10E300004416DDF84C06884201D1012000E00020CF
:10E3100000B11DE00DF20C4002F029FC0DF5C760C4
:10E3200002F025FC40A803F007FD6FF00200B6E5FF
:10E330000DF20C41C0A803F025FBDDF84416DDF812
:10E340004C06884201D1012000E000200028CAD0FC
:10E3500000BF00BFDDF84416DDF84C06884201D14D
:10E36000012000E0002000283FF4E8AD00BF0DF2DE
:10E370000C4002F0FCFB0DF5C76002F0F8FBDDF885
:10E38000640803F0D9FCCDF8040440A8DDF8641853
:10E3900003F0E4FBCDF80404002080E52573203D64
:10E3A0002025730D0A0000002DE9FC4104460D46AE
:10E3B00016461F46DDF82080012033462A462146B6
:10E3C000CDE900700248FFF7EBFBBDE8FC810000DF
:10E3D000D407002010B586B000240D4805900D48E4
:10E3E00004900D48039040200290012002A903AB45
:10E3F00004AACDE9001005A90848FFF7D1FB04469F
:10E40000012C02D1002006B010BD4FF0FF30FAE71A
:10E41000C3000020CB000020D4070020BA3C010834
:10E420002DE9FE4304460D4616461F46DDE90A89DE
:10E4300033462A46214603488DE88003FFF700FD56
:10E44000BDE8FE83D407002010B501220EA10F48BD
:10E4500003F062F904460D2C14D14FF4007300222E
:10E46000114609A002F0AEFD04465CB9012206A1E6
:10E47000002003F051F90446012203A1034803F0F0
:10E480004BF90446204610BD303A00001408002025
:10E490000021034A22F81010024A1154704700006C
:10E4A000E8010020E40100207CB504460D46164634
:10E4B000002000900190200A8DF80000E0B28DF855
:10E4C0000100280A8DF80200E8B28DF803008DF8EB
:10E4D000046005236A460549002000F009F8034856
:10E4E0000088401C014908807CBD0000EE0100202E
:10E4F0002DE9FF4FADF22C4D8B4691461E4600276D
:10E500000024A24600250020CDF828048046CDF83E
:10E51000240440F21C4102A8F1F79CFEBBF1000F5D
:10E5200004D100200DF23C4DBDE8F08F40F2FF30E9
:10E53000B6FBF0F0401C1FFA80F80027F0E0B8F1BD
:10E54000010F13D0A8F10100B84204D042F6FF70C9
:10E55000CDF824040FE040F2FF30B6FBF0F100FBF1
:10E56000116040F43050CDF8240404E0B0B240F41F
:10E570004060CDF824040024DDF82C04000A02A930
:10E580000855641CDDF82C040855641C67480068B5
:10E59000000E0855641C65480068C0F30740085524
:10E5A000641C62480088C0F307200855641C5F485B
:10E5B00000780855641C5E480068000E0855641C0D
:10E5C0005B480068C0F307400855641C5848008841
:10E5D000C0F307200855641C554800780855641C92
:10E5E000DDF82404000A0855641CDDF824040855ED
:10E5F000641C00200855641C01200855641CBBF8ED
:10E600000000000A0855641C9BF800000855641CB3
:10E61000B8F1010F37D04FEA18200855641C01F8F3
:10E620000480641C781CC0F307200855641C781C07
:10E630000855641CA8F10100B8420CD040F2FF322A
:10E6400002FB079102AA101940F2FF32F1F7E9FD2F
:10E6500004F2FF3422E040F2FF30B6FBF0F100FBA1
:10E66000116040F2FF3202FB079102AA01901019DB
:10E67000019AF1F7D6FD40F2FF30B6FBF0F100FB56
:10E68000116004440AE0B9F1000F07D036B102A9C5
:10E69000081932464946F1F7C4FD3444002002A966
:10E6A000085502A802192146FFF78FF9641C0025BE
:10E6B0007F20204948556D1C4FF0000A20E002A839
:10E6C00010F80A007E2806D11A4948556D1C012011
:10E6D00048556D1C12E002A810F80A007F2807D1E7
:10E6E0007E20144948556D1C022048556D1C05E0DC
:10E6F00002A810F80A000F4948556D1C0AF1010ADA
:10E70000A245DCD37F200B4948556D1CAAB20120DD
:10E71000FAF7C8F9DDF828042844CDF828047F1C4E
:10E720004745FFF40CAFDDF82804FBE6CC010020E0
:10E73000D0010020C01300200FB4084B10B504A96D
:10E7400002AA039800F026F9044602A9002000F06E
:10E75000B8FC204610BC5DF814FB0000C3F00008B4
:10E7600002480068C0F30220704700000CED00E092
:10E7700010B5002804DB0A07130E054A135406E0FF
:10E780000A07140E034A00F00F031B1FD45410BDD8
:10E7900000E400E018ED00E000BF00BF00BFBFF3E1
:10E7A0004F8F00BF00BF00BF0948006800F4E06061
:10E7B00008490843001D0649086000BF00BF00BFAC
:10E7C000BFF34F8F00BF00BF00BF00BF00BFFDE71A
:10E7D0000CED00E00000FA0500487047F801002049
:10E7E0000148006870470000F801002002E008C8F6
:10E7F000121F08C1002AFAD170477047002001E0BB
:10E8000001C1121F002AFBD1704700F0010181F302
:10E81000138870470149086070470000F801002024
:10E820002DE9FF5FDDE90220010DDDF838B002437C
:10E8300018D044F61050A1F2FF3141430D140F9847
:10E84000012820D0A5EB0B00401C5FEA000A4FF026
:10E850000004474EDFF81C91A046504616D5CAF179
:10E86000000728E00F98012443A2012808D00021C6
:10E8700000980F9BC0E90021C0E90243BDE8FF9F5B
:10E880006FEA0B01F4E7CBF10000DEE7074612E088
:10E89000F80707D02246334640464946F2F7E2F8E9
:10E8A000804689462246334610461946F2F7DAF882
:10E8B00004460E467F10002FEAD1DDE90201BAF1CD
:10E8C000000F42464B4602DAF2F7CCF801E0F1F7CE
:10E8D0007AFE04460E460022284BF2F74DF903D883
:10E8E0004FF0FF30014607E00022254B204631461D
:10E8F000F1F7C2FDF2F728F9102409E0002C0ADB39
:10E900000A220023F1F730FC019B30321A55641EB5
:10E9100050EA0102F2D1641C019AC4F111031444BB
:10E920000F9A012A03D0012208430DD10AE00843BF
:10E9300004D000204FF0110B0F9080E7A3EB0B05E4
:10E940006D1E0DE05B4504DD4FF0000205F1010591
:10E9500004E003DA4FF00002A5F10105002AECD033
:10E9600000980F99C0E90231C0E9004586E7000030
:10E97000000024400000F03F300000000000F043A1
:10E980000000E03F30380A2801D201207047002003
:10E99000704700002DE9FF4F95B09B46894606461B
:10E9A00000250FE2252877D100242746F84A0121C7
:10E9B000059400E0044316F8013F203B01FA03F000
:10E9C0001042F7D130782A2811D06FF02F03307819
:10E9D000A0F13002092A16D8059A44F0020402EB8D
:10E9E000820203EB42021044761C0590EFE759F8CF
:10E9F000042B0592002A03DA504244F40054059097
:10EA000044F00204761C30782E2816D116F8010F37
:10EA100044F004042A280DD06FF02F023078A0F1C2
:10EA20003003092B09D807EB870302EB4303C71810
:10EA3000761CF3E759F8047B761C30786C280FD0ED
:10EA400006DC4C2817D068280DD06A2814D104E0C1
:10EA5000742810D07A280FD10DE044F400140AE095
:10EA600044F4801401E044F440147278824202D1EC
:10EA700004F58014761C761C307866280BD013DCE5
:10EA8000582877D009DC002875D04528F6D04628CC
:10EA9000F4D047281AD19DE118E0632835D06428C6
:10EAA00079D0652812D195E1702873D008DC6728E9
:10EAB000F1D069286FD06E280DD06F2806D1B5E04F
:10EAC00073282CD0752875D0782874D05A46179999
:10EAD00090476D1C75E1C4F30250022809D0032849
:10EAE0000DD0D9F8001004280DD00D6009F10409EB
:10EAF00067E1D9F80010EA17C1E90052F6E7D9F842
:10EB000000100D80F2E70D70F0E719F8041B8DF886
:10EB1000001000208DF80100EA46012003E059F8BA
:10EB200004AB4FF0FF3061074FF0000102D40DE05D
:10EB300008F101018846B9420FDA8045F8DB1AF87E
:10EB400008100029F4D108E008F10101884681424B
:10EB5000FADB1AF808100029F6D105985B46A0EBFD
:10EB6000080721463846179A00F094FA284400EB2B
:10EB7000080507E04DE029E10DE01AF8010B5A46BF
:10EB800017999047B8F10108F7D25B4621463846FD
:10EB9000179A13E142E00A220092C4F302524FF0A6
:10EBA000000A022A08D059F804CB032A4FEAEC7174
:10EBB0000AD00DE029E02AE009F1070121F007025F
:10EBC000F2E802C1914609E00FFA8CFC4FEAEC71C1
:10EBD000042A03D14FFA8CFC4FEAEC71002907DAC2
:10EBE0000A460021DCF1000C61EB02012D2202E05B
:10EBF000220504D52B228DF80420012203E0E20730
:10EC000001D02022F7E7904659E00A2102E01022C5
:10EC10000DE010214FF0000A00910BE010224FF0A0
:10EC2000000A44F004040827009203E008224FF091
:10EC3000000A0092C4F30252022A05D059F804CB0C
:10EC40000021032A08D009E009F1070121F0070299
:10EC5000F2E802C1914605E01FFA8CFC042A01D1BA
:10EC60000CF0FF0C4FF00008220728D5702806D0C2
:10EC7000009B83F0100353EA0A0305D00EE0402204
:10EC80008DF80420012208E05CEA010206D030225F
:10EC90008DF804208DF8050002229046009B83F039
:10ECA000080353EA0A030AD15CEA010201D16207B0
:10ECB00005D530228DF804204FF001087F1E58281A
:10ECC00004D034A003900EA802900DE036A0F9E71E
:10ECD00053466046009AF1F747FA84460398825CEF
:10ECE0000298401E029002705CEA0100F0D1029886
:10ECF00006A9081A00F1200A600702D524F480341E
:10ED000000E00127574502DDA7EB0A0000E00020E4
:10ED100000EB0A01009005984144401A0590E00379
:10ED200006D45B462146179A059800F0B3F90544CE
:10ED3000002706E001A85A46C05D179990476D1C50
:10ED40007F1C4745F6DBE0030CD55B462146179A4E
:10ED5000059800F09FF9054404E030205A461799C1
:10ED600090476D1C0099481E00900029F5DC08E0D2
:10ED7000029802995A460078491C029117999047C7
:10ED80006D1CBAF10001AAF1010AF1DC65E1000095
:10ED90000928010030313233343536373839616271
:10EDA0006364656600000000303132333435363735
:10EDB00038394142434445460000000000F058F90C
:10EDC0000544761C307800287FF4ECAD19B0284655
:10EDD000BDE8F08F620700D4062709F1070222F090
:10EDE000070CFCE80223E14603F000485FEA080C48
:10EDF00002D00FF2702C0DE05FEA045C02D50FF236
:10EE0000682C07E05FEAC47C02D00FF2602C01E0BE
:10EE1000AFF2700C4FF0FF3823F00043CDF850C034
:10EE200065280CD006DC452809D046281DD0472887
:10EE30003DD13DE0662818D067287ED138E000211A
:10EE4000112F01DB112000E0781CCDE9000106A99B
:10EE50000EA8FFF7E5FCDDE90F010E9A03910021F2
:10EE6000009207F1010A04914DE04FF00040009735
:10EE7000CDE9011006A90EA8FFF7D2FCDDE90F02CB
:10EE800003920E9B11990022DDF80CA000930492CE
:10EE900011B9791C00EB010AB7EB0A0004D4C0F1E8
:10EEA000FF3007F1010A0490AAEB0700019044E04B
:10EEB000012F00DA01270021112F01DD112000E0D0
:10EEC0003846CDE9000106A90EA8FFF7A9FCDDE947
:10EED0000F010E9A0391002104910092BA46210776
:10EEE0000CD40399514500DA8A46BAF1010F05DDC9
:10EEF000009AAAF10101515C302908D0B84202DA27
:10EF000010F1040F06DA0121CDE9011015E0AAF194
:10EF10000101E9E7002805DC049901440491AAEB0A
:10EF2000000102E0411C514500DD8A460499401A67
:10EF3000401C01904FF000400290200704D401983B
:10EF4000504501DBCDF8048000208DF84F00029879
:10EF50000DF14F07B0F1004F25D02B200E900298F5
:10EF60004FF0020800280CDA404202902D200E904B
:10EF700007E00A210298F1F733FC3031029007F8DC
:10EF8000011DB8F10001A8F10108F2DC0298002887
:10EF9000EFD1791E0E980870307800F0200040F014
:10EFA000450007F8020D12A8C01B00F107081498CD
:10EFB000007800B1012000EB0A01019801EBE0713B
:10EFC00005984144401A401E0590E00306D45B4674
:10EFD0002146179A059800F05DF8054414980078CA
:10EFE00018B15A46179990476D1CE00324D55B462B
:10EFF0002146179A059800F04DF805441CE0049846
:10F00000002807DBDDE90301884203DD0098405C4E
:10F01000179901E0179930205A469047049805F156
:10F020000105401C04900198401E019004D12E203F
:10F030005A46179990476D1CBAF10001AAF1010ACE
:10F04000DDDC05E017F8010B5A46179990476D1C57
:10F05000B8F10001A8F10108F4DC5B462146179ADB
:10F060000598ABE62D0000002B00000020000000FA
:10F070002DE9F041044600251E461746880404D4B5
:10F0800005E039462020B0476D1C641EF9D528469E
:10F09000BDE8F0812DE9F041044600251E4690466A
:10F0A000C80301D5302700E02027880404D505E0F7
:10F0B00041463846B0476D1C641EF9D52846BDE868
:10F0C000F0810A68531C0B601070704730B583B034
:10F0D0000446FFF785FB05460020CDE90000024607
:10F0E00021466846F1F7BFFB2846FFF793FBDDE9B1
:10F0F000000103B030BD2DE9F04F95B006460F4634
:10F10000914698460024A246A346002012901390F0
:10F11000149048216846F1F79DF8CDF848D006A82C
:10F1200013900CA81490404603F084FD0546002D72
:10F130006CD1002F6AD0012E11D14246394603F01E
:10F14000F4FF0546002D58D1387800F0800010B14A
:10F150004FF0010B51E04FF0000B02254DE0022E65
:10F1600001D0032E48D1414612A803F0D3FE054634
:10F170004FF0000B00240CE012A850F82400007897
:10F1800000F0800018B10BF1010000F0FF0B601CD3
:10F19000C4B2032C01DA002DEED0002411E0601C73
:10F1A00000F0FF0A08E012AA5146204604F0DEF9FA
:10F1B0000AF1010000F0FF0ABAF1030FF3DB601C53
:10F1C000C4B2022C01DA002DE9D000240BE012AA0F
:10F1D00052F8241004EB440207EBC2001822F1F7A6
:10F1E00020F8601CC4B2032C01DA002DEFD0BBF173
:10F1F000000F02D1022500E00125B9F1000F02D174
:10F200004FF0FF3504E089F800B001E04FF0FF3522
:10F21000284615B0BDE8F08FF8B504460E4664B137
:10F22000334601226946742000F00BF805469DF82C
:10F23000000000F00300207001E04FF0FF35284689
:10F24000F8BD2DE9F04106460F4690461C46204683
:10F2500003F0F0FC0546CDB9C7B1207B38B9214693
:10F26000304604F047F905460DB946F0800642469F
:10F2700039463046D4F840C06368E04784F84C0013
:10F2800094F84C0020B16FF0010501E04FF0FF351C
:10F290002846BDE8F08170B50446204600F099F993
:10F2A0000546B5B9234601222146D020FFF7C9FF04
:10F2B000054675B92078612809D1204604F00BF87D
:10F2C000054635B9204603F067F8054601E06FF0C2
:10F2D0000205284670BD00002DE9F04186B00446C5
:10F2E0000E4600274FF0010845A103C9CDE90301EF
:10F2F000002001900290314605A8FFF78DFF0546DA
:10F3000025B93146002000F0D5F8054614B94FF074
:10F31000FF355EE0002D5CD19DF80C0033460522E0
:10F3200001A9FFF78EFF0546002086F84D002DB994
:10F3300032460721E01C00F073F905462DB932462C
:10F340000521601C00F06CF905462DB932460521F7
:10F35000A01C00F065F905462DB93246052120466E
:10F3600000F05EF905462DB932460821201D00F057
:10F3700057F905466DBBE1789DF8080061F38400FC
:10F380008DF8080061789DF8070061F347108DF84B
:10F390000700A1789DF8070061F384008DF807004D
:10F3A00021789DF8050061F302008DF805002079B1
:10F3B000082802D027794FF000089DF8080067F36D
:10F3C00047108DF808009DF8040068F3C7108DF809
:10F3D000040035B93346052201A903A800F0A4F8BA
:10F3E00005469DF8140030B12DB931469DF8140042
:10F3F00000F060F80546284606B0BDE8F081000040
:10F4000071727374750000002DE9FE4380460D464D
:10F41000164600200290814625A000680090002D2D
:10F4200041D03146002000F045F8044634B9334657
:10F4300002AA4146284603F0ACFF044694BB33467B
:10F44000022201A97020FFF7FCFE044654BB287875
:10F45000012809D10027B068012802D14FF0020924
:10F4600005E04FF0010902E001274FF000099DF887
:10F47000040067F3C3008DF804009DF808109DF8A0
:10F48000050061F303008DF805009DF8050069F3A0
:10F4900005108DF805003346022201A9684600F0E8
:10F4A00043F8044601E04FF0FF342046BDE8FE83F8
:10F4B000707100002DE9FC4106460C4600277420BF
:10F4C000009000BF2346012201A97420FFF7B9FE76
:10F4D0000546ADB99DF8040000F0030787B19DF81B
:10F4E000040020F0030001902346012201A9684690
:10F4F00000F01AF8054642F21070A26C616890475D
:10F500000FB1002DDED066B15DB99DF8040066F341
:10F51000010001902346012201A9684600F004F889
:10F5200005462846BDE8FC812DE9F04385B0064636
:10F53000884617461D4614216846F0F78BFE28467C
:10F5400003F078FB8146B9F1000F3CD1002E3AD090
:10F55000B8F1000F37D097B30A2F31D8002417E045
:10F56000287B50B9305D294603F0C4FF8146305DE9
:10F5700000F07F000DF8140002E0305D0DF814007B
:10F5800018F804106000401C0DF80010601C84B2D4
:10F59000BC42E5D3B9F1000F17D179004A1E9DF89E
:10F5A00000000DF10101D5F844C06B68E04785F813
:10F5B0004C0095F84C0040B16FF0010905E0FFE701
:10F5C0006FF0030901E04FF0FF39484605B0BDE890
:10F5D000F0837CB50446E0200190B62000902046E0
:10F5E00003F028FB0546CDB9207B18B9204603F06F
:10F5F0004BF8054695B923460122694601A8FFF755
:10F6000093FF054642F21070A26C616890472DB9D5
:10F61000207B18B9204603F037F8054628467CBD04
:10F620002DE9F04104460E461546284603F002FB3C
:10F6300007465CB157B92078B04209DD267095F8CD
:10F640004D0040F0010085F84D0001E04FF0FF371C
:10F650003846BDE8F08100002DE9F05F05460E4612
:10F660004FF4802020FA06F8A5F5007404EB44045A
:10F6700004F580542046F1F715F882464046F1F72C
:10F680001AF883460549F0F787FE81465146F0F7A0
:10F69000B5FE07463846BDE8F09F000000247449D7
:10F6A0002DE9F04FA7B006460C4615463046F1F757
:10F6B00002F82590012101FA04F0F0F7FCFF2490F4
:10F6C00040222C4914A8F0F7ACFD402229494031D2
:10F6D00004A8F0F7A6FD95F93E00F0F7E3FF834696
:10F6E0002549F0F759FE82462449F0F7FDFD804692
:10F6F00014A951F824002249F0F780FE83464FF008
:10F700007E51F0F7F1FD82464146F0F745FE814615
:10F7100004A951F824001A49F0F770FE82464FF010
:10F720007E51F0F7E1FD26904FF088412598F0F7E3
:10F730002DFE49460190F0F761FE83464FF07E5161
:10F74000F0F7D2FD0F4903902698F0F725FE834687
:10F750002499F0F721FE02900399F0F71DFE8246EE
:10F7600051464FF07E50F0F749FE0746384627B025
:10F77000BDE8F08FD03701080000A0400080A7440A
:10F780000000C842BD37063410B501460022B1F56D
:10F790007C6F01DBFF200DE007E00B46CC1701EB8F
:10F7A0009474C4F38F01531CDAB23F29F5DC01EBEA
:10F7B0008213D8B210BD10B50146002240F2837307
:10F7C000994201DBFF2010E04FF47A734B4340F283
:10F7D000DD14B3FBF4F399B202E08910531CDAB2E2
:10F7E0003F29FADC01EB8213D8B210BD2DE9F04FAE
:10F7F00089B005460C464E49A06BF0F7FFFD03901B
:10F8000094F91400F0F74EFF83464FF08041F0F773
:10F81000F5FD81460399F0F7BFFD0746208AF0F712
:10F820004AFF81464FF08341F0F7B6FD80463946E6
:10F83000F0F75AFD06462846F0F73DFF824631466E
:10F84000F0F7A4FD079094F91600F0F72BFF4FF0A6
:10F8500093410190F0F7D2FD83460399F0F79CFDA8
:10F8600082460399F0F798FD814694F91500F0F768
:10F8700019FF4FF08D410190F0F7C0FD83460399C9
:10F88000F0F78AFD82464FF07E51F0F72DFD494694
:10F890000290F0F729FD0746608AF0F70CFF8146D9
:10F8A0004FF09141F0F7AAFD80463946F0F774FD1C
:10F8B00006460799F0F770FD0690E07DF0F7FBFE35
:10F8C00006464FF08D41F0F799FD059094F9180028
:10F8D000F0F7E8FE06464FF09441F0F78FFD0490F4
:10F8E000DDE90310F0F758FD81460599F0F7FCFCBF
:10F8F00080460699F0F750FD07460699F0F74CFD53
:10F9000006460699F0F7F0FC08900A490898F0F7C7
:10F910005DFF02D20748089006E000210898F0F742
:10F920004BFF01D200200890089809B0BDE8F08F85
:10F930000000A0450000C8422DE9F34F83B00C46FB
:10F940004FF08041A06BF0F759FD81468149F0F7F7
:10F950001DFD054694F92E00F0F7A4FE83464FF0F6
:10F960009041F0F74BFD814629462846F0F714FDFB
:10F9700082464946F0F710FD0646B4F92C00F0F730
:10F9800091FE83462946F0F707FD82464FF08041FD
:10F99000F0F702FD81463146F0F7A6FC0646B4F9C1
:10F9A0002A00F0F77FFE83464FF08F41F0F7F4FC1A
:10F9B00081464FF081413046F0F720FD82464946AE
:10F9C000F0F792FC0646B4F92600F0F76BFE83468A
:10F9D0002946F0F7E1FC824694F92800F0F762FE30
:10F9E00029460090F0F7D8FC83462946F0F7D4FC6E
:10F9F0004FF08D410190F0F701FD51460290F0F774
:10FA000073FC81464FF09241F0F7F8FC0546A08C5C
:10FA1000F0F751FE82464FF08E412846F0F7EEFC9B
:10FA200083464FF07E51F0F75FFC81465146F0F778
:10FA3000B3FC05460398F0F73EFE81464FF0934134
:10FA4000F0F7A7FC80462846F0F759FE00287BD047
:10FA50004FF08B413046F0F7D1FC83464146F0F73A
:10FA600098FC82463C49F0F797FC81462946F0F71E
:10FA7000C5FC8046B4F93200F0F714FE83464146D7
:10FA8000F0F78AFC82464146F0F786FC81464FF04B
:10FA90009E41F0F7B3FC0546B4F93000F0F702FEE2
:10FAA00082464FF08E41F0F7A9FC81464146F0F7BF
:10FAB00073FC064694F83400F0F7FDFD83464FF0E2
:10FAC0009041F0F79BFC81464FF087414046F0F7AC
:10FAD00095FC4FF0874102904046F0F78FFC4FF0C5
:10FAE000874101904046F0F789FC00900199F0F7BA
:10FAF00053FC83460299F0F74FFC82464946F0F7E3
:10FB00004BFC074694F92F00F0F7CCFD4FF08641EF
:10FB10000190F0F741FC834631462846F0F7E4FBBC
:10FB200039460190F0F7E0FB59460290F0F7DCFB14
:10FB300082464FF08341F0F761FC81464146F0F781
:10FB4000D3FB804602E0FFE74FF00008404605B0D7
:10FB5000BDE8F08F00007A470050C3452DE9F04F13
:10FB600089B005460C46B5F5C87F01DD4FF4C87570
:10FB700094F91900F0F796FD4FF083410790F0F7E4
:10FB80003DFC3D490890F0F7AFFB0646B4F91A007A
:10FB9000F0F788FD4FF08E410690F0F72FFC3749C3
:10FBA0000790F0F7F9FB36490890F0F79DFB074600
:10FBB00094F91C00F0F776FD4FF089410890F0F7BA
:10FBC0001DFC80462846F0F776FD39460690F0F792
:10FBD000E3FB4FF07E510790F0F786FB314608902B
:10FBE000F0F7DAFB814694F90E00F0F75BFD414631
:10FBF0000790F0F7D1FB49460890F0F775FB824675
:10FC000094F93D00F0F74EFD1E490190F0F7C4FB5A
:10FC10004FF07E510290F0F767FB014603904FF0E2
:10FC20007E50F0F7EBFB059094F83C00F0F743FDB5
:10FC30004FF081410190F0F757FB014602904FF0E1
:10FC40008140F0F7DBFB51460390F0F7A5FB0490F1
:10FC50000599F0F7A1FB0C490690F0F797FB0B49CB
:10FC60000790F0F799FB0890F0F762FD00F0FF0BAA
:10FC7000584609B0BDE8F08F000044426F12033AC5
:10FC800075021A3B6F12033B0000C8419A99594014
:10FC90002DE9FF5F05460C46B4F92000F0F702FDA0
:10FCA0008246E08BF0F707FD83464FF08941F0F77D
:10FCB000A5FB80462846F0F7FEFC83464FF08D41B9
:10FCC000F0F79CFB07464146F0F760FB8146514642
:10FCD000F0F762FB064694F92200F0F7E3FC814658
:10FCE0004FF08341F0F758FB0746E08BF0F7E3FC59
:10FCF0004FF08C410090F0F781FB82462846F0F7E8
:10FD0000DAFC4FF090410090F0F778FB83465146C3
:10FD1000F0F73CFB8146E08BF0F7CDFC4FF08C41D7
:10FD20000090F0F76BFB82462846F0F7C4FC4FF0DA
:10FD300090410090F0F762FB83465146F0F726FBB6
:10FD400049460190F0F728FB80463946F0F724FB3E
:10FD5000039030460399F0F7C7FAA0630449A06BFB
:10FD6000F0F74CFB0290029804B0BDE8F09F000051
:10FD70000000A0452DE9F041044688460020E070CF
:10FD8000401E60634146204602F03AFF10B1042055
:10FD9000BDE8F08104F2362002F0B1FC074694F889
:10FDA0003850EB2D03D0E92D01D0E82D34D14AF69F
:10FDB0005520874208D108221BA104F18A0002F0D5
:10FDC000A1FD08B90020E3E704F1430002F097FC2D
:10FDD0000646701E3040F8B9B6F5007F1CDBB6F55C
:10FDE000007F19DC4520055DB5B1681E284098B933
:10FDF0004820005D012803D04820005D02280BD177
:10FE000004F1490002F07BFC30B104F14E0002F035
:10FE100076FC08B10020BBE74AF65520874201D1A5
:10FE20000220B5E70320B3E74641543332202020B7
:10FE300000000000024600E0521C107810B110785B
:10FE40008842F9D110787047F0B503460D461E6818
:10FE5000986A021D680A7789B0FBF7F400BF02CAEE
:10FE600009B90020F0BD8C4200D202E0641A121DD4
:10FE7000F5E700BF10682044F4E70246891ED06908
:10FE8000801E884201D8002070475389106B03FB05
:10FE90000100F9E72DE9F04780460C4604F11A000D
:10FEA00002F02DFC10B10020BDE8F087207800F0B2
:10FEB0003F00401E00EB800101EBC0054FF001093F
:10FEC000002621E01849895D081902F018FC074650
:10FED000B9F1000F11D0FF2D0BD8384602F0D4F83D
:10FEE000824629466D1C38F8110002F0CDF8824593
:10FEF00001D00020D8E7B94605E04FF6FF708742F1
:10FF000001D00020D0E7761C0D2EDBD3207800F046
:10FF1000400038B1B9F1000F04D038F8150008B12D
:10FF20000020C1E70120BFE7503801082DE9F04764
:10FF300082468846DAF80040B8F1000F06D12769FA
:10FF400017B1E069B84215D8012713E04146504681
:10FF500002F0E3FA0546022D02D20120BDE8F08747
:10FF6000681C08B92846F9E7E069A84201D9284683
:10FF7000F4E74746606908B90020EFE700264745E7
:10FF800018D17E1CE069B04200D8022631465046A6
:10FF900002F0C3FA0546012D01D0681C08B92846B5
:10FFA000DCE73DB12569022D03D3E069A84200D901
:10FFB0002F460026E6B93E4600BF761CE069B042F7
:10FFC00004D80226BE4201D90020C7E73146504678
:10FFD00002F0A3FA054605B909E0012D01D0681C1D
:10FFE00008B92846BAE7BE42E7D10020B6E700BF0D
:10FFF0004FF0FF323146204602F06EFE8146B9F1E5
:020000040801F1
:10000000000F08D1B8F1000F05D032464146204616
:1000100002F062FE8146B9F1000F0DD12661E06960
:10002000801E6169814202D86069401E606120794A
:1000300040F00100207107E0B9F1010F02D14FF04B
:10004000FF3000E001200646304687E72DE9F34FF8
:1000500083B08146049800680090D9F80000C76812
:10006000002500BF684603F062FB02900298401C26
:1000700018B9062005B0BDE8F08F0298B0F5803FB2
:1000800005D30298020C28466D1C27F81020029810
:1000900084B2202C03DB2F2C01D05C2C00D111E08A
:1000A000802C06DA214693A0FFF7C4FE08B1062093
:1000B000E0E7FF2D01D30620DCE728466D1C27F87A
:1000C0001040CFE700BF202C01DA04260CE0002608
:1000D00002E00098401C0090009800782F28F8D08B
:1000E000009800785C28F4D0009904980160012DF4
:1000F00004D1681E37F810002E280BD0022D24D111
:10010000681E37F810002E281FD1A81E37F81000DF
:100110002E281AD1002027F8150080460AE0A845AD
:1001200001D22E2100E0202109F1200000F8081062
:1001300008F10108B8F10B0FF1D346F0200109F1E5
:10014000200000F80810002094E708E0681E37F847
:100150001040202C02D02E2C00D002E06D1E002D6D
:10016000F4D100BF002027F815000DB9062081E763
:100170004FF0000A01E00AF1010A37F81A002028BE
:10018000F9D0BAF1000F03D137F81A002E2801D1A7
:1001900046F0030600E06D1E25B1681E37F810001A
:1001A0002E28F8D10B22202109F1200002F0C9FBF2
:1001B0004FF00008C3460820019000BF50460AF1E6
:1001C000010A37F8104004B968E0202C03D02E2C27
:1001D00004D1AA4502D046F00306EFE70198804516
:1001E00001D2AA4516D101980B2802D146F0030688
:1001F00054E0AA4501D046F00306AA4500D94DE0D7
:10020000AA464FF008080B2001904FEA8B604FEA96
:10021000106BD3E7802C0EDB46F0020640F2B511DE
:10022000204601F011FF044604F0800018B104F0EC
:100230007F0033490C5CFF2C10DD0198401E4045C7
:1002400004D846F00306DDF80480B7E722124046E2
:1002500008F1010809F120010A5418E024B12146EF
:1002600028A0FFF7E7FD18B15F2446F003060EE073
:10027000412C03DB5A2C01DC4BF0020B612C06DB1A
:100280007A2C04DC4BF0010BA4F1200084B2404630
:1002900008F1010809F120010C548FE700BF99F81B
:1002A0002000E52802D1052089F8200001980828BF
:1002B00003D14FEA8B604FEA106B0BF00C000C2857
:1002C00003D00BF00300032801D146F0020606F02C
:1002D000020048B90BF0010008B146F010060BF01F
:1002E000040008B146F008062B2000F80960002041
:1002F000C0E60000222A3A3C3E3F7C7F000000001E
:100300005D3801082B2C3B3D5B5D00002DE9FF4F64
:1003100085B09A4603AA0121059800F0C1FB18B1E7
:10032000012009B0BDE8F08FDDF80C904FF03F08D8
:10033000082701E07806070E37B1B9FBF7F0B0FBEC
:10034000F8F0B0F5806FF5D807B9FF274FF40072C9
:100350000021504602F0F5FA0AF5DF764FF0000B67
:10036000444669E0069850F82B50642D07D801D117
:10037000484603E06420B9FBF0F068430546601985
:10038000484501D8601901D3A9EB040505B959E026
:10039000214606F1080003F031F9294606F10C0068
:1003A00003F02CF907983071B4FBF8F0B0FBF7F0CC
:1003B0000490B4FBF8F0B0FBF7F107FB1100C0B2FA
:1003C0000290B4FBF8F008FB1040401CC0B2019052
:1003D00002987070C021049801EA900001990843C6
:1003E000B0700498F0706019401EB0FBF8F0B0FBDC
:1003F000F7F004906019401EB0FBF8F0B0FBF7F185
:1004000007FB1100C0B202906019401EB0FBF8F16A
:1004100008FB1100401CC0B2019002987071C0210D
:10042000049801EA900001990843B0710498F071B2
:1004300010360BF1010B2C44BBF1040F02D20CB1AE
:100440004C458FD300BF4AF655210AF5FF7003F0E3
:10045000E1F8012300225146059800F072FB08B133
:1004600001205EE700205CE7014609B100207047EB
:100470000020FCE7014609B1002070470020FCE79E
:100480002DE9F04104460E46D4F8008000212046B4
:1004900000F0A6FA0546EDB9002700BF4046A16965
:1004A00002F0AEFB054605B113E0E0690078E528EF
:1004B00002D0E069007820B9781C0746B04201D12B
:1004C00007E000270121204600F0EBF80546002D4B
:1004D000E4D000BF042D00D107252846BDE8F081F7
:1004E0002DE9F04704468946204603F0FBF810B199
:1004F0000120BDE8F08749462046FFF7BEFC0746CD
:1005000067634FF40072002104F1380002F019FA19
:1005100060894FF40041B1EB402F01D8084601E05B
:100520006089400206464FF0000800E07608B6F504
:10053000007F05D9304601F064FDB0F10008F5D028
:10054000B6F5007F17D932460021404602F0F9F98E
:10055000760A002500E035446089A84207D97A1957
:1005600060783346414600F0ECFA0028F3D040466C
:1005700001F04DFD10E004F138080126002500E0EF
:1005800035446089A84207D97A19607833464146D4
:1005900000F0D7FA0028F3D06089A84201D00120EA
:1005A000A7E70020A5E72DE9F0470446D4F800A00E
:1005B0000021204600F014FA064616B13046BDE888
:1005C000F0874FF0FF08C1464FF0FF30E06200BFF8
:1005D0005046A16902F014FB064606B15EE0E069F0
:1005E00005780DB9042659E0E069C07A00F03F07AC
:1005F000A771E52D04D007F0080038B10F2F05D002
:100600004FF0FF084FF0FF30E06240E00F2F22D1A3
:100610002B20005D00F0400098BB05F0400038B191
:10062000E06990F80D9005F0BF05A8462069E062EA
:1006300045450CD1E069407B484508D1E169DAF8CD
:100640000C00FFF727FC10B1A8F1010000E0FF202B
:1006500000F0FF081BE0B8F1000F05D1E06902F0DF
:10066000DFFF484500D119E02B20005D00F00100BC
:1006700040B90B2204F12001E06902F043F908B906
:100680000CE004E04FF0FF084FF0FF30E062002183
:10069000204600F006F80646002E99D000BF3046EE
:1006A0008DE72DE9F041044688462768206900F16E
:1006B0002006B6F5001F01D30020A061A06910B983
:1006C0000420BDE8F081C6F30800002845D1A069E8
:1006D000401CA061606938B93889B0EB561F3CD81E
:1006E0000020A0610420ECE77889401E00EA562033
:1006F00098BB2046616901F010FF0546012D01D825
:100700000220DEE7681C08B90120DAE7F869A84290
:100710001DD8B8F1000F03D10020A0610420D0E75C
:1007200020466169FFF702FC05460DB90720C8E7BE
:10073000012D01D10220C4E7681C08B90120C0E7DF
:1007400029463846FFF7CCFE08B10120B9E76561BC
:1007500029463846FFF791FBA0612661C6F30801E0
:1007600007F138000844E0610020AAE72DE9F05FB6
:10077000044689460426D4F800A04FF0FF08C3467B
:1007800053E05046A16902F03BFA064606B14FE03D
:10079000E06905780DB904264AE0E069C07A00F006
:1007A0003F07A771E52D0AD02E2D08D027F0200095
:1007B000082801D1012000E00020484502D04FF078
:1007C000FF082BE00F2F1DD105F0400038B1E06984
:1007D00090F80DB005F0BF05A8462069E0624545D8
:1007E0000CD1E069407B584508D1E169DAF80C008A
:1007F00002F02CFA10B1A8F1010000E0FF2000F097
:10080000FF080BE0B8F1000F04D1E06902F008FF27
:10081000584502D04FF0FF30E06209E00021204649
:10082000FFF73FFF064606B102E0A0690028A8D105
:1008300000BF0EB10020A0613046BDE8F09F2DE959
:10084000FE4F044626682B20005D00F0A00010B18A
:100850000620BDE8FE8F4FF0000901E009F1010913
:10086000F06830F819000028F8D10C2204F12001BA
:10087000684602F059F89DF80B0000F0010028B31B
:1008800040212B2001554FF001080EE043466946F8
:1008900004F12000F26801F019FD2046FFF783FE05
:1008A000054605B104E008F10108B8F1640FEDD385
:1008B00000BFB8F1640F01D10720CAE7042D01D0B1
:1008C0002846C6E79DF80B102B2001559DF80B001C
:1008D00000F0020030B109F10C000D21B0FBF1F085
:1008E000401C00E00120074639462046FFF7C8FDBE
:1008F00005464DBB781E071E26D02069A0EB471188
:10090000204600F06DF80546F5B904F1200002F02C
:1009100087FE824600BF3046A16902F071F90546A4
:1009200005B110E0FAB2E1695346F06802F070FADE
:100930000120F07000212046FFF7B3FE054615B9EF
:10094000781E071EE7D100BFC5B93046A16902F085
:1009500057F9054695B920220021E06901F0F1FF21
:100960000B2204F12001E06901F0DEFF2B20005D85
:1009700000F01800E16908730120F070284668E76C
:100980002DE9F041044626682769E06A401C08B951
:10099000002003E02046E16A00F022F80546E5B9B0
:1009A00000BF3046A16902F02BF9054605B110E001
:1009B00000BFE520E16908700120F0702069B842AD
:1009C00000D306E000212046FFF76BFE0546002D10
:1009D000E7D000BF042D00D102252846BDE8F081F4
:1009E0002DE9F04104460D462668B5F5001F02D2F8
:1009F00005F01F0010B10220BDE8F0812561A76855
:100A00001FB93078032800DBF76A47B93089B0EBAB
:100A1000551F01D80220EFE7F06AA0611CE0708941
:100A20004FEA402811E03946204601F076FD07469E
:100A3000781C08B90120DFE7022F02D3F069B84221
:100A400001D80220D8E7A5EB08054545EBD2394689
:100A50003046FFF712FAA0616761A06908B9022069
:100A6000CAE7A06900EB5520A061C5F3080106F1B3
:100A700038000844E0610020BEE770B5054665B95E
:100A8000FAF75EF9044634B10020FAF7FEFAFF20C7
:100A9000FAF7F4FA01E0002070BD00BF0120FBE787
:100AA0002DE9F04106460F4615462EBB37B1012F02
:100AB0001AD0022F0FD0032F1BD111E00020FAF71C
:100AC000D6FAFAF7E9FA08B9002400E00124012077
:100AD000FAF7CDFA0FE04FF40070288000240AE006
:100AE00008202880002406E0FAF7EFF828600024A8
:100AF00001E0042400BF00E001242046BDE8F081AD
:100B00002DE9F04106460F4690461C4614B90420D4
:100B1000BDE8F0816EB9E2B241463846FAF7DCF939
:100B2000054625B1FF20FAF7A9FA0120F0E70020D9
:100B3000EEE70420ECE7014609B9002070470120E8
:100B4000FCE72DE9F04105460E461746984665B983
:100B500008F0FF0239463046FAF7BEFA044614B9E7
:100B60000020BDE8F0810120FBE70420F9E738B55B
:100B70000546284601F090F804463CB969462846E7
:100B800002F0FBFD04460CB900202860204638BD69
:100B90002DE9FC4780460C46914600254646641EDA
:100BA00013E06B46012201A9484600F001FF0098BE
:100BB000012800D00BE09DF8047000BF06F8017B0F
:100BC0006D1C0A2F00D102E000BFA542E9DB00BF87
:100BD0000020307015B14046BDE8FC870020FBE7DF
:100BE0002DE9F04F89B004460D4607A9204602F0D2
:100BF000C4FD0890089808B9607C0890089818B15E
:100C0000089809B0BDE8F08FA06A00287CD0681C65
:100C1000002843D1D4F8289059F8040B0290022000
:100C20000190A76867B300BF039700200490019864
:100C3000801C019000BF05970498401C0490394621
:100C4000204601F06AFC0746012F02D8022060749A
:100C5000D7E7781C10B901206074D2E70598401CD2
:100C60008742E8D0DDE90101884205D8049849F8B7
:100C7000040B039849F8040B0798C069B842D3D80D
:100C80000198A16A0860DDE90101884203D80020CB
:100C9000C9F80000FAE011200890F7E0E068A842E7
:100CA00000D2E5686561002DF4D0691E2046FFF78B
:100CB000CBF8A061A1690798FFF7DFF88246BAF187
:100CC000000F02D1022060749BE707984089401E04
:100CD000691E00EA51208244A08AC0F3080000285F
:100CE000D8D0E0695045D5D0207C00F0800080B19C
:100CF000E26907994878012304F12C01FFF721FFED
:100D000018B1012060747CE712E0207C00F07F00C5
:100D10002074079948780123524604F12C01FFF70B
:100D2000EFFE10B1012060746BE7C4F81CA0ADE0C9
:100D3000E068A84204D2207C00F0020000B9E56817
:100D4000606906904FF0000BC4F814B0002D6AD013
:100D5000079840894FEA4028069890B1681EB0FB7A
:100D6000F8F10698401EB0FBF8F0814209D30698CE
:100D7000401EA8F101018843606160692D1AA669CF
:100D800012E0A6687EB900212046FFF7CFF806469C
:100D9000012E02D10220607433E7701C10B90120CB
:100DA00060742EE7A660A661D6B325E0A5EB080522
:100DB000606940446061207C00F0020040B100BFE7
:100DC00031462046FFF7B2F8064636B9002515E051
:100DD0003146204601F0A1FB0646701C10B90120E7
:100DE00060740EE7012E03D90798C069B04202D89B
:100DF0000220607405E7A6614545D7D800BF606949
:100E000028446061C5F3080050B131460798FFF7E8
:100E100034F88346BBF1000F03D102206074F0E682
:100E200001E00BEB552BE1686069884205D96069E8
:100E3000E060207C40F040002074A08AC0F30800ED
:100E400020B3E069584521D0207C00F0800078B1C3
:100E5000E26907994878012304F12C01FFF771FE3C
:100E600010B101206074CCE6207C00F07F0020747B
:100E70000799487801235A4604F12C01FFF740FEF8
:100E800010B101206074BCE6C4F81CB00898B8E644
:100E90002DE9F14191B00222694611A801F05AFDF5
:100EA0000446002C7ED1009805904FF4007001F0AC
:100EB000A8F806461EB9112012B0BDE8F0810098CE
:100EC000C66005A8119901F073F9044604B9082415
:100ED000042C05D19DF83F0000F0200000B106244D
:100EE000042C6AD100980190002101A8FFF71EF898
:100EF0000546002405B90724012D00D10224681CF1
:100F000000B9012401F079FB8046BCBB294600985A
:100F1000FFF7E6FA04468CBB0B22202100983830FC
:100F200001F00FFD2E20009981F838001021009863
:100F300080F84310414600984E3002F05FFB2A468D
:100F400000993831009802F047FB2022009938318F
:100F50000098583001F0E8FC2E21009880F85910D4
:100F6000079F3A4600995831009802F035FB01205E
:100F70000099C87005A8FFF762FC0446C4B90C9933
:100F800001F11600414602F039FB2A460C990098FF
:100F900002F022FB10200C99C87201200099C87041
:100FA0002CB900E00CE0009802F054FB044604E089
:100FB0000022294601A802F09FF9304601F027F8E7
:100FC000204679E72DE9FF4F99B00F46154619A83D
:100FD00001F030FB03900398002803DA0B201DB0CA
:100FE000BDE8F08FFC49039851F8200028B100219A
:100FF000F94A039852F8200001700398C0B2169085
:101000000020159007B9F54F1698FFF736FD0290AE
:10101000029800F0010008B10320E0E7029800F018
:10102000040008B10A20DAE778681390139838B9F9
:1010300013AA03211698FFF733FD08B1012013907E
:10104000139840B11398B0F5004F04D81398401E80
:101050001399084008B1012013904FF400793878B3
:1010600000F00F0018907878012804DB78780228C7
:1010700001DC787800E001200690B96889B1B96890
:10108000B1F5004F0DD848464FEAE97109EBD1613F
:101090004911BA68B2FBF1F301FB132109B9B96830
:1010A00001E04FF400710591F868B0F1807F05D838
:1010B000F868411E084008B9F86800E00020079071
:1010C0000798B0FBF9F007901C98B0FBF9F014906A
:1010D000149808B9112082E72C462CB9149901FB09
:1010E00009F000F08EFF04460CB9112077E70020CC
:1010F0001190109000BF11AA01211698FFF7D0FCA3
:1011000028B115B9204600F082FF012067E7189842
:1011100000F0080040B911983F2805D93F201090F1
:10112000DDE91001081A11901198802805D215B92F
:10113000204600F06CFF0E2051E700BF00BF07986B
:10114000802801D980200790189800F0020030B163
:10115000189800F0010010B94FF003080CE018983F
:1011600000F0010028B915B9204600F050FF132007
:1011700035E74FF0020800BF00BF00BF079EB8F17F
:10118000030F31D1A6B911984FEA504B00200490BB
:10119000012603E00498401C0490760090490498CE
:1011A00031F8100020B1049831F810005845F1D9F9
:1011B0001198B0FBF6FA082000EB8A004844401E64
:1011C000B0FBF9F0099020200A90002008904FF61B
:1011D000F570824502D9834882453BD915B920462E
:1011E00000F015FF0E20FAE6A6B911984FEA103B61
:1011F00000200490012603E00498401C049076002F
:101200007949049831F8100020B1049831F81000A1
:101210005845F1D91198B0FBF6FA40F6F5708245C1
:1012200003D9042000EB4A0B07E04FF001080AEB5A
:101230004A00401C032101EB500B0BEB0900401E40
:10124000B0FBF9F0099001200A9005984001B0FB2D
:10125000F9F008900A99109808440F90069A099995
:101260000F9801FB0201089808440E9013990E98FC
:101270000844401E491E20EA01010E98A1EB000B14
:10128000B8F1030F06D10A9858440A900F985844B1
:101290000F9013E00698BBFBF0F100FB11B038B1E2
:1012A000ABF1010B0A98401C0A900F98401C0F905C
:1012B0000698BBFBF0F10998084409900E9800EBE2
:1012C00006111098081A1199884205D915B92046B7
:1012D00000F09DFE0E2082E611990A980A1A0699DE
:1012E000099800FB11210898081AB0FBF6FAB8F12A
:1012F000030F0FD14FF6F57082450BD8079818B938
:101300007008079000B148E015B9204600F07FFE54
:101310000E2064E6B8F1020F31D14FF6F570824528
:101320001CD9079830B94020B0EB460F02D37000AB
:10133000079032E0189800F0020010B14FF0030857
:101340002BE0079820B970000790802800D824E08F
:1013500015B9204600F05BFE0E2040E640F6F57021
:1013600082450CD8079820B970000790802800D8D3
:1013700013E015B9204600F04AFE0E202FE6B8F122
:10138000010F09D140F6F570824505D915B92046FF
:1013900000F03DFE0E2022E600E0EFE600BF4A46E8
:1013A0000021204601F0CDFA0B2210A1204601F0C9
:1013B000BBFA494604F10B0002F02CF966730A9857
:1013C00081B204F10E0002F025F906982074B8F1FC
:1013D000030F11D1002010E0BC000020FC380108F0
:1013E000EC380108F5FFFF0FDE380108EBFE904DE9
:1013F00053444F53352E3000059881B204F111004B
:1014000002F008F91198B0F5803F06D2119881B228
:1014100004F1130002F0FEF804E004F12000119939
:1014200002F0ECF8F82060753F2104F1180002F09A
:10143000F1F8FF2104F11A0002F0ECF804F11C00AD
:10144000109902F0DBF8B8F1030F28D101F0D5F8BC
:101450000146009004F1430002F0D0F804F12400AA
:10146000099902F0CBF8022104F12C0002F0C6F831
:10147000012104F1300002F0CDF8062104F1320020
:1014800002F0C8F8802084F84000292084F8420047
:10149000132294A104F1470001F046FA19E001F08B
:1014A000ACF80146009004F1270002F0A7F8099873
:1014B00081B204F1160002F0ADF8802084F8240017
:1014C000292084F8260013228BA104F12B0001F0BF
:1014D0002BFA4AF6552104F5FF7002F09BF8012320
:1014E0002146109A1698FFF72CFB28B115B9204613
:1014F00000F08DFD012072E5B8F1030F33D1012317
:10150000109A921D21461698FFF71BFB4A460021B0
:10151000204601F016FA7D49204602F06FF87C491A
:1015200004F5F27002F06AF8AAF1010104F5F47012
:1015300002F064F8022104F5F67002F05FF84AF652
:10154000552104F5FF7002F065F80123109AD21DB1
:1015500021461698FFF7F5FA0123109A521C2146EE
:101560001698FFF7EEFA149800FB09F200212046C6
:1015700001F0E7F90F980D900020049048E0B8F1D1
:10158000030F10D16FF00701204602F037F84FF03B
:10159000FF31201D02F032F86FF0704104F10800B5
:1015A00002F02CF80AE0B8F1010F01D1594801E02E
:1015B0006FF007000146204602F020F809981290CB
:1015C00000BF14991298884201D9149800E012982B
:1015D00083465B4621460D9A1698FFF7B2FA28B16A
:1015E00015B9204600F013FD0120F8E44A46002119
:1015F000204601F0A6F90D9858440D901298A0EBE2
:101600000B00129012980028DBD10498401C049023
:10161000069904988842B2D3B8F1030F01D130463D
:1016200000E00898129000BF14991298884201D9DE
:10163000149800E0129883465B4621460D9A16984E
:10164000FFF77FFA28B115B9204600F0E0FC012031
:10165000C5E40D9858440D901298A0EB0B00129021
:1016600012980028E0D100BFB8F1030F02D10C207E
:1016700017900DE01198B0F5803F02D30620179027
:1016800006E0B8F1020F01D1042000E0012017901C
:1016900000BF189800F0080090B911980B90002036
:1016A0000C9023460BA9DDE91602FEF72FFE0190F0
:1016B000019828B115B9204600F0A9FC01988EE4E4
:1016C000002211461698FFF7EBF928B115B920460C
:1016D00000F09DFC012082E415B9204600F097FC43
:1016E00000207CE44E4F204E414D452020202046D6
:1016F00041543332202020004E4F204E414D452092
:1017000020202046415420202020200052526141B8
:1017100072724161F8FFFF00F7B582B01646039878
:10172000019001A800F086FF0546002D02DA0B208B
:1017300005B0F0BD0C4850F825400CB100202070D9
:10174000029810B10020029908700749029841F8E8
:1017500025000EB90020EBE7002202A903A801F042
:10176000F9F807463846E3E7BC0000202DE9F74FBB
:1017700090B0044616461CB9092013B0BDE8F08F9E
:1017800006F03F06324603A911A801F0E3F805462A
:10179000002D75D1039804904FF4007000F031FCD7
:1017A0008346BBF1000F01D11120E6E70398C0F892
:1017B0000CB004A8119900F0FBFC05462DB99DF86A
:1017C0003B0000F0800000B1062506F01C00002858
:1017D00057D045B1042D03D104A8FFF730F80546D2
:1017E00046F008060AE09DF8160000F0110008B166
:1017F000072503E006F0040000B10825002D51D1B3
:1018000006F0080000284DD000F0F7FE01900B997B
:1018100001F10E00019901F0F1FE0B9901F11600A2
:10182000019901F0EBFE0B99039800F049FF814606
:1018300020200B99C87200220B99039801F0CCFE6E
:101840000B9901F11C00002101F0D8FE0120039941
:10185000C870B9F1000F25D00398D0F834A0002249
:10186000494604A801F048FD0546DDB951460398F4
:1018700001F0C6F90546A9F101000399086111E0DC
:101880007BE07DB99DF8160000F0100008B104253A
:1018900008E006F0020028B19DF8160000F00100F3
:1018A00000B107254DB906F0080008B146F0400622
:1018B0000398406B20620B986062002D5AD10B99FF
:1018C000039800F0FDFEA0600B9901F11C0000F0F0
:1018D0000AFFE0600020A062039820600398C0889F
:1018E000A080267400206074E06160614FF4007293
:1018F000002104F12C0001F024F806F0200058B378
:10190000E06848B3E0686061039840894002029053
:10191000A768D4F80C800DE03946204600F0FDFDA4
:101920000746012F00D80225781C00B9012502982E
:10193000A8EB000815B902988045EDD8A7615DB9FC
:10194000C8F3080040B139460398FEF796FA82467C
:10195000BAF1000F01D102250CE00AEB5820E0613A
:10196000E26903994878012304F12C01FFF7C8F8D4
:1019700000B10125584600F04AFB0DB1002020605F
:101980002846FAE630B593B004460D462946684627
:1019900001F0B6FA04E014F8011B684601F078FA89
:1019A00020780028F7D1684601F094FA13B030BDD2
:1019B0002DE9FF4F85B0044615469A46DDF818B06C
:1019C0000020CAF8000003A9204601F0D6FE0490CA
:1019D000049810B9607C049018B1049809B0BDE86F
:1019E000F08F207C00F0010008B90720F6E761695C
:1019F000E068401A01900198854200D9019DA8E055
:101A0000A08AC0F30800002874D103984089401EC2
:101A1000616900EA5129B9F1000F1FD1606910B95D
:101A2000A06802900CE0A06A28B120466169FEF728
:101A30000BFA029004E02046A16900F06EFD0290CE
:101A40000298022802D202206074C7E70298401C64
:101A500010B901206074C1E70298A061A1690398E0
:101A6000FEF70BFA064616B902206074B6E74E443C
:101A70004FEA5528B8F1000F29D009EB0800039967
:101A80004989884203D903984089A0EB0908039942
:101A90004878434632465946FFF732F810B10120E4
:101AA00060749BE7207C00F0800068B1E069801BD7
:101AB000404509D2E169891B0BEB41204FF40072CC
:101AC00004F12C0100F030FF4FEA482737E0E069CD
:101AD000B04220D0207C00F0800080B1E269039900
:101AE0004878012304F12C01FFF72BF818B10120ED
:101AF000607473E710E0207C00F07F00207403998D
:101B000048780123324604F12C01FEF7F9FF10B1A9
:101B10000120607462E7E661A08AC0F30800C0F5A6
:101B20000077AF4200D92F46A08AC0F3080204F123
:101B30002C0011183A46584600F0F6FE00BFED1B87
:101B4000DAF800003844CAF80000BB446069384441
:101B50006061002D7FF454AF00203FE72DE9F34191
:101B6000A2B023A800F066FD022209A922A800F075
:101B7000F1FE0446002C7DD1099816904FF40070B8
:101B800000F03FFA07461FB9112024B0BDE8F081EC
:101B90000998C76016A8229900F00AFB04462CB9E0
:101BA0009DF8830000F0A00000B10624002C6ED147
:101BB000202201A81D9900F0B7FE302216A90AA81C
:101BC00000F0B2FE0AA8239900F0F2FA04465CB9CC
:101BD00018990C98884205D11A990E98884201D11B
:101BE000042000E008200446042C46D10AA8FEF791
:101BF00026FE0446002C40D1119D13220DF1110147
